:020000040000FA
:100000009028002029120000AB6C0000151200009F
:100010001512000015120000151200001512000044
:10002000000000000000000000000000D5130000E8
:1000300015120000000000009513000015120000CA
:100040005D1500005D1500005D1500005D150000E8
:100050005D1500005D1500005D1500005D150000D8
:100060005D1500005D1500005D1500005D150000C8
:100070005D1500005D1500005D1500005D150000B8
:100080005D1500005D1500005D1500005D150000A8
:100090005D1500005D1500005D1500005D15000098
:1000A0005D1500005D1500005D1500005D15000088
:1000B0005D1500005D1500005D1500005D15000078
:1000C0005D1500005D1500005D1500005D15000068
:1000D0005D1500005D1500005D1500005D15000058
:1000E0005D1500005D1500005D1500005D15000048
:1000F0005D1500005D1500005D1500005D15000038
:100100005D1500005D1500005D1500005D15000027
:100110005D1500005D1500005D1500005D15000017
:100120005D1500005D1500005D1500005D15000007
:100130005D1500005D1500005D1500005D150000F7
:100140005D1500005D1500005D1500005D150000E7
:100150005D15000010F8012B11F8013B012A28BFA2
:100160009A42F7D0D01A7047034613F8012B002AA1
:10017000FBD1181A0138704703488368DB6903B163
:1001800018476FF057007047B88C0000024883682A
:100190009B6903B118477047B88C000010B4034640
:1001A00006480A4681680C691CB11946234610BCF2
:1001B00018476FF0570010BC704700BFB88C0000A4
:1001C00010B50F4C204608F07AF8A8B1A3685B6A16
:1001D0000BB120469847FFF7D9FFA3682BB11B6CE2
:1001E0001BB10022074906489847A3681B6A0BB158
:1001F00003489847002010BD6FF01500FBE700BFD3
:10020000B88C0000090200002DE9F04F664D8DB05A
:10021000AB68DB6A23B12846984708B9FFF7ACFF03
:10022000FFF7AAFF58B1614C2368A3B9002200234D
:100230005F4804F07BFB206068B9FFF7A7FFAB685D
:10024000DB6A03BB5B4F5C4D3B78032B1FD8DFE8B9
:1002500003F02134839C2368D9681A8AAB68DB6871
:1002600073B151489847014620680C3006F0A5FD4F
:100270002068068A002EE2D101F05AFC2660DEE7F3
:100280006FF05701F0E7484898470028DAD10DB0E1
:10029000BDE8F08F494C01212046FFF77FFF002881
:1002A000F5D02078431E012B01D90528CCD105F0CB
:1002B000D0FE012328603B70C6E7DFF800B1DFF80D
:1002C00000A19BF8000005F0C4FE2968401A5044C4
:1002D000FFF764FF2B6804461E1A2E60002E50D1D3
:1002E00001230022CDE900B30620002301F08EFD9A
:1002F000DFF8D0908046C9F8000008B93870C6E72A
:100300009BF80000022822D005281BD0012801D12B
:100310009AF802602E6005F09CFE2949024608F119
:100320000C0006F038FDD9F800000C3006F04DFD49
:100330002B6898420ED2D9F8000001F0F9FB032394
:100340003B701EE0BAF80230C3F30D06E2E7BAF8DC
:100350000260DFE70223F3E71A4E296833681A8A3E
:10036000D8681044FFF71AFF31682E680B8A361AD6
:10037000034404460B822E601EB9134808F00FF99F
:100380003E70002C7FF460AF81E7296803A8212923
:1003900028BF2121FFF702FF2B6804461B1A2B60A0
:1003A000002BEED1CCE700BFB88C0000D0090020B4
:1003B0008402002025130020CC09002024130020F3
:1003C00020130020C80900206C02002038B5094D18
:1003D0004FF0FF324FF0FF33284604F0A7FA0446EF
:1003E00001F064FD10B1204601F0A2FB04F05EFFB5
:1003F000EEE700BF6C02002070B5184888B001F02D
:1004000061FD00220023CDE9062300236FF00802DE
:10041000CDE90133CDE9032300934FF48062104B03
:100420001049114804F012FD10490F4808F042F934
:100430000A4D0F4E0F4C4FF0FF324FF0FF3328465E
:1004400004F074FA0146304608F0A9F8A3685B6925
:10045000002BF0D020469847EDE700BF5402002063
:10046000CD030000501300205003002074920000C0
:1004700084020020B88C0000014B1B68184700BFA5
:100480000000002030B585B004460D461022002142
:10049000684608F094FB02238DF80230044B2A468C
:1004A00021466846019305F079FB05B030BD00BFD9
:1004B0007904000080B505460E461746984604F0BC
:1004C00095FF034608F084FB0446DFF81890424687
:1004D00049F8003039463046A84754F8090000F082
:1004E0000BFF00BF080000002DE9F047058B044614
:1004F0002807904611D4022905F0070540F0CC806A
:10050000204606F06DF878B10138218B042811D807
:10051000DFE800F0C2106D85950001290CBF45F0A1
:10052000100545F02005258388F31188BFF36F8FF0
:10053000BDE8F08701F0070AAA4500F0A580002772
:10054000B9463E46A368002B00F0BC8041F008018C
:10055000218388F31188BFF36F8FA168002900F011
:10056000BA800D68002900F0B68033465246204616
:10057000D1F80480C047002D76D02B6829461D464F
:10058000F0E701F007035A1F012A1BD8002221F0CF
:100590000701062B276889B2C4E9002209D13B462E
:1005A00003E0628B013262831B68002BF9D141F0BA
:1005B00002012046218306F013F800287AD041F08A
:1005C000200176E0042B0AD121F0070189B22046F0
:1005D000218306F005F810B141F020012183218B21
:1005E00001F0070AAA454FD00027B946AAE72369B8
:1005F00021F0070141F00601062DD3F80090218378
:100600002DD1B9F1000F3FD041F00801218388F3CB
:100610001188BFF36F8F20463949C84729E021F080
:100620000701236941F0040189B2042DD3F8049035
:100630002183E6D000274FF0040A3E4682E721F0EE
:100640000701236941F0050189B2052DD3F808900F
:100650002183D6D000274FF0050A3E4672E70027D7
:100660004FF0060A3E466DE72B4687E7B9F1000FCB
:10067000D1D1EFF31188202383F31288BFF36F8F5A
:10068000238B23F008032383258BEA062ED525F040
:100690001003238305F007056669218B002EBFF642
:1006A00070AF00232768C4E9003321F0070141F04F
:1006B00001012183218B4FF0000901F0070AAA45AF
:1006C0007FF440AF002F9CD041F00801218388F3D4
:1006D0001188BFF36F8F002FC8D03D68394633466D
:1006E0005246204605F0A8FF2F46F4E7AB067FF5FB
:1006F0001BAF25F02003238305F0070500E700BFAB
:1007000065660000034A13680BB952681360002045
:10071000704700BF0400002030B50C460E4985B07C
:100720000291D0F8D4110546CDE9003100F1F00175
:100730004FF0FF33204603F027FC50B9012384F823
:100740006C30D5F8D03123B1204605B0BDE830403B
:10075000184705B030BD00BFA769000038B50C468A
:100760001146054606F021F9034638B928460449E2
:1007700006F01BF903460020236038BD0120FBE78B
:10078000A29400002DE9F04F0123814605694668D7
:1007900087B005F56377D7E8EF2F002A03D1C7E8C4
:1007A000E13F0029F7D10CBF1A46002240F0B48087
:1007B000B368B16A05F5F8781C1F104606F079F9A0
:1007C000844272D8013A00F0A180B2FA82F24FF06E
:1007D0000044D44072682046073222F00302C5F874
:1007E0008822B16A06F065F9C5F88C02B36A404602
:1007F0006343033323F0030302EB4302230103EBC0
:100800004403093323F0030303EBC403C5F8802238
:100810001A440832C5F87C227368C5F88442C5F8CA
:1008200078323F4BC5E9B363D9F80030C5F82432BC
:10083000316800F0DFF90446002834D1D9F810B04F
:10084000D9F804A0D9F800300BF53A790590049353
:100850004846DAE90734012B08BF103C07F01EFFB9
:10086000DAF824002F4904AB01EB80214FF48062B9
:1008700048460093234604F031FA2B490BF53670B5
:1008800007F0C5FEDAE9050183685C684CB15B4698
:10089000264AA047044630B9DAE9050183681B6996
:1008A0002BB96FF05704002129E0013285E70122BE
:1008B000984704460028F6D11D4B2846C5F8D0318C
:1008C0001C4BC5F8D4311C4B0393D5F83832029336
:1008D000D5F83032CDE90083D5F89032B26AD5F838
:1008E000881300F04FF904460028DCD105F1F00030
:1008F00003F0F0FB0028C5F890030ADB022138461C
:1009000006F087F8204607B0BDE8F08F6FF00B04C3
:10091000C9E76FF01504C6E76FF07704F2E700BF90
:10092000FD69000050170020E3690000D76900004E
:100930003D090000896B0000436A000013B50446BE
:1009400040B100230122CDE90032074BD0E9091262
:1009500003F0CAFA236F1B6823B1606F02B0BDE8D1
:100960001040184702B010BDA294000013B5044611
:100970000846216901F56371D1E8AF1F022910D142
:1009800093B1A0B10121CDE900311346D0E909129C
:1009900003F0AAFA074B984208BF6FF00B0002B0B1
:1009A00010BD6FF00F00FAE76FF04C00F7E76FF043
:1009B0000100F4E72EF8FFFF2DE9F74388461546BE
:1009C000066906F56373D3E8AF3F022B5FD1136866
:1009D00023B96FF0150003B0BDE8F0831B78002B3E
:1009E000F7D0D6F88893B9F1000F33D106F5EC773C
:1009F0004FF0FF324FF0FF33384603F0E3FE30464E
:100A00002A6801A9FFF7AAFE019C1CB9384605F027
:100A1000FEFFDEE705F1080323676B6984F86C903D
:100A20006367646460B1384605F0F1FF21463046E3
:100A3000A36E2A68FFF770FE0020C8F80040CAE7DE
:100A40002022296804F1480008F03AF8384605F0F9
:100A5000DEFFF1E730460F4905F0A7FF0446002806
:100A6000B7D005F1080303676B694064436700234F
:100A700080F86C3020222968483008F021F822469E
:100A80000121304600F060F80028D5D0A1E76FF0D2
:100A90000F00A0E7A294000010B50C46006900F515
:100AA0006373D3E8AF3F022B0FD189B10A4900F538
:100AB000367007F0D8FD204607F039F9782200217A
:100AC000204608F07CF8002010BD6FF00F00FBE717
:100AD0006FF00100F8E700BFD40900202DE9F04FC6
:100AE00005460E4690460027D0F8C4A085B0AAF56A
:100AF000BE7421463046FFF72DFBE0B9114BA4F13F
:100B0000480B0293DAF810303246CDE900832946CB
:100B10004FF0FF335846AAF5E27903F035FA60B991
:100B20007823012203FB079383F86C20DAF80C305A
:100B30000BB158469847783417B105B0BDE8F08F2F
:100B40000127D6E7B76B00001FB5144690B18AB1F4
:100B5000012912D10A4B00F1F0010293D0F8D431EF
:100B6000483201934FF0FF332046009303F00CFA14
:100B700004B010BD6FF01500FAE70020F8E700BFE1
:100B8000B76B00002DE9F04387B00E46DDE90E811A
:100B90001446DDE910251F4630B329B3DFF850C0F5
:100BA00000F1F009002D08BF65469EB9CDE9034468
:100BB00000F5E2742046059607F053FB03ABCDE940
:100BC00000432A463B464146484603F0FDFA07B03B
:100BD000BDE8F083002241460E9248462A4607B0FF
:100BE000BDE8F04303F046BC6FF01500EFE700BF2F
:100BF000DD0A0000F0B50E46044689B0002872D028
:100C0000436B0BB9394B436301232246E363002353
:100C1000D4F8981004F1400042F8301FCDE90133B8
:100C20004FF0FF330093D4F89C3006F054FD304A67
:100C300006AB92E8030083E80300184603F05AF875
:100C40000546D8B904F1340003F036F80546A8B9D2
:100C5000616B284805AA06F01AFD054670B9059B88
:100C60009A6872B10C33D4F89400C4F8A03005F03F
:100C7000D3FFC4F8D40030B96FF00B05284609B093
:100C8000F0BD0346EFE7D4F8940005F0C5FFC4F8C3
:100C9000D8000028F0D0D4F88C30D4F8A010C4F8D4
:100CA000A8300423C4F8AC30C4F8C4300223A362D3
:100CB000114BB4F89420D4F8D470C4F8B810C4F828
:100CC000D010D4F89010236204F1A403A4F8B0204B
:100CD000C4F8A470C4F8C010A4F8C820C4F8BC00BC
:100CE000A661E362CAE76FF01505C7E780920000CE
:100CF000308F00008A920000848F0000014B036057
:100D000000207047B08F000008B5044805F05BFC78
:100D1000BDE80840024805F056BC00BF92920000B2
:100D2000C7920000014804F0F7BD00BFB08F00007B
:100D300038B5044618B90F4B0F485B68984761688F
:100D4000B1F5683F10D0B1F5680F0DD00B4DA94239
:100D50000AD011F46861206807D00146084807F0FE
:100D60006EFB00232360656038BD142207F027FF67
:100D7000F9E700BF80010020F59200002C5F5CA91C
:100D8000FC0E002008B560B34368B3F5683F0ED091
:100D9000B3F5680F18D0144A934220D000684FF082
:100DA000FF324FF0FF3303F00DFD58B115E0012283
:100DB0000368D3E8EF1F002903D1C3E8E02F002820
:100DC000F7D10AD1002008BD0368084A1B7803F553
:100DD000807352F82330002BF4D00548F3E7054820
:100DE000F1E76FF4E040EEE72C5F5CA900000350F0
:100DF000E98FFFFFEA8FFFFF08B520B34368B3F523
:100E0000683F09D0B3F5680F13D0114A93421DD043
:100E1000006803F04FFD14E000220368D3E8EF1FE1
:100E2000012903D1C3E8E02F0028F7D109D00948F0
:100E300008BD00210368084A1B7803F5807342F857
:100E400023100020F4E76FF4E040F1E70348EFE7F8
:100E50002C5F5CA9E98FFFFF00000350EA8FFFFFC2
:100E600010B5044618B91D4B1D485B689847636868
:100E7000B3F5683F2FD0B3F5680F2CD0194A9342D1
:100E800019D1236803BB4FF0FF324FF0FF332146E7
:100E9000154803F069FC08B923681BB90F4B1348C8
:100EA0005B68984714220021206807F088FE4FF401
:100EB0006863636008E0B3F5683F0DD83A2B03D050
:100EC00040F6BA629342DED1206807F0F0FA636818
:100ED00043F03A03636010BD054AF3E78001002048
:100EE000F59200002C5F5CA9FC0E00201B93000013
:100EF0003A00003A08B5064940231422054807F095
:100F000090FABDE808400449044804F077BD00BFEA
:100F1000FC090020FC0E0020B88F0000CC8F0000E0
:100F200030BFFFF7FDBF00BF2DE9F04105460B4E76
:100F3000DFF82C80324606EB0807CC1B2046094917
:100F400007F030FEA01942460021083C07F037FEAA
:100F50006C6707F10800BDE8F08100BF00000000E9
:100F600004000000308F0000074A936893F90E10C8
:100F7000002907DB526993421FBF044A536843F0BC
:100F800080535360704700BF1011002000ED00E057
:100F9000154B9A6A12F0007F9A6A14BF1E201D201A
:100FA00012F0807F9A6A18BF1F2012F4801F9A6A7D
:100FB00018BF022012F4002F9A6A18BF212012F4E1
:100FC000802F9A6A18BF222012F4003F9A6A18BF35
:100FD000232012F4803F9A6A18BF24206FEA02424D
:100FE0006FEA12429A62704700ED00E010B5194BAB
:100FF0000246986A9C6A10F4805F14BF172016207E
:1010000014F4006F9C6A18BF1820A40509D5986BCA
:10101000986A000404D51AB19A6A22F400429A62CE
:1010200019200C4B9A6A12F4806F9A6A18BF1A2022
:10103000D2050CD49B6A13F4005F18BF1C20054A2C
:10104000936A43F47F43936200230B7010BD1B200F
:10105000F5E700BF00ED00E010B51C4B0246986AB2
:101060009C6A10F0100F14BF1120102014F0080F0C
:101070009C6A18BF1220A40709D5586B986A00060D
:1010800004D51AB19A6A22F080029A6213200F4B9B
:101090009A6A12F0010F9A6A18BF142012F0200FFA
:1010A0009A6A18BF1520D40658BF9B6A074B9A6AE4
:1010B000920642BF5A6A22F400525A629A6A42F079
:1010C000FF029A6200230B7010BD00BF00ED00E02C
:1010D000F0B5474B04465B6800258BB0C3F30803AB
:1010E00085F31188BFF36F8F02F07F40B0F17F4F1F
:1010F00011D102F00C0008280DD010074CBF0C468F
:1011000001250022033B8DF80720032B05D8DFE8DB
:1011100003F02462665F2C46F3E700239DF8072066
:10112000CAB902AE04F1200732462068616808346B
:1011300003C2BC421646F7D1099A002D53D0C2F320
:10114000080121B96FEA52226FEA42220992184639
:1011500002A905F0A0FD0BB0F0BD254BDA6A91079E
:10116000DBD4DA6A002AD8DBDA6A5200D5D55A69AC
:10117000A16942F480725A61BFF34F8FBFF36F8F42
:101180005A6931F8021C22F480725A61BFF34F8F02
:10119000BFF36F8F4DF60272914209D09A6AD2B2B4
:1011A00042B101200DF10701FFF756FF0346B5E7F5
:1011B0002368B3E79A6A12F47F4F05D001200DF13E
:1011C0000701FFF713FFF1E79B6AB3F5803FA4D354
:1011D000FFF7DEFEEAE700200DF10701E4E700205B
:1011E0000DF10701EDE722F4FF7222F00102ADE7F5
:1011F00000ED00E0064B5A6942F010025A615A694C
:1012000042F480625A615A6922F008025A617047BA
:1012100000ED00E0EFF30880EFF3098101B57246BD
:10122000FFF756FF01BD00BF002080F31488BFF315
:101230006F8F002080F30A8880F30B8801F046FE50
:1012400000200E490860BFF34F8F0D4880F30888D7
:1012500000F02CF8202080F311880A484FF4006138
:10126000401880F30988EFF314800221084380F3CB
:101270001488BFF36F8F00F003F9000094ED00E0D5
:1012800090280020501B0020002318460649D1F862
:101290009020C2F30722934200DB7047C1F89830D8
:1012A000C1F8A0000133F6E700ED00E010B572B61A
:1012B000002484F31388FFF7E7FF23464FF0FF3045
:1012C0000C4A03F120010133102B42F82100F8D120
:1012D00000234FF0FF30074A03F160010133102B68
:1012E00042F82100F8D162B6BFF34F8FBFF36F8F82
:1012F00010BD00BF00E100E0084B9B6883420BD1AA
:10130000EFF3058343B1064B5A6842F080525A60AE
:101310005A6A22F400425A6207F0A0BA1011002063
:1013200000ED00E06FF00A01084A9368D9670849A8
:1013300098674B6843F080534B60002383F3118818
:10134000BFF36F8F9368D86F704700BF10110020F4
:1013500000ED00E0EFF31183202383F31288BFF345
:101360006F8F4FF00061084A53699360074A5160DC
:10137000596F074A116000219A6F996782F31188AB
:10138000BFF36F8F704700BF1011002000ED00E029
:10139000180F00200E498A684FF030001044EFF318
:1013A000098C80E8F01F74467046FFF7D3FFA6460D
:1013B00007498A6802F1300090E8F01F8CF3098831
:1013C00002F1000004B505F07BFCBDE80440704765
:1013D000101100201EF0040F0CBFEFF30880EFF394
:1013E0000980816911F8021C0229FFD001B505F0BE
:1013F00058FC01BD40B2002807DB01234109034A24
:1014000000F01F00834042F82130704700E100E007
:1014100040B200280CDB01220649430900F01F00FE
:101420008240203341F82320BFF34F8FBFF36F8FEB
:10143000704700BF00E100E0054B420953F822204D
:10144000012300F01F0003FA00F01040704700BFB6
:1014500000E100E040B2002801F10101ACBF00F161
:101460006040064B4FEA4111C9B2ABBF00F5614085
:1014700000F00F0080F800131954704714ED00E0DD
:101480000B4A08B50B4B22F07F029A60BFF34F8FD7
:10149000BFF36F8FD3F8882022F47002C3F888203E
:1014A00003F08EF804F040F800F04CF803F0C8F8B0
:1014B0000000000000ED00E042F8203C009B0B49DA
:1014C00042F81C3C019B21F0010142F8183C029BB0
:1014D00042F8081C42F8143C4FF0807342F8043C78
:1014E0000023203A02658367704700BFB5040000FF
:1014F00000B50D4B15469860426F0C4B0E461A60B6
:10150000436E83F30B882C4686F309884FF0000066
:10151000074B984720464FF000014FF000024FF074
:101520000003044C204700BF10110020180F0020BA
:10153000C96C0000B50400001022014B1A6170470D
:1015400000ED00E0002320210348C2180133452BA1
:1015500082F80013F9D1704700E100E008B5EFF31D
:101560000583064A103B02EBC30152F83300496879
:101570008847BDE80840FFF7F7BC00BF088D0000B2
:101580001FB5094C094A23460121094800F0FAF821
:1015900000230393074B0121E41A01A8019302944D
:1015A00000F0FAF804B010BD000007200000002091
:1015B000DC8F00005003002010B50C7A0B6804F09B
:1015C0001F0223F01F031A43CB68640923F01F0393
:1015D000054943EA440343F00103C1F89800C1F808
:1015E0009C20C1F8A03010BD00ED00E010B5074B05
:1015F000D3F89030C3F30723013B984202D8FFF79A
:10160000DBFF10BD6FF01500FBE700BF00ED00E051
:101610002DE9F04F0F46144606464FF000084D4D99
:1016200085B0B84580F29280D6F80490B9F1000FE9
:1016300036D0B9F11F0F40F2878019F01F0F40F02C
:101640008380D6F800A01AF01F0F7DD1504605F018
:1016500077FB834609EB0A00013805F071FB8345EF
:1016600072D11BF1160F6FD05C456DDDC5F898B0D7
:10167000D5F89C10C5F898B0D5F8A03021F01F011E
:1016800043F01F0AD6E900321A44994202F1FF39A9
:101690001ED1CA4508D131465FFA8BF005F059FBDF
:1016A00008F101080C36BCE73146C5F898B0D5F80A
:1016B0009C3022F01F0203F01F031343C5F89C3037
:1016C000E0B205F046FB10F1160F3DD0441CE7E7F1
:1016D000C5F898B0D5F8A020013B23F01F0302F015
:1016E0001F021343CA453146E0B2C5F8A030E8D026
:1016F00005F02FFB10F1160F26D0C5F898B0D5F8DD
:101700009C209DF808300AF1FF3A62F304038DF83B
:101710000830D5F8A0309DF808205B0863F3471225
:101720008DF80820D6E900321344009323F01F03FC
:101730005344A3EB0903013023F01F036946C0B2F1
:101740000393FFF753FFBEE76FF01504204605B083
:10175000BDE8F08F00ED00E00522044BC3F89420B3
:10176000BFF34F8FBFF36F8F704700BF00ED00E0F6
:10177000BFF35F8F0022024BC3F89420704700BF75
:1017800000ED00E010B5034C2278FFF741FF207018
:1017900010BD00BF261300202DE9F74F294D8A46C2
:1017A00006464FF00008AB46274FD0451BDAD6F867
:1017B0000490B9F1000F3FD031680846019105F05F
:1017C000BFFA0199044609EB0100013805F0B8FAA7
:1017D00084424FF014021D4B08D002FB08F36FF057
:1017E00015024BF8032003B0BDE8F08F14F1160F7B
:1017F0002C60F8D01978A142F5DD02FB08B0C7F8DB
:101800009840C7F89840D7F89C4000F10801007B49
:1018100064F304000871D7F8A0000C79400860F365
:1018200047140C71D7F89C1021F01F016960D7F89C
:10183000A01021F01F01296108F1010814350C36B0
:10184000B3E700BF1C0F002000ED00E026130020CE
:10185000F0B54149414CD1F890302568C3F30723D6
:101860009D4287B075D80020FFF782FF3C4BC1F83E
:10187000C030854216D13B4C01A82570FFF73EFAD7
:1018800000250646384FAE4213D100202378324956
:10189000D1F89020C2F30722934254DBFFF75CFF9C
:1018A00000202FE0616801EB0011FFF785FE013099
:1018B000DFE70199280101EB0513DA683A40B2F538
:1018C000001F21D0B2F5800F2BD0B2F5801F38D188
:1018D0005A689B680958013B22F01F00034401200D
:1018E000844623F01F0340EA4C10CDE902218DF815
:1018F000100002A920780593FFF778FE00281DDA72
:101900006FF0150007B0F0BD5A689B680958013B9D
:1019100022F01F0003444FF0020C012023F01F03AC
:10192000E1E75A689B680958013B22F01F00034415
:101930004FF0000C062023F01F03D4E72378013377
:10194000237001359FE7C1F89830C1F8A00001333A
:101950009EE74FF0FF30D5E700ED00E0E88F000094
:10196000AAFF4400261300200000F0FF08B5064936
:10197000064821F00701C1F1005202F5E02204F00F
:10198000C8FD002008BD00BFF3600020300F00201C
:1019900070B541690446867A0A4D59B1437ADB072E
:1019A00006D42C2303FB06535B6A1B689B6898478D
:1019B000002363612C20214606FB0050BDE87040E7
:1019C00006F0F8BD9C0200202C21827A054B01FB19
:1019D00002339A6A1B7F801A1B3323F00303B0FB88
:1019E000F3F070479C02002038B52C24827A064B15
:1019F00004FB02335B6AD3E901240C601568FFF72E
:101A0000E3FF04FB005038BD9C0200202DE9F04F9D
:101A100085B00546684691461C4690469A46039115
:101A200006F079FFDDE90067EFF3118B202383F3E4
:101A30001288BFF36F8F698B002942D02B8B8B42AA
:101A400026D900220023284602F070FF0446F8B190
:101A50008BF31188BFF36F8F039B002B4FD032465F
:101A60003B46684606F07BFF2C21A27A2C4B204691
:101A700001FB02335B6A03A91B681D68DDE90023D3
:101A8000A847606100283BD12046FFF781FF31E085
:101A9000698B4B1E6B838BF31188BFF36F8F2B7F8A
:101AA0002A8BAC6A1B3323F00303521A02FB034454
:101AB0001B4B1C4AEB1A9B105343A3722B7FE37200
:101AC000CAE78BF31188BFF36F8F54EA090409D07A
:101AD00007F07EF8144A154B12589A420ABF8846FE
:101AE000C846C24642465346284602F01FFF0446F7
:101AF0000028B1D10024204605B0BDE8F08F636115
:101B0000012300252381039B29466382E27A6560D5
:101B100004F1180007F053F863692582E360EAE7EF
:101B20009C020020A38B2EBA080000008808002029
:101B300070B52C250B4C00B970BD037A4668013B8B
:101B4000DBB20372002BF7D1C3604360837A05FBDD
:101B500003431B6A13B198473046ECE7FFF718FFC1
:101B6000FAE700BF9C02002000F01F0240090DD0E0
:101B700001280DD1094B03EB8203D3F8002222F098
:101B8000E04242EA0171C3F800127047044BF2E7E9
:101B90000023803253F82230FFDE00BF002884503B
:101BA0000025845038B50124134B144DC3F800456B
:101BB00002230321C5F8D0360020FFF7D5FF2046C9
:101BC0000321FFF7D1FFC5F804472146C5F80449B2
:101BD0002120C5F8004BFFF7C7FF21462020FFF763
:101BE000C3FF21460B20FFF7BFFF21460A20FFF766
:101BF000BBFF002038BD00BF001000500040005067
:101C000007B50DF1070005F00DFC114B98421CD1F2
:101C10004FF480620F4B1049C3F8B8254FF40062AF
:101C2000C3F83C259DF8070005F0F0FB0B499DF833
:101C3000070005F0E6FB01209DF80730984001F011
:101C400063FA002003B05DF804FB6FF00B00F9E7C6
:101C50000000AD0B00A002502CA0025028A10250A1
:101C6000052370B5144D154E2C780134B4FBF3F3F5
:101C700003EB8303E41A05F0B2FB114A137823B196
:101C800056F82430C01A072814D94FF05023D3F83F
:101C9000141141B10021C3F81411D3F814312C7080
:101CA0000CB9012313702C7805F099FB46F8240039
:101CB000012070BD0020FCE7281300203C0F00200D
:101CC0002713002048B1054B054A1B68B3FBF2F30C
:101CD0005843044B43F0010318477047C0000020ED
:101CE00040420F00508F00000149024804F0C7BC79
:101CF0001C900000500F00204FF47F032DE9F041AD
:101D0000D3F830210646072A0D46D3F8343120D1C6
:101D1000023B032B02D8124AD35CD3B14FF05024BC
:101D20004FF0010800270520C4F81886C4F814767F
:101D300005F065FB4046C4F8148605F060FBC4F866
:101D40001476C4F8187630462B46BDE8F0410021E1
:101D500018474FF050230022C3F81426F3E700BFC2
:101D6000579300001FB578B100230193039301231B
:101D700069460848029304F095FC029B9B0700D13A
:101D8000039B05B05DF804FB024805B05DF804EB69
:101D900004F0DFBC500F002010B50E4B0C461B7832
:101DA000012B0BD1097E03290FD0052902D001296F
:101DB0000DD1042104F10C0004F0F6FF064B21467E
:101DC000186806F0ECFB002010BD0221F2E76FF06E
:101DD0001500F9E7E00100206C0F0020052838B558
:101DE000054608D82A21C140C90704D5064804F091
:101DF000CAFF044610B90024204638BD01210C302A
:101E000004F0C5FF2576F7E7200300202DE9F04117
:101E10000446DDE90667062829D8DFE800F0042833
:101E200036281B281D001D4804F0ADFF0546F0B103
:101E300000F10C080121404604F0A9FF2C76BEB148
:101E4000B7B1404604F0C1FF874220D92846FFF7CA
:101E50006FFE0CE01248E7E712490978012906D124
:101E60003478022C07D0052C09D0012C0AD000258B
:101E70002846BDE8F0810C480136013FD4E7042430
:101E80000748F9E700240548F6E70748CCE73A4653
:101E90003146404604F07FFFEAE700BFC802002059
:101EA000F4020020E00100209C020020038A014689
:101EB00023B1034B186883689B681847122070474A
:101EC0005000002010B5084B084C1860206806F040
:101ED000F6F930B1206806498368BDE810401B68F8
:101EE00018476FF0120010BD6C0F0020500000204A
:101EF000991D00002DE9F74F064600780D4604288D
:101F00009246D2F810B001F1FF3325D0052873D0E6
:101F100002284AD1032B48D9002200230320FFF7CF
:101F20005DFF0446002840D00422D6F8013000F1BD
:101F30000C0738460DEB0201019304F02CFFBDF8AD
:101F40000630053D9D4246D1384604F03EFF8542AD
:101F500041D82A46711D44E0012B26D973783E2BC7
:101F600028D1F378022B23D00D2B23D13379012BE9
:101F700020D1B6F80570C7F30017B6F80130033D5D
:101F8000B5EB132FADF804300FD1AFB14FF000080F
:101F90004FF0000942464B4639469DF8040004F0D4
:101FA00024FF044658B9002FF4D003B0BDE8F08FE9
:101FB0000127E2E70027E0E74FF4A028E8E700F177
:101FC0000C07022201A9384604F0E5FE384604F069
:101FD000FCFE854203D92046FFF7AAFDE5E72A4625
:101FE000F11C384604F0D7FE21465046DBF800309D
:101FF00003B0BDE8F04F1847032BD6D900220023C9
:10200000FFF7ECFEDFF83880044698B10422D6F8DA
:10201000013000F10C0738460DEB0201019304F08A
:10202000BAFE0023C8F80030BDF80630053DC3F302
:102030000D0387E7D8F800300133C8F80030B4E763
:10204000700F0020102208B5034B0120C3F8402474
:10205000FFF788FE002008BD00300050084B70B527
:10206000C31A0D4607499B100446594340220648AF
:1020700004F01DFF2B4601462046BDE8704018477E
:10208000880F0020B76DDBB67C8C0000402373B551
:102090000B4C0093041B0B460D460A49A4106143E8
:1020A0000646094A094804F02EFF011E05DA3046AB
:1020B0002B4602B0BDE87040184702B070BD00BFAB
:1020C000880F0020B76DDBB6716F00007C8C0000BC
:1020D00010B5EFF31184202383F31288BFF36F8FC1
:1020E000074A136823F00201DB07116002D40120C4
:1020F00005F04BFA84F31188BFF36F8F10BD00BF5A
:10210000281000202DE9F84300220321064605206F
:10211000FFF7A0F9114800F0FDFF114B984219D1CB
:1021200001F008F800244FF01C090C27DFF8348078
:102130003569414609FB045004F0A1FA002807DB89
:10214000012307FB04551C44042CAB67F0D100208D
:10215000BDE8F8836FF00400FAE700BF69220000D1
:102160000000AD0B749000007FB500220123CDE983
:10217000022304ABCDE90433094A6B46CDF800D005
:10218000CDF804D004F0EDFE002805DB4FF48042CA
:102190000023684602F020FC07B05DF804FB00BF96
:1021A000A76F00000C22104B014602FB00330020F9
:1021B00030B4D3E91C521867EFF31180202484F364
:1021C0001288BFF36F8F9C6F04F0C00444F00204C8
:1021D0009C6780F31188BFF36F8F1DB12B4630BC15
:1021E0000248184730BC7047880F00207C8C0000E4
:1021F00010B4EFF31182202383F31288BFF36F8FA3
:102200001748016841F002040460C80707D482F34C
:102210001188BFF36F8F012010BC00F0A3BF4FF0F7
:102220005021D1F80C04D1F80C14C907EFD5EFF305
:10223000118083F31288BFF36F8F0A498B6F03F00D
:10224000C00343F002038B6780F31188BFF36F8FE5
:1022500082F31188BFF36F8F002010BCFFF7A2BF7D
:1022600028100020880F0020062812D8DFE800F090
:10227000040F1111110D0B00064B986F10F00700A1
:1022800007D1FFF78FBF0220FBE70320F9E701200A
:10229000F7E77047880F00202DE9F041012207463B
:1022A0003649D1E8EF3FC1E8E02F0028F9D133B932
:1022B000334934484B60CB608A6004F0F3F97B1EED
:1022C000012B2BD8012F07D14FF05023D3F81C340A
:1022D00003F00303022B21D006F0E6F90546F8B916
:1022E000294B1B78E3B14FF0502302220646C3F876
:1022F00008234FF05024DFF89480D4F81824D4F841
:102300001834D20315D503F00303022B01D0012F9B
:102310000FD16DB386F31188BFF36F8FBDE8F081E5
:10232000EFF31186202383F31288BFF36F8F01250B
:10233000DFE7C5B1304604F0E7FCD4F81835DBB26E
:10234000012BDAD1D4F80421002AD6D00022C4F817
:102350000421D4F804210222C4F818252022C8F848
:102360008021A360C9E70021212003F021F8E4E7E0
:102370004FF050230222C3F80423CFE7840F00203C
:10238000740F0020A40F00204B13002000E100E098
:10239000F0B5406801F01F04057B87B044EA45149E
:1023A0000569002D63D0B2F5001F00F1100506D1BC
:1023B0002146284605F069F9002007B0F0BD002746
:1023C000B2F5800F01AE0197776039D1B3F1007F8C
:1023D00014BF052304238DF804300023CDE90463E2
:1023E0000393836823FA01F111F001011AD1B2F1CC
:1023F000A07F17D104F01F03620903F180032AD0E4
:10240000012A3AD11E4A52F82330DB070AD40DF1D3
:10241000030632462146284601F0C8F9194B984276
:102420001BD002962146284603AA01F07BF8164BE2
:1024300098421FD101222146284601F019FABBE734
:10244000B3F1C06F05D0B3F1007F14BF01230223A5
:10245000C1E70323BFE70D4AD5E73146284601F01F
:1024600001FA094B9842DCD06FF00B00A5E76FF042
:102470008500A2E76FF015009FE751F82330FFDEDB
:10248000002884500400AD0B0000AD0B00258450E3
:1024900038B545682B69B3B11035284601F0D2F93B
:1024A000044680B90146284601F09AF9084B984243
:1024B0000BD122462846074901F072F92246052130
:1024C0000D20FEF7C7FF002038BD6FF00400FBE7CA
:1024D0000000AD0BD92400004209034670B502D0BC
:1024E000012A17D070BD0D4E326951680029F9D00C
:1024F000012503F01F030C689D400029F2D08A6873
:102500002A4002D030464B6898472CB123682146B8
:102510001C46F2E7024EE7E72346F8E7A48C0000EA
:10252000908C00002DE9F04340F206354668D00655
:1025300048BF0320337B02EA050558BFC2F34010B1
:1025400087B001F01F07B5F5837F144647EA4317AC
:102550008DF8030044D00FD8062D18D007D8B5B198
:10256000022D3FD06FF0150007B0BDE8F083B5F540
:10257000807FF7D101250AE040F20222954233D054
:10258000B5F5407F32D0B5F5007FEBD102250123B0
:10259000220303FA01F12BD573689960326972BB8B
:1025A00007F01F037F0928D0012F75D13C4A02EBA9
:1025B000830284F48033D2F80012C3F30043C4F3DF
:1025C000404444EA430421F4706144EA800421F069
:1025D0000F0144EA05230B43C2F800320020C3E791
:1025E0000725D4E70425D2E70525D0E70325CEE764
:1025F000630344BF7368D960D0E72A4AD7E710362F
:10260000394630460DF1020201F0D0F814F4403F93
:1026100080460CD13946304605F035F8224B9845B6
:10262000DCD130469DF8021001F016F9D6E74FF0E4
:10263000000901AB3946304603AACDE90439CDE99A
:102640000199CDF80C9000F06DFF174B984289D19D
:1026500014F4003315D09DF8033084F48034C4F3AF
:1026600000448DF80E3039464B46304603AA8DF8AB
:102670000C508DF80D4001F011F80B4B9842CDD065
:1026800070E7CDE9043339460DF10303304603AA60
:10269000039300F047FFF0E7803352F82330FFDE6A
:1026A00000288450002584500000AD0B10B504466E
:1026B0000269A2B0C2F880001649002001F00AFAAF
:1026C000002203212A20FEF7C5FE8422002101A852
:1026D000646806F074FA0023012001AA61680432DC
:1026E000D940C90744BF00FA03F142F8041C21682D
:1026F000D940C90748BF00FA03F103F1010348BFFD
:10270000D163102BEAD101A801F0FCF9002022B01E
:1027100010BD00BF47700000036803F01F025B0993
:10272000026004D0012B034818BF00207047024804
:10273000704700BF00288450002584502DE9F04FD9
:102740001546834640F2FF18DFF88891DFF888A12C
:1027500085B000EB8101594503D1002005B0BDE8EB
:10276000F08FDBF80030C3F3C322082AC3F3080458
:1027700000F2AA801B0E444508BF4FF0FF3419F841
:102780000270222B00F2A380DFE803F012191F224F
:10279000252B22A1A1A1A13A67A1A1A1A1A1A1A13B
:1027A000A1A16A7F8285A1A1A1888F9295989B00A3
:1027B000C5F80C45601C5DD10BF1040BCBE7C5F8E7
:1027C0001445621CF8D000265DE0C5F80845F1E725
:1027D000C5F81045F5E7631CC5F80845ECD00026A0
:1027E00004E0661CC5F80C45E6D0012603A8039456
:1027F000FFF792FF0122039B02FA03F3C36008E094
:10280000C5F80845002FDCD1631CD5D0002606276B
:102810003246DBF80030039403F40040002818BF70
:10282000002203A818BF012601930092FFF774FF4E
:10283000039C019B00EB8400D0F80042C3F3412CC1
:10284000009A3B0243EA8C03134304EA0A0423433D
:1028500043EA4603C0F80032AEE7C5F80C45D1E7BD
:10286000C5F86045601CDBF80030A5D0C3F3004319
:10287000002BBAD0012603A80394FFF74DFF039B5A
:1028800006FA03F383603246C3E7C5F86445E9E717
:10289000C5F86845E6E7C5F86C45E3E7C5F82445A3
:1028A000621C89D001260022B3E7C5F8284581E7DC
:1028B000C5F83045F4E7C5F83445F1E7C5F83845C3
:1028C000EEE7C5F83C4575E76FF0150046E76FF099
:1028D000850043E7A0930000F0F0FCFF2DE9F041F4
:1028E00004460D46476805F0DFFE4FF0200888B922
:1028F000264B1B7873B16426606804F0CEFCF0B9F7
:10290000012004F07CFD013EF6D10021212002F0DF
:102910004FFDF0E7EFF31186314688F31288BFF3DD
:102920006F8F606804F0B9FCA8B986F31188BFF313
:102930006F8FEFE786F31188BFF36F8FE5E7EFF353
:102940001186314688F31288BFF36F8F606804F0F8
:10295000A4FC0028EED0FB6900201D706368FA69B2
:102960001B68C3F844250122C3F84825C3F8200199
:10297000D3F82041C3F85801D3F858019A6081F385
:102980001188BFF36F8FBDE8F08100BF4B130020AB
:10299000F7B50546002203210820FEF75BFD08205D
:1029A000FEF728FD6B681A691868C0F82425997D20
:1029B0005A7D0A43198B1B7D0B431343C0F86C35BA
:1029C0006E68D6E9004313F0010348D02F6907F180
:1029D0000C0004F027FD304B98425AD1387B04F1AB
:1029E0000C0204F5907104F016FD387B012707FAFC
:1029F00000F000F089FB0823C4F80035F369C4F83F
:102A000044350023C4F84835A760D4F85831002B6A
:102A1000FBD00021C4F800156B6801AADC682046D1
:102A200004F084FB002805DB019B226819791868F3
:102A3000FFF784FE08216A681368C3F80015117A4D
:102A400051B9126AC3F834250122C3F83825C3F8F6
:102A50001011D3F810111A60002003B0F0BD082245
:102A6000C4F80025F269C4F84425C4F848350123A8
:102A7000A360D4F82031002BFBD00023C4F8203110
:102A8000D4F820310123E3604FF48073C4F8043399
:102A9000BBE76FF00400E0E70000AD0B01238340CB
:102AA00070B5DC430B4AD2E8EF1F01EA0405C2E827
:102AB000E65F002EF7D14FF4803282400648C0F81E
:102AC0000823BFF35F8FBFF36F8F0B4214BF01204A
:102AD000002070BDD01000200050015070B40E498D
:102AE00022F07F46D1E90034D01AC31844F1000423
:102AF000C1E90034A6F50013B3F5400F09D2074B26
:102B00001B681A0A1B069C19054B42F10005C3E914
:102B1000004570BC02F0E2BD78070020D410002010
:102B200080070020D9B101230D4A8340D2E8EFCFBE
:102B30004CEA030CC2E8E1CF0029F7D14FF480330F
:102B4000084A8340C2F80433074BD3E8AF3FC34081
:102B5000DB0742BF4FF40012044BC3F8002170475B
:102B6000D010002000500150CC10002000E100E007
:102B70000D4B1868010A0006BFF35F8F0B4BD3F8AB
:102B80000435181841F10001B3F5801F0AD2084B33
:102B9000D3E90023904271EB030303D210F180705C
:102BA00041F10001704700BFD410002000500150D7
:102BB000800700202DE9F04F85B016461F460446D9
:102BC0009DF840A0FFF76AFF0190FFF7D1FFB042E8
:102BD00071EB070352D23B4B301A67EB010198426D
:102BE00071F100014DD2384B03EB0413D3E90223FA
:102BF0009F4208BF964258D04FF48038334908FAB4
:102C000004F8204626F07F4BC1F8488304F0DBFB34
:102C10004FF00309584604F15005AD00ADB205F17F
:102C2000502504F5A87305F580350293029A20F02B
:102C30007F4341F82230C1F84483D1F80435244A57
:102C4000C01A033820F07F4090422ED9286868B11E
:102C5000D1F80435A3EB0B0020F07F40B0F5000F56
:102C6000039322D9204604F0AEFB039BBAF1000F78
:102C700007D109EB030009F10109D7E7BAF1000F09
:102C800009D06FF0150520460199FFF74BFF284644
:102C900005B0BDE8F08F01230E4AA340D2E8EF0F44
:102CA0001843C2E8E10F0029F8D107490E98230123
:102CB000C8500F9B01EB04120025C2E90267536064
:102CC000E1E700BF010080006807002000500150CC
:102CD000FDFF7F00CC1000207FB500254FF0FF30B6
:102CE0004FF0FF31194C1A4B0226C4F80833C4F8D0
:102CF0004833184BC4F80855C3E902014FF4803338
:102D00004FF40012C4F80433134B0321C4F80463D6
:102D10001520C3F880212A46FEF79CFB1520FEF7FC
:102D200069FB01230D4AA360236013600C4B0D4A1D
:102D3000009328460023CDE90155FFF73BFF3046BD
:102D4000FFF7AAFA284604B070BD00BF005001503A
:102D500003000F006807002000E100E0D010002011
:102D6000DD2A0000FFFF7F002DE9F7432E4BD3F84B
:102D7000042390070BD5D3F8042142B10022C3F8F5
:102D800004212A4AD3F80431136801331360264A18
:102D9000D2F80433D90326D5254BD3E8EF1F21F011
:102DA0000100C3E8E40F002CF7D1CB0702D4D2F81E
:102DB0004031C3B100251C4CC4F84051D4F8403117
:102DC000FFF7D6FEEFF31182202383F31288BFF3BF
:102DD0006F8F184BD3E90267B042B94106D282F334
:102DE0001188BFF36F8F03B0BDE8F0834FF0FF3859
:102DF000D3E900104FF0FF391D60C3E902894FF499
:102E00008033C4F84833C4F84051D4F8403182F3D9
:102E10001188BFF36F8F0029E5D0009032463B4602
:102E200028468847DFE700BF00500150D41000203B
:102E3000CC1000206807002030B5431C124C85B030
:102E400005D08442A8BF0446012CB8BF0124FFF777
:102E50008FFE0E4B0C4DD3E90013401AB0F5000F56
:102E60000FD22218AA4228BF2A4600205218084929
:102E7000CDE90100009143F10003FFF79BFE05B08F
:102E800030BD2A46F1E700BFFFFF7F007807002032
:102E9000DD2A000008B5FFF76BFE024B1B68C01A65
:102EA00008BD00BF780700204FF47F03D3F830211E
:102EB000D3F83431072A05D1023B032B02D8024A4A
:102EC000D05C704700207047BB93000008B5FFF747
:102ED000EBFF58B1644BD3F8202A3AB90D21C3F85F
:102EE000201A0121C3F81C19C3F81C290022D300A1
:102EF00003F57F03D3F80013013107D0D3F8001393
:102F00000132D3F80433202A0B60F0D1FFF7CCFF55
:102F1000002840F0A080FFF7C7FF40B1534B544A50
:102F2000C3F830254FF050230122C3F858254FF441
:102F30007F03D3F83021D3F83431072A09D1023B7B
:102F4000032B06D84B4AD35C1BB100224A4BC3F873
:102F50004C25FFF7A9FF50B14FF05023D3F80024C0
:102F6000D10742BF0022C3F81421C3F818214FF43F
:102F70007F03D3F83021D3F83431072A09D14FF039
:102F80005023D3F80024D20744BF6FF00102C3F8E6
:102F90000024FFF789FF18B16522334BC3F80C27D3
:102FA0004FF47F03D3F83021D3F83431072A16D1F8
:102FB000314BD3F82034002B11DA4FF05023032289
:102FC000C3F8182501229A60D3F80421002AFBD007
:102FD0000022C3F804210122DA60C3F818254FF457
:102FE0007F03D3F83021D3F83431072A23D1023BB1
:102FF000032B02D8214AD35CEBB17E221A4B1B492A
:10300000C3F80C27C3F83C297F231D4AC2F81831A6
:103010000023C1F8043EC1F8083E01F54821C1F87B
:103020001031C2F82431C2F82C3102F5FF1202F53A
:103030008052C2F8A032134AD2F88C3043F4406375
:10304000C2F88C30104A114B1168C3F84415D2698C
:10305000C3F84C2508BD2922034BC3F80C270322D3
:10306000C3F83C2757E700BF0040005000900350D2
:103070004400EFBEB793000000200350B39300005C
:103080000020005000ED00E00080FF0000600050D4
:1030900030B50468ACB1B4FA84F30122C3F11F0364
:1030A000DBB29A4024EA0202D0E8EF5FA54204D1E5
:1030B000C0E8EC2FBCF1000FF6D1EAD102480B704A
:1030C00030BD0248FCE700BF0000AD0B0200AD0BB5
:1030D00010B50368CB40DB0710D401238B40026896
:1030E00043EA0201D0E8EF4F944204D1C0E8EC1F5C
:1030F000BCF1000FF6D1F2D1014810BD0148FCE748
:103100000000AD0B0400AD0B014BC3F80405704784
:1031100000700150044B1A7922B9012218601A710B
:103120000248704702487047D81000200000AD0BDD
:103130000C00AD0B08B50A4B1B6833B10520FEF738
:103140007BF910B90520FEF755F94FF05023012205
:10315000C3F81825C3F81425C3F8802508BD00BF9F
:10316000D810002010B5032845D8DFE800F0180279
:10317000554F00224FF480730121002003F15023AA
:1031800018601C68012402F150221460284A126859
:10319000002A47D04FF05023C3F804132BE04FF020
:1031A0005023D3F81814D3F81824C90312D502F009
:1031B0000303022B05D0012B02D0002004F034F9C8
:1031C00001234FF050220221C2F8183508224FF493
:1031D0008273D2E7D3F81424D207F1D5D3F81C2494
:1031E00002F00302013A012AE7D8114A12681AB123
:1031F0000222C3F8042310BDD3F80421002AFBD017
:103200000022C3F80421D3F80431F4E718224FF464
:1032100090734FF48071B0E720224FF492734FF413
:103220000071AAE71A68002AFCD018601B68E2E760
:10323000D81000204FF0502310B5D3F8002152B120
:103240000020C3F80001D3F800210122C3F80823AD
:10325000234B1B6898474FF05023D3F8042182B1C9
:103260000022C3F80421D3F80421D3F81824D3F89A
:103270001824022102F00302012A28D1C3F81815EC
:103280009A604FF05023D3F8202162B10022C3F896
:103290002021D3F820214FF48072C3F80823104B6B
:1032A00005201B6898474FF05023D3F82421AAB17A
:1032B0000022C3F82421D3F824214FF40072C3F86C
:1032C0000823074B0620BDE810401B681847C3F8C9
:1032D0000813034B01201B689847D2E710BD00BFBD
:1032E000D810002001460148FFF7D2BEC4000020DC
:1032F000036803F01F025B09026004D0012B03483E
:1033000018BF002070470248704700BF0028845053
:1033100000258450034A4309D35C00F01F00184481
:10332000C0B27047BF93000070B50546FFF7F2FFCB
:103330000C4C083034F810300E46DA0508D5C3F3CB
:10334000432304EBC302284654F8333052689847AD
:10335000A3682BB131462846E268BDE870401847A3
:1033600070BD00BFC800002008B5FFF7D3FF034BB6
:10337000083033F81000400B08BD00BFC800002023
:1033800008B5FFF7C7FF034B083033F81000C0F350
:10339000400008BDC800002008B5FFF7BBFF034B85
:1033A000083033F81000C0F3401008BDC8000020FA
:1033B000034611F0010010B5CCB20BD1A207C4F343
:1033C00040000DD5074A106A58601062003818BFD7
:1033D000012005E004490A6A1A600A62002AEDD059
:1033E00010BD00BF002884500025845010B5FFF7A1
:1033F00091FF124A083032F81030D9051CD5C3F3BA
:10340000432123F4F85322F81030002002F10E0477
:1034100034F8023F13F4807F03D0C3F3432399426F
:103420000AD001303028F3D1002342F8313004486B
:10343000BDE81040FFF74CBE10BD00BFC800002023
:1034400040010020F0B5054600200126044607464D
:103450008C420BD1114BD3F87C2132B10022C3F83E
:103460007C21D3F87C3140F00040F0BDE3B29B00FA
:1034700003F580729B0806FA03F31D420BD002F19C
:10348000A04202F55042D2F800C0BCF1000F02D0B9
:103490001760126818430134DAE700BF00D000500B
:1034A000F7B506460846FFF735FF1A4F00F1080545
:1034B00037F815300C46DB072AD5304604F0BFF844
:1034C0002046FFF769FF58B12046FFF74DFF002265
:1034D000316800B201EB8003C3F81025C3F8102552
:1034E0002046FFF783FF002301A827F81530019439
:1034F000FFF7FEFE019B00EB8300D0F80022064B95
:10350000134043F00203C0F80032044803B0F0BD9A
:103510000348FBE7C8000020F0F0FCFF0000AD0B03
:103520000400AD0B2DE9F0431646804685B00846F1
:10353000FFF7F0FE0D463168044609B32846FFF751
:103540001FFF18B12846FFF727FF10BB00230DF11E
:103550000F02CDE900338DF80E308DF80F3028467C
:103560000B460DF10E0104F012F8484A04F108016F
:1035700032F8113023F0020343F0010322F8113036
:1035800073687BB328461F785968FFF7F9FE10B1BE
:10359000E9B13F4829E03D4A04F1080032F8103013
:1035A00023F02003DB04DB0C22F8103079B1032F69
:1035B000EFD87168D1F804E0D8F800109EF800C088
:1035C00001EB8C01A7B9C1F81075C1F810752F4A2D
:1035D00004F1080132F8113023F01C0343EA870399
:1035E00022F81130B3683BBB2A4805B0BDE8F08330
:1035F000D1F810E543EA4C332EF0030EC1F810E584
:10360000D8F8001043F0200301EB8C0EDEF8101503
:1036100022F8103021F44F3121F44071CEF810150A
:103620002902DEF8108501F47C5141EA074141EAA4
:103630000801CEF81015CAE72846D3E90067FFF75E
:10364000D5FE002ED0D0114DD5E90023964203D1EE
:103650009F4201D1002209E00F480DF10F01FFF751
:1036600017FD0C4B9842C0D19DF80F2005EBC2030B
:1036700008345F6035F8143045F8326043EA42237D
:1036800043F4807325F81430AEE700BFC800002073
:103690000400AD0B0000AD0B400100202DE9F0430C
:1036A0000C46804685B0204611461D46FFF732FE87
:1036B000064629B32046FFF763FE18B92046FFF7F8
:1036C0006BFE18BB334F06F1080937F8193013F0B9
:1036D0001C0F02D04B78012B18D001238DF80F302E
:1036E00000234A1CCDE9001320468B1C0DF10F016D
:1036F00003F04DFF37F8193043F0030327F8193072
:10370000002D44D02046FFF73BFE18B9224805B0F3
:10371000BDE8F083002295F800C0D8F800301D4FB6
:1037200003EB8C03C3F81025C3F8102506F108023B
:1037300037F812104FEA8C0E21F02001C904C90C91
:1037400027F812106E7816B3D8F80000AD787044E0
:10375000D0F81035360423F4991323F4F853C0F845
:103760001035230203F47C5306F440362D05D0F8BF
:1037700010E5334305F480152B4341EA4C3143EA0D
:103780000E0341F02001C0F8103527F8121003484D
:10379000BDE700BFC80000200400AD0B0000AD0B6A
:1037A000014BC3E902127047C800002010B508465B
:1037B0001446FFF7F1FD50B10846FFF7ABFD054B8E
:1037C000083033F8103004485B0B237010BD0348F9
:1037D000FCE700BFC80000200000AD0B0400AD0BEB
:1037E00070B5154D064695F880401CBB21466022F9
:1037F00005F1100005F0E3F9214630682E6F8E4286
:103800000ED10023C0F87C31D0F87C3140F3073072
:10381000FDF7F0FD0123094885F88030AB6770BDE6
:10382000CBB29B0003F580727C2B04BF845083587D
:103830000131E4E70248F2E7C80000200000AD0BC8
:103840000C00AD0B034B93F88000003818BF01202B
:10385000704700BFC80000200148FFF739BC00BF17
:103860003C0100200148FFF713BC00BF3C010020D1
:1038700073B503681646D3F804230546002AA8BF8B
:103880004FF000420846A8BFC3F804230C46FFF7D8
:1038900083FD00B30846FFF773FD0146D8B9204603
:1038A000FFF762FD04B2A4000346286804F58072A5
:1038B0008150296882582144D1F8102542F0010234
:1038C000C1F810252EB10122296802FA03F3C1F8CC
:1038D000043302B070BD2046FFF71CFD0E4B0830CC
:1038E00033F81030C3F38203042B11D0052B11D011
:1038F00001A80194FFF7FCFC019A0369D34003F08F
:103900000103991C204602B0BDE8704003F088BE58
:103910000321F7E70221F5E7C80000202DE9F04F69
:10392000684BDFF8A481D3F80403D8F87010C0B254
:1039300089B040F00040FFF785FD051E2FDAC24632
:1039400000235AF87C1F06A8CDE90633FFF730FDA7
:103950004FF0000B5D4B0DF118090193019A12F81D
:10396000013B0192DA081AF8022003F0070322FA59
:1039700003F3DA071CD409F10409BBF1000F14D0DA
:10398000D8F870104FF00040FFF75CFDD8F87C10BD
:1039900006A8FFF70DFD0028DAD125F00045012427
:1039A000002D76D109B0BDE8F08F4FF0010BD5E7BF
:1039B000474B5B440293D9F800100029DBD091FA01
:1039C000A1F1B1FA81F1029B1C7841EA441420462E
:1039D000FFF7A0FC083038F81070C808BB08039344
:1039E000012319F8002001F0070103FA01F122EA8E
:1039F000010209F8002005A80594FFF779FC059A53
:103A0000039B803250F82220C7F382065B073746BB
:103A1000C2F3014222D520463946D6B2FFF784FCD4
:103A200005A80594FFF764FC059B803350F823300C
:103A3000C3F301439E4207D10021204603F0F0FD6D
:103A40003146204603F0ECFD05A80594FFF750FC35
:103A50000122059B02FA03F30362ACE7022A0CD1B0
:103A60000321204603F0DCFD06F00503012BEBD11A
:103A700039462046FFF758FCE6E70221204603922C
:103A800003F0CEFD032EF3D0039A032ADCD1022EDD
:103A9000EDE795FAA5F3B3FA83F304FA03F29B007A
:103AA00003F1A04303F55043D3F81005D3F81015E4
:103AB000C0F30520C1F3014125EA0205FFF734FCFC
:103AC0006EE700BF00D00050C8000020CF93000078
:103AD000CF93000070B5084C0E462379154643B9C4
:103AE0002A20FDF787FC0123044823712660A56086
:103AF00070BD0348FCE700BFE01000200000AD0BE4
:103B00000C00AD0B002330B50D4A50F8234003F5EF
:103B1000A2710133102B42F82140F6D10023084A4C
:103B200000F13C0103F5B27451F8045F0133102B2E
:103B300042F82450F6D1D0F88030C2F8043330BDBA
:103B400000A002500123024A8340C2F804337047A8
:103B500000A002500123024A8340C2F80833704794
:103B600000A00250F8B5012600270B4B0B4DD3F8EF
:103B70000C4304B9F8BD94FAA4F0B0FA80F006FA48
:103B800000F324EA0304064B82009F502B68002BAD
:103B9000EFD0A9689847ECE700A00250E0100020A1
:103BA00000A102502DE9F0410E4617460C4D55F884
:103BB0001C4FAC4203D16FF01200BDE8F0813146DA
:103BC00054F8440CA4F14408FCF7C4FA30B9C7F81F
:103BD00000804046BDE8F04103F04DBE2468E8E7B0
:103BE000EC10002010B5D0E909124A60416A00F1DA
:103BF00024031160C0E909334368044603B19847C0
:103C0000054A936833B11279062A03D9072022683E
:103C100002499847002010BDEC100020D19300000D
:103C20002DE9F04107460D460B4E56F80C4FB442B5
:103C300002D16FF001000AE0394654F8240CA4F1D7
:103C40002408FCF787FA20B91DB1C5F80080BDE84B
:103C5000F0812468EBE700BFEC10002038B5044683
:103C600000B30068F0B10378E3B10021FFF7D8FF9B
:103C7000D8B104F11C03C4E907330D4B04F124024D
:103C8000196903F10C00A16260621A610A609D6803
:103C900035B11B79062B03D9072022680549A847AF
:103CA000002038BD6FF01500FBE76FF01000F8E75B
:103CB000EC100020D393000010B5036893B11B787B
:103CC00083B18368012B0DD8084B00F14401436098
:103CD000074B1A6A03F11C048264446400201962D1
:103CE000116010BD6FF01500FBE700BF4C01002014
:103CF000EC10002038B5114C0546216819B10020A0
:103D00000131216038BD2422204604F058FF2B6881
:103D10002846A3602B79237104F10C03C4E9033313
:103D200004F11403C4E9053304F11C03C4E90733A7
:103D300000F018F80028E5D12168E0E7EC10002039
:103D400038B5074D2C68013C2C6044B900F012F8DE
:103D500021462846BDE83840242204F030BF38BD53
:103D6000EC10002008B50248FFF778FF002008BDDE
:103D70004C0100200148FFF735BF00BF4C01002077
:103D80000EB4431E062B33B588BF0020094B05AC8B
:103D900054F8045B53F82010074802F014FC214645
:103DA00028460194FCF76EFB02B0BDE8304003B03A
:103DB000704700BFB0910000E69300002DE9F04F7E
:103DC00087B017469B460446DDF840A000284BD03C
:103DD000056A35B12D6825B1AC4607B0BDE8F04F96
:103DE0006047A36A9F4242D80026BE4203D100200A
:103DF00007B0BDE8F08F182303FB06F8D4F82C9029
:103E0000A26909EB08052B1D0593CAB968696968A1
:103E10000368B5F80CC0C91AAB680CF1030E5D1E3F
:103E200005EB0C155B4205EB4E051D4005EBCC0385
:103E300085680633A94228BF4FF0FF3103F0E8FC44
:103E400059F8083020460293236AB1B29B6A019365
:103E50005AF8263000935BF82620059B03F029FDD5
:103E60000028C5D10136C0E76FF01500C0E7014852
:103E7000BEE700BF40F4FFFF10B5044690B1028DCD
:103E800043899A4209D0084A936833B11279032AC8
:103E900003D942680549042098472046BDE81040F0
:103EA00004F0F1BD10BD00BFEC10002081940000B3
:103EB00030B544898C4212D9436A013C5D882C405C
:103EC00003EBC40359609A60BFF35B8F426A538867
:103ED00001335380438D01334385002030BD0148B9
:103EE000FCE700BF41F4FFFF70B4039E144660B1CD
:103EF000006A50B14BB1013407D0002E05DBD0F879
:103F0000844014B1A44670BC6047014870BC70473F
:103F10002DF8FFFF70B4039E144660B1006A50B1E3
:103F20004BB1013407D0002E05DBD0F8944014B11A
:103F3000A44670BC6047014870BC70472DF8FFFF75
:103F400070B50C4611461E460E4B05462022002930
:103F500008BF1946204604F09EF90123E362049B42
:103F60006662A362059B25626363069BA363079B4E
:103F700063646A6804F13C03C4E90F526B60226C0D
:103F8000136070BDA29400002DE9FF47DDF8348076
:103F90000E4691469A460546002876D0002974D0F0
:103FA000B8F1000F71D001F16407384603F011FE3B
:103FB000BAF1FF3F49D1346E06F1500204F180009E
:103FC000844204F01F0C07D2C4F3411152F82110AF
:103FD00021FA0CF1C90736D4012104F07F046009ED
:103FE00052F8203004F5806A01FA0CF104F2014421
:103FF0000B4304F07F0442F8203034666B6C4A4671
:1040000003930E9B2946CDE901830C9B3046009318
:104010005346FFF795FF384600F0BAFC2C7874B190
:1040200096F8A4405CB1AB6A013330D10021284638
:1040300003F00EFE044610B1284603F0DFFD2046D3
:1040400004B0BDE8F0870134BAE7BAF5806FD5D384
:10405000AAF580637F2B06F150010FD8580951F85B
:10406000204003F01F0324FA03F2D2070BD40122ED
:1040700002FA03F3234341F82030BFE7054C3846EA
:1040800000F086FCDBE7044CF9E7024CD7E700249C
:10409000D5E700BF2DF8FFFF29F8FFFF08B58368BB
:1040A0001A0C0AD1094A93682BB11279022A02D953
:1040B000032007499847002008BDA3F5803383609B
:1040C0001B0C0CBF01200020F6E700BFEC10002005
:1040D000A394000038B50446E0B100F16405284619
:1040E00003F055FED4F8B4309B6953B9D4F8A84016
:1040F000103C002C00DC084C284603F046FE20460D
:1041000038BD012BF7D1D4F8BC0003F04AFDA0F173
:104110001004EEE7014CF2E72EF8FFFF2DF8FFFF49
:1041200038B50446E0B100F16405284603F02FFEDF
:10413000D4F8B4309B6953B9D4F8AC40103C002C8F
:1041400000DC084C284603F020FE204638BD012B39
:10415000F7D1D4F8B80003F024FDA0F11004EEE785
:10416000014CF2E72EF8FFFF2DF8FFFF2DE9F04399
:1041700085B00F46904603A90D9A0546994603F06F
:10418000C9FF0446E0B10C9E039BD5F8C0009E42D7
:10419000A8BF1E460168D0F808C0611A33464A46D7
:1041A000614528BF4FF0FF3103F0F8FA234642463D
:1041B00039462846009603F04DFF05B0BDE8F08370
:1041C0000048FAE72EF8FFFF2DE9F0438BB00E46CA
:1041D000DDE9128915461F46044620B9954D28464B
:1041E0000BB0BDE8F0830029F8D0002BF6D00021F9
:1041F000A822C0F8D01004F0E2FC012204F164000F
:10420000114604F0E1F98C4BC4F8B460E5677462C0
:10421000C4F88430894BD4F8B450C4F88830884B43
:10422000C4F88C30874BC4F89030874BC4F8943076
:10423000864BC4F89830864BC4F89C30854BC4F844
:10424000A030AB6943B9B9F1000FC7D099E80700B6
:1042500004F1A80383E80700AB69012B07D0D4F869
:10426000B400E0B96FF01505B9E74307F7D4D4F807
:10427000B4000028F6D0036A002B00F0D8809B68B9
:10428000002B00F0D48098474206EED50021D4F8E8
:10429000B40003F06AFD05460028E8D09FE7036AF2
:1042A000002B00F0C4801B69002B00F0C0809847F1
:1042B00000F0010084F8A400D4F8B4008369E3B9E5
:1042C00099F80830002B00F0858008F10C03C4F841
:1042D000C430B8F1000F81D0D8F80820002A00F0CF
:1042E000A4809B68002B00F0A0805B4B04935B4B89
:1042F00005935B4B06935B4B07938369012B07D1B7
:10430000564B0493544B0593564B0693544B0793CB
:10431000002104F1C803C4E9323306ABC4F8C0700D
:1043200002220093019104ABFFF748FD05460028E7
:104330007FF455AFD4F8B4309A693AB9F26A12688A
:10434000C4F8B820F26A9269C4F8BC209B69012BBA
:1043500007D1F36A9B69C4F8B830F36A1B68C4F8E4
:10436000BC30D4F8BC0003F0B7FBF36A1B68DF6213
:10437000F36A9B69DF62D4F8B430D3F81890B9F1CE
:10438000000F07D1D4F8AC300993D4F8B8305B896A
:104390004B4521D894F8A430C4E9004463B100230C
:1043A0000293314B204601933523304A0394009306
:1043B00004F10801FFF7C4FDD4F8B4008369002BB1
:1043C0007FF40DAF042103F0D0FC064600283FF433
:1043D00006AF24E043467AE74046D4F8AC1003F039
:1043E0008AFE0646D0B139680890411AB8680022A2
:1043F000814228BF4FF0FF31D4F8AC30384603F08B
:1044000007FA009601230022D4F8B80008A903F0A7
:104410007DFA064618B909F10109B6E7144ED4F839
:10442000B40003F09BFC3546D9E6114DD7E66FF09A
:104430000505D4E62DF8FFFF6D410000E37D000087
:10444000557F000015810000558000009B7D000015
:1044500021410000D5400000C4940000CA9400002F
:10446000817F0000897D0000077E0000D09400005D
:104470002EF8FFFFF0B505460E46174687B0074AEF
:1044800003AC07CA84E807000C9A3146009228461C
:104490003A460194FFF798FE07B0F0BD388F000050
:1044A00038B5EFF31185202383F31288BFF36F8FA4
:1044B000064B9C6803F016FF85F31188BFF36F8FDE
:1044C0002046BDE83840FCF717BF00BF10110020A0
:1044D00038B5094B53F82040013053F82050A5421D
:1044E00000D838BD636823B1204603F0FEFE0834CF
:1044F000F5E723689847FAE7D0910000012270B5EC
:104500002A4B032086B01A70FFF7E2FFFCF7FCFB92
:1045100003F007FF0420FFF7DBFF254C254D26465F
:10452000AE4204F1300410D300F084FE204C224E41
:10453000AC4226D300F092FEFBF75EFF1F4A137BCE
:1045400023F00103137306B070BD54F80C3C0593BF
:1045500054F8103C049354F8143C039354F8183C5A
:10456000029354F81C3C019354F8203C009354E906
:104570000A2354E90C0100F02BFC54F8303C5E6532
:10458000CDE7D4E90A23B3F1FF3F08BFB2F1FF3F03
:1045900005D052EA0301206803D104F08EF83034CC
:1045A000C6E73146183001F01FF8F8E74B1300203A
:1045B000308F0000308F0000E987000008080020DD
:1045C00008B50348034A0021121A03F0A6FE08BDED
:1045D00050030020501300200023012270B586B044
:1045E000CDE904230F220193CDE9023214234FF4C5
:1045F000A0720E4D0E4E03FB00550E4906EBC01681
:10460000044602FB00110C4B3046009500F0E0FB25
:10461000737B2C7423F004037373084B013403EB96
:10462000C423EE606B6006B070BD00BF10110020A7
:10463000880700205023002089840000501B0020A0
:10464000BFB50020FFF744FF2D4B03F5006282F356
:10465000088883F30A880024E0232A4D2A4E85F82F
:104660002230EC772C766C76AC7685F820406B6A3D
:10467000264F43F4E0236B6285F82340FCF7BAFD34
:10468000FCF75AFF4FF0FF33AB62EB62FDF7E0F847
:10469000FCF776FF40F201131D4D2846AB81C5E9BA
:1046A000194401F0CBF8B56003F008FE0120FFF7D4
:1046B0000FFF0220174DFFF70BFF00F0EFFD164B29
:1046C00075610593012315494FF48062CDE90343D9
:1046D00028463B46CDE90144009400F079FB0646AC
:1046E0006A7B284622F004026A7304F022F820460E
:1046F000FFF772FF3A4631462846FCF7F9FE00BF45
:10470000501B002000ED00E010110020FD440000CF
:104710002809002008080020D394000090240020DD
:1047200038B5064C064DAC4201D3002038BD2046BA
:10473000D4E9011203F0F6FD1434F4E7F00100208F
:1047400004020020002038B5054C064DAC4200D3D1
:1047500038BD204603F04BFE0028F9DB1C34F5E79A
:10476000EF010020EF01002073B50C46EFF311813B
:10477000202585F31288BFF36F8FC5685DB1256072
:104780002B68C360836901338361002081F3118842
:10479000BFF36F8F11E052EA030603D16FF00B00F5
:1047A0002560F3E7CDE900230246083000F08EFCD7
:1047B00018B9034B9B685B69236002B070BD00BFF2
:1047C000101100202DE9F341044617461E46EFF371
:1047D0001188202383F31288BFF36F8FC368334A95
:1047E0007BB180689168884219D057EA060318D1D6
:1047F00088F31188BFF36F8F6FF00F0002B0BDE830
:10480000F081916891F90E100133E36093682161A2
:10481000A36088F31188BFF36F8F0020EEE7216952
:10482000F2E791F90E1090F90E306FF07E02994286
:10483000A8BF19469142B8BF11468B422DDD03F047
:104840002EFE054622464146CDE90076184800F086
:104850003DFC0028E1D0EFF31186202383F312887A
:10486000BFF36F8FA068D0B1236821699C420AD042
:104870004BB193F90E309942A8BF19466FF07E03F1
:104880009942B8BF194603F00AFE40B131460848C4
:1048900000F08CFC6FF00A00B0E70025D2E7002D95
:1048A000F4D186F31188BFF36F8FF3E71011002066
:1048B0004C13002038B58368044663B3194A9268E4
:1048C00093422BD1C368012B03D9013BC360002065
:1048D00038BDEFF31185202383F31288BFF36F8F68
:1048E0000169806803F0DBFD204603F081FFA060D2
:1048F00058B190F90E2022610022C26703F019FF1F
:104900002946094800F052FCE1E7E06085F3118890
:10491000BFF36F8FDBE76FF01500D9E74FF0FF3083
:10492000D6E700BF101100204C13002037B5114608
:10493000EFF31185202282F31288BFF36F8F046892
:104940009CB12368426823F003039442036008BFCC
:1049500043600121204603F016FE044685F31188CA
:10496000BFF36F8F204603B030BD51EA0302F5D08C
:1049700000F10802CDE900131046294600F0A6FB1D
:104980000028EFD1014B9B685C69EBE71011002018
:1049900038B50446EFF31185202383F31288BFF363
:1049A0006F8F03F025FF48B10022C26703F0C1FEFC
:1049B0002946BDE83840074800F0F8BBD4E9023288
:1049C0009A4218BF01330221A36004F1100004F0E1
:1049D0002DF8EDE74C13002013B5EFF311812024DF
:1049E00084F31288BFF36F8F846844B1013C846004
:1049F00081F31188BFF36F8F002002B010BD52EA1F
:104A0000030406D181F31188BFF36F8F6FF00F009D
:104A1000F3E7CDE900230246014800F057FBECE73D
:104A20004C1300201FB5094A02AB92E803004FF473
:104A3000007283E80300009305494FF0FF330548F7
:104A400000F04CF9002005B05DF804FB448F000035
:104A500090280020880800202DE9F04305464FF0FB
:104A6000FF364FF0FF37DFF82C8185B0EFF3118967
:104A7000202383F31288BFF36F8FD5F880408CB961
:104A8000022105F1980003F0AFFD002860D100235A
:104A90004946CDE90067029305F188023E4800F0DF
:104AA000ABFCE3E7D5F8842023689442C5F8803056
:104AB00008BFC5F88430D5F8983043F00203C5F834
:104AC0009830E36823F0040343F00103E360636874
:104AD00089F31188BFF36F8F20469847EFF3118950
:104AE000202383F31288BFF36F8FE368D90623F086
:104AF000010237D4E260E3689A071AD5D8F80000BB
:104B000023F00203E360A0B10021026888B143688A
:104B10009C4237D1036869BBD8F80420C8F800303C
:104B2000824201D1C8F80430002340F8083BFFF767
:104B30002FFFD5F8983023F00203C5F8983089F399
:104B40001188BFF36F8FDB0590D400F0AFFB8DE7CA
:104B500005F1900400220121204603F0A1FE002867
:104B6000F8D194E723F01103E36004F11000FFF79C
:104B70000FFFC0E70B60D8F80430834208BFC8F8C5
:104B80000410D1E722B11368014610461A46BDE76A
:104B90001346F9E7301100204C130020F8B5C36824
:104BA00004469A070F46C3F340062CD45B071AD479
:104BB0000B680BB983680B60E368DD0742BFA3682D
:104BC00002263B603D6858BF0126002D3AD01F4B9E
:104BD0009B68AB420AD0D5F89830D807C3F380025F
:104BE00014D46FF0120600233B6025E003F05CFD57
:104BF000D5F898300028F0D1D907C3F3C002F0D51A
:104C000052B15B0708D46FF00F06ECE7002AFAD127
:104C1000C3F3C003002BF6D100232360D5F8843002
:104C200063B9C5E92044284603F0EAFCE36843F091
:104C30000403E3603B68A3603046F8BD1C60C5F820
:104C40008440F0E76FF01506CDE700BF101100209B
:104C50002DE9F041C368074603F00503002B0C461D
:104C600014BF4FF001084FF0000822D08668D6F834
:104C7000805025B1AF4201D02D68FAE7012501220D
:104C8000002104F1100003F09FFC2046124903F0BC
:104C9000BEFCE36843F01003E3609DB13B68236012
:104CA00073B9D6F884303BB9C6E92044304603F0E6
:104CB000A7FC4046BDE8F0811C60C6F88440F5E7DB
:104CC0003C60F3E7D6F880302360D6F88430C6F82D
:104CD0008040002BEAD1F0E7FF850000F0B50446E4
:104CE000002089B0C4E920000E9D04F18800C4E9C9
:104CF000220004F19000C4E924004DB32879002873
:104D000040F2011008BF0120C4F8980000204FF0C5
:104D1000FF364FF0FF37CDE90330CDE90100CDE993
:104D2000066720460B4B009400F090F855B12968B7
:104D300011B1204603F0BEFC6B791BB1237B43F01D
:104D400001032373204609B0BDE8F04003F0B5BC71
:104D50000120D9E7594A000030B50A46044685B01B
:104D6000EFF31185202383F31288BFF36F8FD0F800
:104D7000983013F0060F1DD1B1B143F00C03C4F805
:104D80009830204603F03CFC00234FF0FF320293A2
:104D90004FF0FF332946CDE900230C4804F190027F
:104DA00000F02AFB05B030BDD0F8800048B143F0D8
:104DB0000403E4E743F00401C0F89810002AE0D0AF
:104DC000DBE785F31188BFF36F8FEBE74C1300200F
:104DD0002DE9F043984685B000F15803C0E9163339
:104DE000109B002603730423073222F00705437348
:104DF0000F9B01EB05090F4683734946C0E9066620
:104E00008660C6730446FCF78FF80E9B073020F0CF
:104E10000700E066C4E9197502930D9BA9EB000930
:104E200001930C9B4A460093394643462046FCF7C3
:104E300043FB054B66659B6803B11B6F48462367C0
:104E400005B0BDE8F08300BF10110020F0B50025CB
:104E500087B00595109DDDE9127604950F9D0446F7
:104E600003950E9D02950D9D01950C9D0095FFF7F4
:104E7000AFFFB6F1FF3F08BFB7F1FF3F05D056EADD
:104E8000070305D1204600F0A3F9204607B0F0BD86
:104E90003A463346024904F1180000F0A5FBF4E756
:104EA000E987000038B50D4D2B4653F8184F9C424A
:104EB00000D004B9EC68AB6838B95A7BD20604D18B
:104EC000A26912B9DA897F2A05D89C4202D020460D
:104ED00000F0D2FA23466B6138BD00BF10110020EC
:104EE00008B590F90D200146002A437B04DA03F04F
:104EF0007F03437303F0E3FB044B9868431A584263
:104F00005841BDE80840FFF7CDBF00BF1011002099
:104F100070B490F90D30427B002B29DBD30627D1EA
:104F200083692BBB134962F07F0242730A4652F831
:104F3000184F944218BF2346CC6923B9C0E9002416
:104F40002060C8610CE090F90E5093F90E60B542F4
:104F50000AD0AE4208DD5A68C0E9003210605860DD
:104F6000002070BCFFF79EBF9C42E7D01B68E4E7BF
:104F700070BC704710110020002A2DE9F0410E4648
:104F80000CBF10210821427B044611420FD141EA97
:104F90000203D20918D1437308291BD00120FFF75F
:104FA00081FFBFF35F8F637B23F060036373284B44
:104FB0009B68A34245D1EFF30583002B41D13046D6
:104FC000BDE8F041FCF7AEB903F07F03437303F093
:104FD00076FBE1E7A36813B1204603F078FB04F108
:104FE000180003F07FFCA56D04F15807AF4211D003
:104FF0004FF0000875B1284603F069FB05F1180071
:1050000003F070FC2846C5F87C80FFF781FFA56D92
:10501000AF42EFD10E4FBB689C42BFD1EFF3058387
:10502000002BBBD00120FFF73DFF40F20113094DDB
:10503000AB8100232846C5E9193300F0FFFBBD60B2
:10504000AFE786F31188BFF36F8FBDE8F08100BF33
:10505000101100202809002070B590F90D2001469C
:10506000002A437B04DA03F07F03437303F027FB3A
:10507000154A4B7B104663F07F034B7350F8183F83
:10508000D469834208BF002323B9C1E90004216029
:10509000D1610CE091F90E5093F90E60B5420ED03B
:1050A000AE420CDD5868C1E900300160596090687B
:1050B000BDE87040431A58425841FFF7F3BE9C4286
:1050C000E3D01B68E0E700BF10110020F8B5124BD9
:1050D0000C46DDE9067611469868104A1060EFF339
:1050E0001182202282F31288BFF36F8F9D682846B9
:1050F00003F0F7FAB6F1FF3F08BFB7F1FF3F06D064
:105100003A463346064905F1180000F06DFA20468C
:10511000BDE8F840FCF706B9101100203811002056
:10512000E9870000F8B50446EFF31186202383F3E6
:105130001288BFF36F8F437B49B2DA0619D18569B4
:10514000BDB903F07F03437303F0B9FA437B164AFA
:1051500063F07F0343731346817353F8180F98422B
:1051600018BF0546D0695DB9C4E900300460D46158
:1051700011E00020A17386F31188BFF36F8FF8BD93
:1051800095F90E70B9420BD08F4209DD6B68C4E906
:1051900000531C606C600120FFF784FE0120EAE7E9
:1051A000A842E1D02D68DEE71011002049B9EFF3E5
:1051B000058030B9054B5A699B689A4201D0FCF7CB
:1051C000B1B881F31188BFF36F8F704710110020C1
:1051D00010B5EFF31184202282F31288BFF36F8F92
:1051E000427B510704D484F31188BFF36F8F10BD45
:1051F00022F004024273FFF78BFE2146BDE8104007
:105200000148FFF7D3BF00BF4C130020034648B945
:10521000EFF3058232B9064A51699268914201D092
:10522000FCF780B883F31188BFF36F8F704700BF1E
:1052300010110020EFF31181202383F31288BFF3B4
:105240006F8F054B9A68D37B013BD37381F3118831
:10525000BFF36F8F704700BF1011002038B5EFF318
:105260001185202484F31288BFF36F8F0A4B00202E
:105270009A68D37B0133D373FFF714FE85F311884B
:10528000BFF36F8FEFF3118084F31288BFF36F8F3A
:10529000BDE83840FFF7BABF10110020024B03F100
:1052A0001802C3E90622704710110020F8B5EFF389
:1052B0001185202383F31288BFF36F8F1949886803
:1052C000437B03F07F03437303F0F9F908468B68CF
:1052D0005A7B62F07F025A7350F8182FCC698242D1
:1052E00008BF002222B9C3E900042360CB610CE0AF
:1052F00093F90E6092F90E70BE420ED0B7420CDDEB
:105300005168C3E900210B6053600120FFF7CAFD1B
:105310002846BDE8F840FCF705B8A242E3D0126881
:10532000E0E700BF1011002050EA01032DE9F04131
:1053300005460E4603D1FFF7B9FF00202BE0831C82
:1053400071F1FF3329DB03F0E2FA2C18EFF3118837
:10535000202383F31288BFF36F8F124F124BB8686C
:105360001860FFF7BDFDB86810492A46334618306B
:1053700000F03AF9BA684046537B43F01003537388
:10538000FBF7D0FF03F0C3FA201A63EB03030128F5
:1053900073F10003D1DBBDE8F0816FF00104241A42
:1053A000D4E700BF1011002038110020E987000069
:1053B000B1F1FF3F08BFB0F1FF3F08B506D10A4B7E
:1053C000986803F0C5F94FF0FF3008BDFFF7ACFF58
:1053D0004FF47A7147F6FF730022C0FB0132D80BFD
:1053E00040EA4240F1E700BF10110020014B9868ED
:1053F000704700BF10110020D3B5DDE90667089C97
:10540000CDE90067FFF762FE1CB1034B9B685B6947
:10541000236002B0D0BD00BF101100200122044B58
:10542000C01A044BC0105843034B1A54704700BFB6
:10543000A8090020ABAAAAAA4C130020C3897F2B7D
:1054400012D80A4B1B6863B1094B90F90E201B68F8
:105450009A4209DB437BDB0606D1064BC31A18BF11
:10546000012303F0010070470023FAE740110020F8
:105470003C1100208807002070B50E4B0E4C1E7C9E
:10548000054606EB460304EBC304204603F02AFA64
:1054900000220A4B28469A55FFF7D0FF48B1084B27
:1054A0002046BDE870401A680649013AD31700F05B
:1054B0009BB870BD10110020A80900204C130020DB
:1054C000401100201D54000038B5EFF31185202352
:1054D00083F31288BFF36F8F104B114A9C681068DA
:1054E000A04206D1FFF7C8FF85F31188BFF36F8F85
:1054F00038BD00211B7C11600A4AD35C002BF3D01D
:105500002046FFF79BFF0028EED0637BDB0602D12D
:105510002046FFF7A1FD2046E4E700BF1011002060
:10552000381100204C13002008B50648064A0749E8
:10553000121A02F0F4FEBDE80840054A0549064883
:1055400002F0EDBE000000204C030020F0940000AB
:1055500000000000F094000000000020034B1B68D6
:105560000BB9FDF797BC0020704700BF4411002025
:1055700030B570B10B4B5B6898420AD0036843B1F9
:10558000D3E90421D0E90445121941EB0501C3E92F
:105590000421D0E9003213605A600023C0E90033CF
:1055A00030BD00BF7801002010B50E4B1C689C4236
:1055B00004D1FFF7D3FF6FF0004010BDFFF7CEFF1F
:1055C000002CF8D0D4E904321B1A62EBE072B3F17C
:1055D000004F72F10001EEDA002AACBF184600203D
:1055E000EBE700BF78010020B3F1FF3F08BFB2F145
:1055F000FF3FF8B504461D4616465ED08160EFF3C6
:105600001187202383F31288BFF36F8F013275F166
:10561000FF3324DA6FF001032D49D1E900209B1AF2
:105620004FF0FF3262EB00009E1B60EB0500012E85
:1056300070F1000301DA01260020C4E90460254E60
:10564000D6F800C07568B44508BF4FF0000CBCF137
:10565000000F0DD1C4E900652C6074601CE0FFF7F9
:105660007DFF013645F10005361845EBE070E4E7B3
:10567000DCE90420D4E90431934271EB000E1DDA19
:10568000D21ADCF8043060EB0100CCE90420C4E954
:1056900000C31C60CCF804403368B34209D09C427C
:1056A00007D10D4B1C6824B9FFF77EFF2146FDF79B
:1056B000C3FB87F31188BFF36F8FF8BD9B1A61EBB3
:1056C0000001AC45C4E90431C4D0DCF800C0BEE739
:1056D000C009002078010020441100202DE9F84F76
:1056E000EFF3118C202383F31288BFF36F8FDFF861
:1056F000B0A0DFF8B0900024C9F80000DAF800008C
:105700000025504508BF0020274FE046D7E900217B
:10571000D9F8003078B3D0E9046C4FEAE37EB342A5
:105720007EEB0C0B05DAF61A6CEB0E04C0E9046490
:1057300021E0B21841EBE671C0E90445C7E9002158
:10574000FFF716FF88F31188BFF36F8F83689847C0
:10575000EFF31188202383F31288BFF36F8FD9F8FA
:105760000030DAF800009B1B5045C446C9F80030F1
:10577000CBD1D7E9002100249A1841EBE373C7E9A4
:105780000023C9F80040FFF70FFF2146FDF754FB47
:1057900088F31188BFF36F8FBDE8F84FFFF794BE11
:1057A0007801002044110020C009002010B5EFF35B
:1057B0001184202383F31288BFF36F8FFFF7CEFE8F
:1057C0000346054AD2E90001181841EBE37184F35E
:1057D0001188BFF36F8F10BDC009002038B5034694
:1057E000EFF31185202282F31288BFF36F8FC1601F
:1057F000012181600068834206D185F31188BFF3DF
:105800006F8F0024204638BDD0E9003213605A6003
:105810000023C0E9003303F0C3F8294604460248D8
:10582000FFF7C4FCEEE700BF4D1300200A46014617
:10583000014803F015B900BFF0010020014B0367D8
:10584000704700BFF001002038B504460D4602F055
:105850002BFF20B9064B9B681B6F0BB938BD054B5E
:105860002A4621461846BDE8384003F0F9B800BF83
:1058700010110020F001002010B50A4C23681BB164
:1058800001232360002010BD00F0F4F80028F7D0B9
:105890000138072803D8044B53F8200010BD0348F3
:1058A00010BD00BF48110020E8910000FE8FFFFFEF
:1058B000BFF34F8F0549064BCA6802F4E0621343F9
:1058C000CB60BFF34F8F00BFFDE700BF00ED00E0EE
:1058D0000400FA0530B44FF0FE3200250B4B0C4C9F
:1058E0000C494968C3F80024C3F80424C3F8082409
:1058F000C3F80C24C3F81024C3F81424C3F81824E4
:10590000C3F81C24C4F8005530BC0847005084502C
:105910000040845080010020024BD0E90012C3E90E
:10592000001270478001002010B5044650B1636832
:1059300013F0685F05D0064A934202D000236260EC
:10594000236010BD034B04485B689847EFE700BF36
:105950002C5F5CA98001002008920000C8B1436858
:105960000D4A934213D013F0685F0ED0012350E824
:10597000002F194640E8001C9CF0000FF7D1012AC7
:10598000F5D0BFF35F8F002070470448704704488C
:1059900070476FF4E04070472C5F5CA9E98FFFFF10
:1059A000EA8FFFFF034680B1426809498A420AD064
:1059B00012F0685F05D0BFF35F8F002210461A60B7
:1059C000704704487047044870476FF4E0407047E0
:1059D0002C5F5CA9E98FFFFFEA8FFFFF10B504463B
:1059E00020B10023034A2360626010BD0248FFF724
:1059F00071FFF6E73A00003A3092000070B5194C9A
:105A0000D0F804C00668C4F804C0D0F808C0C06864
:105A1000C4F808C0E06026600868134B134D186096
:105A20004868D5F818215860886812F0685F986057
:105A3000C8680969D860196112D000230C4A05F5BD
:105A40008A70C5F81431C5F8B831C5F81821C5F801
:105A5000BC21B047236805F5DC70BDE870401847ED
:105A600070BD00BF9C010020880100206011002053
:105A70002C5F5CA908B500F011F830B900F010F8FF
:105A800038B9054AC2F80C0A08BD00F037F80320FF
:105A900008BD042008BD00BF00508450002070479E
:105AA00010B5114800F048F800B110BD0F4800F0E3
:105AB00043F80028F9D10E4C204600F03DF80028AC
:105AC000F3D10C4B0C481C6000F036F8014600285E
:105AD000EBD100F02DF8044608B1204610BD00F0CF
:105AE0003FF82046FAE700BFDC010020D801002083
:105AF000D4010020CC010020D001002008B50848C6
:105B000000F024F8074800F021F8074800F01EF8DC
:105B1000064800F01BF8BDE8084000F00BB800BFD5
:105B2000DC010020D8010020D4010020D001002099
:105B300000207047704700BF08B5034B02681B6820
:105B400010689847002008BD9C01002008B5034B51
:105B500002685B6810689847002008BD9C0100201F
:105B600070B5094C094D2069AB68984718B1084BCE
:105B700008485B6898470021074AEB681160206974
:105B8000BDE87040184700BF880100209C0100203C
:105B900080010020549200005C1100202DE9F04F9C
:105BA00043688DB015468046029383789A0740F18A
:105BB0000D8100240E78002E00F00A81252E0BD0D6
:105BC0004B1C0393013441463046029B9847002802
:105BD000C0F2F6800399EDE74E788B1C252E0393D7
:105BE000F0D00027B946BB46BBF11F0F38D8A6F14D
:105BF0002003102B0AD8DFE803F02A09093009092D
:105C0000092109090928092D09091F00A6F13003F6
:105C1000092B33D92A2E37D11BF0400F55F8043BFE
:105C200040F08280002BA7BF4BF0200B9946C3F1B8
:105C300000094BF0280B01E04BF0010B039B13F81C
:105C4000016B0393002ECFD130E04BF0020B4BF0F1
:105C5000040BF3E74BF0080BF0E74BF0100BEDE70C
:105C6000BBF17F0F19D8A6F13003092BD2D81BF056
:105C7000400F03D00A2101FB0737DFE70A214BF071
:105C8000200B01FB0939D9E72E2E06D11BF0400F5E
:105C900040F09E804BF0400BD0E76C2E31D02BD8DB
:105CA000682E36D06A2E3CD04C2E3AD0002F46F0CB
:105CB0002003B8BF2BF04002A3F16501BCBF002751
:105CC0001FFA82FB022901D9612B2FD10735072743
:105CD000DFF8ACA225F0070508351BF0080F66D0E9
:105CE0000AEB070B56465E4563D1A4EB0A0AA9EB03
:105CF000070906EB0A026FE1742E9FD07A2E9DD021
:105D0000D4E71BF0800F18BF4BF4007B4BF0800BE7
:105D100094E71BF4807F18BF4BF4007B4BF4807B2F
:105D20008CE74BF4207B89E71F4687E7A6F16301E8
:105D3000122900F2F080DFE811F013004F00EE00AE
:105D4000EE00EE00EE004F00EE00EE00EE00EE0082
:105D5000EE00FE00E900EE00EE001B00EE00AF00DA
:105D600055F8043B01270DF1180A8DF81830B4E7F7
:105D700055F804AB834BBAF1000F08BF9A461BF0ED
:105D8000400F504614BF39464FF0FF3102F0A8FED5
:105D90000746A2E741462020029B984700280FDBD8
:105DA000013EB742F6D34C44B146A41B98E74E4699
:105DB000F7E7414616F8010B029B9847002892DA54
:105DC00098F8023043F0040388F802304FF0FF34B3
:105DD00020460DB0BDE8F08F1BF0800F34D01BF4CF
:105DE000007F2CD0073525F00705AA4669685AF8C8
:105DF000080B2BF010050029ADB237DA404245F40C
:105E0000806561EB41010DF1180B0A235A4602F03F
:105E100073FEA0EB0B0301936B0662D5019B25F08B
:105E200001019F4289B240F3A180002E00F09980C9
:105E300015F0100240F09C80BB460D4623E0AA46B8
:105E40005AF8040BC117D4E7AA461BF4807F5AF80E
:105E5000041B01D10846F5E71BF4007F19BF48B2C7
:105E600041F3C01108B241F3C031C2E750EA010367
:105E7000C9D11BF0400FC6D0002FC4D12BF01102A6
:105E8000BB46019795B240F2064115EA01021CBFDC
:105E90000BF1010B00222CE02BF010020A231FFA59
:105EA00082FB1BF0800C49D01BF4007115BF073535
:105EB000AA4625F007055AF8040B1EBFAA466968D2
:105EC0005AF8080B50EA010545D12BF016051BF0D6
:105ED000400FADB242D0002F40D12BF017020197F6
:105EE00095B215F0100248D0019B002E42D103F16B
:105EF000010B29075AD4EB0706D5D9456FDDA9EB6D
:105F00000B030199CB465F185B4649E04BF0100B41
:105F100010237826C5E7782B04D1C6F1780343F027
:105F20001003BEE741462520029B98470028FFF654
:105F300047AF023447E608230026B2E7AA461BF41F
:105F400080715AF8040BBDD01BF400711ABFC0B2A7
:105F5000614680B2B6E72BF0060295B20DF1180B40
:105F600054E725F01105BB46ADB28CE70D46B8E706
:105F70003B460D4603F1020BBBE7DDF804B082E7B8
:105F8000E8940000E1940000CDE90432414620206D
:105F9000029B98470028FFF613AF049B059A013334
:105FA0009945F1DCA4EB0B019B46CC180AB34146A2
:105FB0003020029B98470028FFF602AF8EB90134CB
:105FC0002744391B019B994224DC1D4655BB019A8D
:105FD000A9EB0B09554622441446914433E0019F36
:105FE00092E7023441463046029B98470028E7DAA0
:105FF000E6E640F206410D42E2D015F0020F04F150
:106000000104414614BF2B20202015F4806F18BFD7
:106010002D20E9E741463020029B013498470028B3
:10602000CFDACDE606AB013D4146585D029B98476D
:106030000028CBDAC4E641462020029B0134984771
:106040000028FFF6BDAEA9EB0403002BF3DCC1E58D
:106050007047022806D0052804D001280CBF032071
:106060000020704704207047836800EBC101B3F53E
:10607000004F2CBF51F8220031F81200704700EB9E
:10608000C1018068B0F5004F2CBF41F8223021F8E3
:1060900012307047012208B5FFF7E6FFD04008BD77
:1060A000836800EBC101B3F5004F08D34B681AB108
:1060B00043F001034B60704723F00103FAE74B887C
:1060C0001AB143F001034B80704723F00103FAE754
:1060D00053000122FFF7D3BF8368B3F5004F34BFED
:1060E00004230823C91A081AC0087047B0F5004FE6
:1060F00034BF04230823481C0833A0EBD300B0FAB4
:1061000080F0C0F11F0070472DE9F04117460322CF
:106110000E460446FFF7A8FF8642054607F104082D
:106120000AD10122E368BA4023EA0203E3600023B4
:1061300044F82830BDE8F081314602222046FFF7BE
:1061400093FF06462B4601460322204644F828507A
:10615000FFF795FF334629462046BDE8F04102226D
:10616000FFF78DBF70B50D4686680446FFF792FFB6
:10617000B6F5004F014601D3012809D03046FFF79C
:10618000B5FF294602462046BDE87040FFF7BCBF78
:1061900070BD2DE9F04705468068FFF7A7FF05EBC6
:1061A000800ADAF8109088460646B9F1000F1BD035
:1061B0000327DAF8104028462146FFF76BFF4045D9
:1061C00007D3324621462846FFF79EFF2046BDE80A
:1061D000F087032221462846FFF746FF013FCAF811
:1061E000100001D08145E4D14FF0FF34EB68013657
:1061F000B4401C40EAD094FAA4F2B2FA82F2131D21
:1062000055F82340DEE72DE9F04114460E460546D9
:10621000FFF740FFA4EB0608371B07444246314610
:106220002846FFF755FF3A4621462846FFF750FF1C
:106230004346002221462846FFF721FF21462846F3
:10624000FFF728FF3B46211800222846BDE8F04111
:10625000FFF715BF2DE9F041164604460F46FFF73C
:1062600019FF314605462046FFF714FF05442A462C
:1062700039462046FFF72CFF31462046FFF70AFF3C
:106280002B46311800222046BDE8F041FFF7F7BE4B
:106290002DE9F0410D4686680446FFF7FBFEB6F592
:1062A000004F014601D3012832D03046FFF71EFFD0
:1062B00004EB80010E6996B90122E3688240134322
:1062C000E36002220D612B4629462046FFF7D7FEE8
:1062D000032229462046BDE8F041FFF7D0BE022246
:1062E00031462046FFF7C0FE0746034629462046B2
:1062F000FFF7C5FE0322334629462046FFF7BFFEBF
:1063000039462B462046FFF7BAFE02223146E1E726
:10631000BDE8F081F8B50C460546FFF7BBFE261830
:10632000012231462846FFF79FFEC3070CD43146B1
:106330002846FFF717FF21462846FFF7ABFE214608
:1063400022182846FFF786FF002221462846FFF73D
:106350008BFE271A012239462846FFF785FE10EAF0
:10636000020613D139462846FFF7FCFE2146324685
:106370002846FFF779FE2246211A2846FFF76AFFD2
:10638000214632462846FFF76FFE241A214628464A
:10639000BDE8F840FFF77CBF38B571B10568002251
:1063A0002846FFF799FE044601462846FFF778FE87
:1063B0002146BDE83840FFF7ADBF38BD70B506686F
:1063C00009B9002070BDB368B3EBD10FF9D9B3F5AB
:1063D000004F34BF04230823CC1D1C44E40821468D
:1063E0003046FFF7D6FE05460028EAD00146304683
:1063F000FFF750FEA04209D92C44294630462246D8
:10640000FFF701FF21463046FFF742FF30460122E9
:106410002946FFF745FEB368B3F5004F34BF0423A8
:10642000082303EBC5031844CCE72DE9F8430668BD
:106430001446B26801F1FF39B2F5004F34BF0423AE
:10644000082319EA01090F460BD0494239408B4213
:106450004F4628BF0B46894654B900252846BDE85B
:10646000F8839942F8D82146BDE8F843FFF7A6BF64
:10647000B2EBD40FF1D9B2F5004F34BF0422082299
:10648000E11D3944C91A11443046C908FFF781FE9D
:1064900080460028E1D0B36809EBC005B3F5004F92
:1064A00034BF042308231D4435447B1E1D44B5FB23
:1064B000F7F57D43A5EB090529463046FFF70CFEAD
:1064C0002C44073424F00704A41B804507464FEAF8
:1064D000E40408D2024641463046FFF794FE4146A6
:1064E0003046FFF7D5FE39463046FFF7D3FD384436
:1064F000844208D2394630462246FFF784FE2146C0
:106500003046FFF7C5FE012239463046FFF7C8FD89
:10651000A4E7B2F5802F2CBF082304232DE9F04116
:106520000026D21A8C18CD1D25F0070524F007048B
:10653000641BE408056021462046AC60EE60FFF76E
:10654000D5FD421D9200013002F107074FEAD7073F
:106550003146A2F1100205F11000B8BF324602F038
:106560002EFB3A4631462846FFF7B2FD3346324607
:1065700031462846FFF783FDA4EB0708284631463D
:106580000122FFF78DFD42463946FFF7A1FD3B464C
:10659000324639462846FFF772FD21462846FFF766
:1065A00097FD4346324621462846FFF768FD2146BF
:1065B00028460122FFF774FD3946BDE8F041FFF798
:1065C00067BE002070470FB407B504A951F8040B4B
:1065D0000191F9F757FF03B05DF804EB04B0704781
:1065E000038B13F0070305D10368002B0CBF0020B9
:1065F00003207047022B05D1408BB0FA80F0400990
:1066000080007047012B05D10368002B0CBF0020D0
:10661000052070470020704710B50C4600B111B935
:106620006FF0150010BD081D00F0B7F80028F9D173
:10663000A368032BF6D9F3E72DE9F0410D46074691
:106640001946281D90461E4600F0BBF8044638B196
:106650003346424629463846A446BDE8F0416047E5
:10666000BDE8F08110B4EFF31182202484F3128886
:10667000BFF36F8F416110BC0121F9F735BF38B509
:106680000C46054658B151B10B6843B14B6833B164
:106690001C22002102F093FA00202C6138BD6FF01B
:1066A0001500FBE770B505460E46FFF7B5FF041E63
:1066B00014DBEFF31182202383F31288BFF36F8F73
:1066C0004FF6FF716B8B2C8B8B4204F0070407D1C4
:1066D00082F31188BFF36F8F6FF00A04204670BDFC
:1066E000022C0CD101336B8382F31188BFF36F8FBF
:1066F0000023224631462846FFF79EFFEEE7062C90
:1067000014D8DFE804F004131313041A0400002360
:1067100033606B683BB9C5E90066ACB90221284615
:10672000F9F7E2FEDAE71E606E60F6E782F31188A1
:10673000BFF36F8F6FF00404D0E782F31188BFF3CB
:106740006F8F6FF08504C9E782F31188BFF36F8FF5
:10675000C4E710B5EFF31182202383F31288BFF34F
:106760006F8F048B04F00704022C0AD0012C0CBF9D
:106770006FF004006FF0850082F31188BFF36F8F14
:1067800008E0438B013B9BB2438323B92146F9F7D1
:10679000ABFE204610BD2046EEE7034640B14268FE
:1067A00002F00302022A06D0032A04D0012A05D0EF
:1067B0006FF0150070471A68002AF9D00020986021
:1067C000704710B54268034602F00302022A4FF0F8
:1067D0000004816007D0032A02D05C60002001E041
:1067E00018685C6010BD18685C600028F6D0FEF781
:1067F000F5FFF3E7704720B183682BB11B6833B115
:1068000018476FF0150070476FF004007047184686
:10681000704720B183682BB15B6833B118476FF0C4
:10682000150070476FF0040070471846704730B489
:1068300050B149B142B1846854B1E56845B141F8FD
:10684000040BE36830BC18476FF0150030BC70478C
:106850006FF00400FAE710B5044650B1006858B173
:10686000836863B11B6953B16168984700B92060C0
:1068700010BD6FF01500FBE76FF00100F8E76FF057
:106880000400F5E730B41346044650B1006860B127
:1068900082686AB195685DB10A46AC46616830BCF1
:1068A00060476FF0150030BC70476FF00100FAE7E9
:1068B0006FF00400F7E70369D3F8900370476FF0B7
:1068C00085007047084608B5114618B101F0E2F995
:1068D000002008BD6FF00100FBE7084608B511462F
:1068E00018B101F0CEF9002008BD6FF00100FBE700
:1068F00013B504460846216901F56371D1E8AF1F5D
:10690000022909D15BB168B100931346D0E909129D
:10691000FDF700FB02B010BD6FF00F00FAE76FF05B
:106920004C00F7E76FF00100F4E72DE9F8431C464F
:10693000DDE90853164698460F46006939B34AB355
:1069400044B36A1C43F10003022A73F1000324D20A
:10695000226842B1D0F890339A4204D96FF00B000C
:106960002360BDE8F88305EA080909F101035A42EA
:106970005A412146384601F096F988B9B8F1FF3FEF
:1069800008BFB5F1FF3FF0D06FF06800E9E76FF0A6
:106990000100E6E76FF01500E3E76FF08500E0E740
:1069A00030600020DDE701F0C2B938B50D4604467D
:1069B00000F148012846F9F7CDFB30B1284604F133
:1069C000C001F9F7C7FB20B90120782303FB004081
:1069D00038BD0020FCE702F5367102F53A7001F08F
:1069E00032BED0F8B030A0F53670003B18BF01239E
:1069F00000EB8300D0F8C40201F0E5B8C86828B104
:106A0000096983681B680BB1002218477047FDF7BE
:106A100051BFD0E8EF3FC0E8E21F002AF9D170472C
:106A200010B5436804691B68C4F8883304F5EC703A
:106A300001F03DFD002104F56370FFF7EAFF084611
:106A400010BD2DE9F34117460D4679B30B786BB3B2
:106A5000D0F8C440A4F5E27814344FF0FF324FF080
:106A6000FF332046FDF7AEFE2A46404601A9F9F75E
:106A700075FE019E2EB9204602B0BDE8F041FFF739
:106A8000C6BF58B12046FFF7C2FF3B462A463146F3
:106A9000404602B0BDE8F041F9F73EBE202229464B
:106AA00006F1480002F00CF8B766E4E702B0BDE872
:106AB000F081030103EB4003093323F0030303EBED
:106AC000C00348430330083320F00300184440005B
:106AD00070472DE9F84306464FF001090569D0F8E3
:106AE000048005F56377D7E8EF3F022B03D1C7E8B1
:106AF000E29F002AF7D141D195F86C30002B40D1AC
:106B000095F8E430002B3CD12846D5F8881300F0E6
:106B100054F8044680BB73683669D3E9050183687D
:106B20001B693BB322469847044628BB06F53A76D4
:106B300049463046FEF710F9304605F5F876FAF783
:106B4000DBFB3046D8F8001000F074F8044698B922
:106B50000146E822304602F032F821464FF4F67240
:106B6000284602F02CF821463846FFF752FF20460F
:106B7000BDE8F8836FF057040221F5E76FF0770462
:106B8000F5E76FF00F04F2E710B50846029B1146D7
:106B900052B993F86C202AB90122184683F86C2068
:106BA000F9F7CCFE002010BD1A6F5468002CF9D004
:106BB0005A6FA047F6E701F0BAB838B50D4604465B
:106BC00060B1F03001F054FB0DB1002038BDC4F8C5
:106BD000C451C4F8C851C4F8CC51F6E76FF01500A1
:106BE000F4E70268D2F8E03013B1D2F8DC101847AD
:106BF00070477047836913B9D0F8883019707047AF
:106C0000012070478369012B04D1D0F888301878AF
:106C1000C0B270470420704738B5C41DE400204658
:106C200001F038FF054618B12246002101F0C7FFE8
:106C3000284638BD38B504463022002101F0BFFF98
:106C40001822002104F1BC0001F0B9FF1822002134
:106C500004F1A40001F0B3FFD4F8D800FDF70CF95B
:106C6000D4F8D400FDF708F9002304F13400C4F887
:106C7000A03000F02AFDFDF763F8E36E04F1400553
:106C80000BB12846984738220021284601F097FF8B
:106C9000002038BDFEE7012801D1EFF30583FDF7A1
:106CA000FFBB01460068FFF7F6BF08B5FAF738F9F1
:106CB000BDE80840FAF758B900210120FFF7EBBF03
:106CC000436E83F30B88704761B662B680F3118818
:106CD000BFF36F8F704708B572B6002383F3118836
:106CE000BFF36F8FFAF7BCFF50B1BFF34F8F30BFC8
:106CF00000BF00BF00BF00BF00BF00BF00BF00BF9C
:106D000062B6BFF36F8F08BD10B5044672B600239C
:106D100083F31188BFF36F8FFAF7A2FF50B1BFF36F
:106D20004F8F20BF00BF00BF00BF00BF00BF00BF2C
:106D300000BF00BF84F31188BFF36F8F62B610BD30
:106D400040E800F313F4803FD8B208BF6FF015009D
:106D5000704730B50C684B6885B00A894D8900943E
:106D6000013B24F01F04234402F01F0242EA4512B3
:106D700023F01F0369468DF808200393FAF736FCC9
:106D800005B030BD7047416A8968FAF73FBE836835
:106D90000B440360704730B484880568A31883806F
:106DA000281930BC01F0FEBE0268531E03608388C0
:106DB0000133838002F8011C704703468288521A0F
:106DC000828000680844186070478388C2888168A0
:106DD000D21A03685B1AD01A70470B464FF0502244
:106DE0000121C2F81416002118470120FAF7F6BF56
:106DF00000692430FDF7CCBD38B50C46097E022968
:106E000003D0042910D051B90121056904F10C0007
:106E1000FFF7CAFF228AE168281DFFF733FD2046ED
:106E2000FAF786FE002038BD0521EEE738B5046983
:106E300000200D46FBF706F9B0B9E06BFFF7DBFC6D
:106E400010B110F1780F0FD1E06B04F10C02211D8D
:106E5000FFF7EDFC40B94FF40042002304F1240099
:106E6000FDF7BAFD00B9256038BD10B50469201DD5
:106E7000FFF7F1FC034648B9E06BFFF7CAFC034695
:106E800020B900F005F8034600B92060184610BD8F
:106E900008B50020FAF766FF002008BD0C22036940
:106EA000C9B201FB0233986F00F00700704770B55C
:106EB000C9B20369EFF31185202484F31288BFF36C
:106EC0006F8F0C2606FB0134A46F14F0C00408D0A9
:106ED000A24206D085F31188BFF36F8F4FF0FF30C9
:106EE00070BD012206FB01339A6785F31188BFF359
:106EF0006F8F436803EBC1035B6898470020EFE79F
:106F00008022FFF7D4BFF8B5069F0469C9B2EFF33A
:106F10001186202585F31288BFF36F8F0C2505FBA2
:106F20000144A56F05F0070CBCF1010F0CD1A76758
:106F300086F31188BFF36F8FC4E91C23436853F8AD
:106F4000313098470020F8BD05F0C005AF4286F308
:106F50001188BFF36F8F0CBF6FF077004FF0FF30D9
:106F6000F1E713B580240094FFF7CDFF02B010BD08
:106F700010B41C240069CBB203FB0400002110BC38
:106F800010470320FCF7EEB80220FCF7EBB8002016
:106F9000FCF7E8B8032000F0F8BA022000F0F5BAD8
:106FA000002000F0F2BA1046FDF7F2BC4368002062
:106FB0005B681B690B607047436802EA01005B680D
:106FC00021EA020198600020D960704743680020E0
:106FD0005B6899607047436800205B68D9607047C0
:106FE00043685A68536821EA03000B409060002010
:106FF000D360704710B503695868F8B1884219D159
:107000009C680868A142586000D198600020086020
:107010002AB15A680A609A68596002B999600020DA
:1070200010E0814206D10868206098688142EDD165
:107030009C60EBE7044600680028F2D1002AE8D102
:107040006FF0150010BD30B451F820500C4601EB24
:1070500080023DB10146AC46D4F88000002330BC2C
:10706000126C604730BC704710B500690F299FBF94
:1070700000EB810440F821202364002088BF6FF0DA
:10708000150010BD00207047102070470F290ED842
:1070900043685B68CB40DB0709D501228B00DBB27C
:1070A00003F1A04303F5283300201A6070476FF006
:1070B0001500704738B50F290C46056933D8436869
:1070C0001B68CB40DB072ED5D5F8841021FA04F3DA
:1070D00003F001031AB99BB96FF0770022E0002B8F
:1070E000FAD111B92A20FAF785F90122D5F88430AE
:1070F000A2401343C5F88430E0B2FCF723FD0AE058
:10710000E0B2FCF727FD0122D5F88430A24023EA43
:107110000203C5F88430D5F8843013B92A20FAF771
:1071200077F9002038BD6FF01500FBE730B54368F4
:107130001360057A446804EBC504A34202D36FF0E0
:10714000010030BD5C798C4201D00833F0E70020AB
:10715000F7E743681B68D3F88004C3F880047047DE
:1071600042681368D3F8100150B10020126A1278F7
:107170000A70C3F81001D3F8102101221A60704779
:107180004FF0FF307047002A0FDD42681368D3F8D4
:10719000100158B10020C3F81001D3F810010120EC
:1071A000126A12780A70186070470020704710B594
:1071B000436819680369EFF31182202080F3128875
:1071C000BFF36F8F00241868847301201B68D87385
:1071D0004FF48003C1F8043382F31188BFF36F8F3B
:1071E00010BD012103691A68917300221B68DA73CC
:1071F0007047026903461168C87B40B15B681B6831
:10720000D3F8580118B100230B61136898897047AF
:1072100043681B68D3F81001003818BF012070477D
:10722000102243681B68C3F8042370471022436888
:107230001B68C3F8082370474FF4007243681B684B
:10724000C3F8042370474FF4007243681B68C3F807
:107250000823704738B5436804461D68D5F80433E1
:107260005B0205D4D5F8040310F0100006D138BD38
:10727000FFF7BFFF0028F5D00120F8E72046FFF711
:10728000C7FF003818BF0120F1E7012070470369EC
:10729000186801601B685A60704702680346D2F89C
:1072A000580140B95B68DB0706D4D2F820010038EA
:1072B00018BF012070470120704710B4436802696D
:1072C0001B68D3F80413C90517D5D3F82011A1B151
:1072D000EFF31181202484F31288BFF36F8FD3F86A
:1072E000204134B10024C3F82041D3F820410124C7
:1072F000DC6081F31188BFF36F8F1468D3F85811E5
:107300005CB161B1002121611468A47B3CB14FF4F0
:107310008000C3F808031368997310BC7047D3F852
:10732000241121B10021C3F82411D3F824311268AB
:107330001368002BF1D0516810BC18472DE9F041BB
:1073400006690546336801279C8910339442A8BF1B
:107350001446D3E8EF2F002A03D1C3E8E07F0028CA
:10736000F7D10CBF3B4600232BD1336822469868E7
:1073700001F018FCEFF31188202383F31288BFF388
:107380006F8F69680846FFF788FF326840B9044686
:10739000106188F31188BFF36F8F2046BDE8F0813C
:1073A0000B689268C3F844250022C3F84845C3F827
:1073B0002021D3F82011C3F85821D3F858219F6019
:1073C000E7E71C46E9E7002200F150039B009BB26F
:1073D00003F1502303F580331A601B68704708B52A
:1073E000FBF7C6FB08BDFEF747BA08B5F9F79AFCEC
:1073F000F9F780FDBDE80840FEF73EBA004700F00F
:1074000059BF40F00040C1F88000704740F0004094
:10741000C1F88000704740F00040C1F88000C2F819
:1074200080007047FBF75EBF73B503285DD8DFE8C7
:1074300000F0021826344FF050230222C3F808232C
:107440000122DA600022C3F80421D3F804310024B9
:1074500001238DF80730032847D8DFE800F02C48D7
:1074600065824FF050230122C3F808235A6000229E
:10747000C3F80021D3F800310DF10704E8E74FF01D
:1074800050234FF40072C3F8082301225A620022ED
:10749000C3F82421D3F82431D9E74FF050234FF417
:1074A0008072C3F808230122DA610022C3F8202188
:1074B000D3F82031CBE742F210754FF05026D6F8C2
:1074C000183403F4803334B97BB10120FFF797FF00
:1074D000013DF4D109E0D6F8182402F0030222702D
:1074E0001BB19DF807000128F0D002B070BD42F238
:1074F00010754FF05026D6F80C3403F480333CB9A5
:10750000002BF2D00120FFF77AFF013DF3D1ECE729
:10751000D6F80C2402F001022270002BE5D09DF871
:1075200007000128EFD0E0E742F210754FF0502637
:10753000D6F85C3403F480333CB9002BD5D001205D
:10754000FFF75DFF013DF3D1CFE7D6F85C2402F0F1
:1075500001022270002BC8D09DF807000128EFD04F
:10756000C3E742F210754FF05026D6F85434DB03CF
:10757000BBD52CB90120FFF742FF013DF5D1B4E79F
:107580009DF807000128F6D0AFE7FFF74DBFF7B52C
:107590001646DDE90847019001A81D46FBF7A8FE45
:1075A000019BB6F1000C18BF4FF0010C00EB8300FB
:1075B0000B1E18BF0123002D43EA4C0314BF4FF0EC
:1075C0000C0C4FF0000C002C43EA0C0314BF4FF4DA
:1075D000706C4FF0000C002F43EA0C0314BF4FF403
:1075E000403C4FF0000CD0F8002243EA0C0322EAA2
:1075F000030301B109780EB13678760019430DB155
:107600002D78AD0031430CB12478240229430FB109
:107610003F783F040C433C43C0F8004203B0F0BD48
:107620001FB50DF10F03019300238DF80F101A46BB
:1076300019460093FFF7ABFF05B05DF804FB38B5C2
:10764000054608460C46FBF7A7FEB0B10846FBF717
:1076500097FE90B90846FBF787FE01232A6883400E
:10766000C2F808332A6803B202EB8303D3F810256B
:1076700022F00302C3F8102538BD2046BDE838408B
:107680000021FFF7CDBFFBF70BBFFFF7D8BF37B522
:107690000C46154690B1037883B179B10B786BB184
:1076A00062B101A9FCF7BCFA50B9019883684BB1EB
:1076B0002A46214603B0BDE8304018476FF0150058
:1076C00003B030BD6FF01200FAE701464068C368AE
:1076D00003B1184770472DE9F04389B0109E044666
:1076E000894690460021202268461F46129D01F0DF
:1076F00066FA1F2E97BF01234FF0FF33B34003F10B
:10770000FF332361119BC4E90098C4E902766361E9
:10771000183445B10FCD0FC495E80F0084E80F0071
:1077200009B0BDE8F0836D46F4E773B50468661CE4
:1077300031D08568A9422ED264182CD05E18AE4292
:1077400088BF6B1A056A35B100930523A847034625
:10775000184602B070BDBFF35B8F1946A41A10190A
:1077600019B140EA0205AD070AD103290DDC013841
:1077700011448A42ECD010F8014F02F8014BF8E7AF
:107780000078013902F8010BE9E750F8044B04399D
:1077900042F8044BE9E76FF02103D9E773B50468B9
:1077A000651C32D08568A9422FD264182DD05E188E
:1077B000AE4288BF6B1A456ACDB100930523A84736
:1077C00002B070BD12F8015B013905701546A018B2
:1077D00019B140EA0206B607F4D103290ADC013DDB
:1077E000014488420CD1BFF35B8F1846E8E7194685
:1077F000A41AEBE755F8042B043940F8042BECE706
:1078000015F8012F00F8012BEBE76FF02100D7E707
:1078100073B51C46036815465A1C29D082689142EC
:1078200026D25B1824D066189642866A88BF541AFE
:1078300036B105232A460094B047204602B070BDF9
:10784000184622464AB9294601F0B9F9BFF35B8FC1
:10785000F3E700F8015B013AF4E78307F9D14FF051
:1078600001336B43032AEEDD40F8043B043AF9E7A9
:107870006FF02100E2E70020704710B4046B02466D
:107880000B4684B9C1681F2998BF23FA01F44168E7
:1078900061B18068834209D21069184051F82430E0
:1078A000184410BC7047234610BC18474FF0FF30F7
:1078B000F7E730B5059CC4E90002039A21811989D4
:1078C000E260049A618121856261D3E9002502EBBF
:1078D0000113C4E906128A1C236203EB42036A1CEB
:1078E00013446D422B406362836953B90139E269E5
:1078F0008B4202EB031206DB002393736FF07F03CE
:10790000D373002030BD0133D381F0E72DE9F04F70
:10791000B0F830A004465546002685B002EB0308B7
:1079200091460E9A00EBCA031FFA88FB9A63A3F8EC
:107930003CB008F1FF32C3690F1D0192B0451ADC5B
:10794000238D2586A3EB0B032385236A61895A883F
:1079500001390A4003EB4203A3F804A0BFF35B8F95
:107960000020226A538801335380638D013363857D
:1079700005B0BDE8F08FE06A2A0157F8041C03EB5C
:107980000515029303680392C91A83680837994260
:1079900028BF4FF0FF31FFF770FFDDE9023298504A
:1079A00000226A6057F8082CAA60019A9642ACBF80
:1079B00000220122B145D8BF42F00202AA8101365D
:1079C000ED89BBE7F0B550B3456A448E6B88A3429E
:1079D00030D0631C43864389BFF35B8F013B1C405F
:1079E00005EBC4056B689EB209B1AD680D60D0F8B7
:1079F0001CC09BB20CEB031100EBC3039D8F078DE2
:107A00002F44013D07859D878D896F070ED5058E13
:107A1000CD8100210686986B996302B11480F0BD78
:107A20009D8FC989013D0CEB01119D878D89ED0763
:107A3000F6D4ECE70020F2E7C36903EB0113986882
:107A4000704770B5C369C56A09015E586B6BE3B9CD
:107A50002C69621C09BF6B6834401C68341B2146CA
:107A60002846FFF70AFF864207D02B6901331C44E2
:107A7000AB689C42F3D34FF0FF342868431C09D015
:107A8000AB68A34206D9204470BD314628469847CA
:107A90000446F2E70020F7E770B5BFF35B8F0D46B1
:107AA000016A1646838E4A8804469A4212D05A1CAE
:107AB00082864289013A134001EB4301898829807B
:107AC00089B2FFF7BEFF2A88E36903EB02139B68C4
:107AD000336070BD0020FCE710B50268936912693D
:107AE000920017D543B9438E026A81694489013BEC
:107AF0001B1B02EB4102938003689B69012B08D199
:107B0000838E426A81694089013B1B1A02EBC102E4
:107B1000938010BD23B9026A138843F001031380D8
:107B200003689B69012B01BF426A138843F001037C
:107B30001380EEE710B5BFF35B8F036804461A6944
:107B40009B6912F0005F1AD07BB9036A426A5B88B6
:107B50008169013B02EBC10292889B1A628D9BB244
:107B60009A4214D80023638510BD012BFAD1436AD1
:107B7000026A5B888169013B02EB4102ECE763B971
:107B8000436A1B88DB4303F00103002BEAD06369DF
:107B9000002BE7D020469847E4E7012BE2D1036AA7
:107BA000EFE7036A828E598891420AD041890139F0
:107BB0000A4003EB42039A88C36903EB02139868F7
:107BC000704700207047BFF35B8FC36803B118474D
:107BD00070474FF0FF324FF0FF33FCF7FDBE10B19E
:107BE000C36A0133C362704738B1C26A013AC262E4
:107BF0001AB9026B02B110470262704770B50446B1
:107C0000056A05F164063046FFF7E3FF636AA3F5F2
:107C100080637F2B0BD801225909503503F01F03D5
:107C20009A4055F8213023EA020345F82130D4E97F
:107C30000F124A60E16B04F13C0311602046C4E975
:107C40000F33FFF7D1FF3046BDE87040FCF7A0BE10
:107C500010B58CB0436A04460B912022014602A85D
:107C60000A9300F018FB28230122CDE900322046B8
:107C70003522616A02ABFCF737F900EAE0700CB01C
:107C800010BD30B1006A20B119B1D0F8883003B10D
:107C90001847704730B1006A20B119B1D0F88C3064
:107CA00003B11847704730B1006A20B119B1D0F85C
:107CB000903003B11847002070472DE9F84306467D
:107CC0008846174699460468A64201D1002520E05F
:107CD0007A1CA4F13C0502D06B6ABB4219D0B8F102
:107CE000000F22D020224146284600F0D7FEE0B9FE
:107CF000B9F1FF3F02D0AB6A4B450AD07B1C0BD0D9
:107D00002468B442E2D054F8183CA4F13C059F42E8
:107D1000E8D12846BDE8F883AB6A0133F9D024687E
:107D2000B442D3D0A4F13C05D9E72468CCE710B520
:107D3000044690B1036A83B102784AB193F8A43043
:107D400033B1436AB3F5806F02D30121FFF780FF9F
:107D50002046BDE81040FFF751BF10BD20B1036AB7
:107D600013B15B6803B11847704708B530B1036AB7
:107D70003BB1DB682BB19847002008BD6FF01500C0
:107D8000FBE76FF00500F8E77047FCF701BE4FF026
:107D9000FF324FF0FF33FCF71FBEF8B50C4600F181
:107DA00064070546A4F110063846FFF7F0FF304699
:107DB000FCF774F980B154F8083C24F8083CD5F875
:107DC000CC3044F80C3C05F1C80344F8103CC5F82D
:107DD000CC6054F80C3C1E603846FFF7D6FF0020FC
:107DE000F8BD38B50D4600F164042046FFF7CFFF1B
:107DF00055F8083C204603F5803345F8083CBDE8BB
:107E00003840FFF7C2BF2DE9F04188B00E9C282A08
:107E10008846D4F8C0006ED101688568A8EB0101DE
:107E2000A94228BF4FF0FF3120236A46FFF77DFCAF
:107E300004F16406D8F820703046FFF7A8FF3B46EF
:107E40004FF0FF3269462046FFF737FFD8F824305D
:107E50000546E0B1D0F8308003F00103B8F1000F1F
:107E600002D0DBB9AF6230E0002BFBD04FF0FF3324
:107E700083623046FFF789FFAB6B83BBD4F8803059
:107E8000002B38D03A4669462046984733E0DB0756
:107E90001FD43046FFF779FFE36FF1E74FF0FF3370
:107EA0008362FFF79CFE3046FFF76FFFAB6BA3B911
:107EB000D4F880301BB13A46694620469847304690
:107EC000FFF765FF2846FFF78FFE3046FFF75DFF9F
:107ED00011E03046FFF759FFD0E74FF00108284680
:107EE0009847D4F880301BB13A46694620469847F7
:107EF000B8F1000FE3D1002008B0BDE8F081F0B583
:107F000004468E680D46B6B23146D0F8B80085B04A
:107F1000FFF792FDD4F8B43007469A6942B900954C
:107F2000CDE902500123D4F8B80002A9FFF7EEFC16
:107F3000D4F8B4309B69012B05D13A463146D4F8C8
:107F4000B800FBF7B5FFD4F8B80005B0BDE8F040C5
:107F5000FFF7F0BD70B500F16406A1F1100504460D
:107F60003046FFF714FF2846FCF798F818B1294669
:107F70002046FFF7C4FF3046BDE87040FFF705BF5D
:107F8000F0B5036885B05F6A07F164063046FFF715
:107F9000FEFED7F8B4309B69002B4DD0012B46D1A3
:107FA000D7F8B80003AA0DF10A01FFF775FD0446E2
:107FB0003046FFF7EAFE002C3CD0BDF80A303046D0
:107FC000A360FFF7E4FE4FF0FF33002162683846FC
:107FD000FFF773FE0546FFF702FEA368304603F580
:107FE0008033A360FFF7D1FE7DB1AB6A696C0133CA
:107FF00008BF2368284608BFAB622368A2890091A6
:10800000D5F834C004F11001E0473046FFF7BFFE59
:108010002846FFF7E9FD2046FCF740F818B1214655
:108020003846FFF76CFF3046FFF7AFFEAEE730464D
:10803000FFF7ABFE05B0F0BDD7F8B8000DF10A02AE
:1080400003A9FFF7BFFCD7F8B43004469B69012BA6
:10805000AED1A5E72DE9F041A3F1100653F8085C75
:10806000002388B00693ADF81E3004461023CDE9F6
:1080700004120E9FD0F8C000ADF81C700168D0F853
:1080800008C0711A0DEB0302614528BF4FF0FF31A4
:1080900004F16408FFF782FB4046FFF778FED4F84E
:1080A000B430ADB29B69CBB9D4F8A820D4F8B430C1
:1080B000D4F8BC009B69C3B9CDE9026200960122E5
:1080C00002A9FFF723FCD4F8BC00FFF733FD4046BC
:1080D000FFF75BFE384608B0BDE8F0812946D4F8CA
:1080E000BC00FFF7A9FC0246E0E7012BEBD12946D3
:1080F000FBF7DEFEE7E710B548B149B143688B42B4
:1081000006D382680468D21A5B1A4360A01810BDB7
:108110000020FCE72DE9F3470546D0F8B4000E46F1
:10812000904618B9002002B0BDE8F087036A002B22
:10813000F8D09B68002BF5D098474307F2D543F65B
:108140009823B8F1000F18BF984605F1640705F1B0
:10815000C8093846FFF71BFED5F8C8404C452BD060
:1081600054B3D4E90023536022681A60C4E9004480
:10817000D5F8B43021899B69ADF806107BB1012B8D
:1081800014D03846FFF701FEBDF8063004F11000A8
:1081900003F58033A3603368103B3360C3E7D5F841
:1081A000A8303360D5F8B4309B69E8E7D5F8BC0057
:1081B000FFF742FC3060E4E7D5F8B430D3F818A0FC
:1081C000BAF1000F36D13146D5F8BC000DF10602E8
:1081D000FFF7F8FB04460028D3D1D5F8BC301B8D3F
:1081E000B3B93846FFF7D1FDB8F1000F9AD0D5E901
:1081F0002D3218211289DB6A01FB0233D5F8D02019
:1082000022BB21200021FDF7D3F808F1FF38A0E7B9
:10821000D5F8A810D5F8C400FFF76DFF0446D5F8CF
:10822000A830ADF806A033603846FFF7AEFD002C4D
:10823000DAD0A9E7BAF1010FD3D13246D5F8BC00A4
:108240000DF10601FFF728FC0446EDE71969284601
:1082500090476FF4FB639842D3D000287FF479AF46
:1082600060E720B119B112B1C0E901220160704785
:1082700010B5044618B910BD3C38FFF758FD20680A
:108280008442F9D10023C4E92E33D4F8B400BDE808
:108290001040FFF763BD034608463AB9F7F764BFDD
:1082A00010F8011B03F8011B0029F7D0013AF7D1A0
:1082B0001A70F3E708B1F9F705BD7047704740B190
:1082C000C368587810F001001EBF1878B0FA80F02B
:1082D00040097047EFF31183202383F31288BFF323
:1082E0006F8FFEE708B5FFF7F5FF10B5D0E9003452
:1082F00033B90020E268537843F00103537010BD96
:10830000204698470028F4D00028B8BF4042FF28F4
:10831000A8BFFF20E3681870ECE700F050BC00F045
:1083200041BC704710B400F10C04C0E9034410BC18
:10833000FEF7EFB82DE9F04F054689B0DDE9126789
:1083400091463B46324606A8059105F1140A00F015
:10835000E2FADDE90634CDE90234EFF311844FF09F
:10836000200888F31288BFF36F8F05F10C0B4A4683
:1083700028460599FEF759F830B184F31188BFF308
:108380006F8F09B0BDE8F08F3E43F6D0DDE90223E0
:1083900006A800F0E4FADDE906675A462146504691
:1083A000CDE90067FCF792FEEFF3118488F31288A1
:1083B000BFF36F8FDBE738B50446EFF31185202359
:1083C00083F31288BFF36F8FFDF7E6FF04F10C0013
:1083D00000F031FA30B1294604F11400BDE838400C
:1083E000FCF7E4BE85F31188BFF36F8F38BD416998
:1083F000836843EA010212F003020FD1C2600269EE
:10840000013A01FB023382689A4201D90020704789
:10841000C2681A604269C3609B1AF4E76FF01500E6
:10842000704710B5C0E904320023816083610446BF
:10843000FFF7DDFF0028A8BFC4E9004410BDF8B570
:1084400004460D46EFF31186202383F31288BFF311
:108450006F8FC7686FB900F0CBF950B1C76745613E
:1084600000F067F9314604F10800BDE8F840FCF778
:108470009DBEE3682B60A369E560013BA36186F3C1
:108480001188BFF36F8FF8BD202408B5EFF3118377
:1084900084F31288BFF36F8FFEF71DFCF6E790F9A7
:1084A0000E308B4201D0FCF73DBE002070470346E2
:1084B0000020C3E90033C3E9020070472DE9F84307
:1084C000994604460D4690469DF8203000F1080676
:1084D000EFF31187202282F31288BFF36F8F03B16D
:1084E0004568304600F084F958B10023C0F8148084
:1084F000C36700F01EF930463946FCF757FE0020EE
:108500000CE0B9F1000F1BD00821FDF79DF938B937
:1085100087F31188BFF36F8F6FF00B00BDE8F8830E
:108520000122C0F804800260016801F003015DB916
:1085300022680A430260626820606AB960600BE0EA
:108540004046C8F80090EFE72A68032A10D8016077
:10855000616839B9C4E90000042104F1100000F099
:1085600065FAC8E70A6802F0030202430A60E5E719
:1085700022F003020A4302602A6802F0030240EA82
:1085800002032B60E8E710B5044630B10268930798
:1085900003D0446809B100F076FA204610BD0123EB
:1085A00007B5009300230A461946FFF787FF03B07B
:1085B0005DF804FB002307B50A4600931946FFF750
:1085C0007DFF03B05DF804FB5AB18A4209D300F184
:1085D0001003C0E90212C0E90000C0E90433002022
:1085E00070476FF015007047012302688B4022EA44
:1085F0000303036022FA01F000F0010070477047A6
:1086000020B100228830114600F04AB9704738B5D1
:1086100004460D461022002100F0D1FA656038BDF5
:1086200013B501900846EFF31184202383F31288D9
:10863000BFF36F8F01A9FCF7B1FA84F31188BFF380
:108640006F8F02B010BD10B5FFF7EAFF041E08DD02
:10865000EFF31180202383F31288BFF36F8FFCF7B1
:10866000D5FD204610BD70B50D46EFF311862023D1
:1086700083F31288BFF36F8FFCF7EAFA044686F3A0
:108680001188BFF36F8F38B14FF0FF324FF0FF33D7
:1086900005F11000FCF7A0F9204670BD08B5A02236
:1086A000002100F08CFA08BDEFF30580003818BFF8
:1086B000012070476FF057007047FCF789BDD0E983
:1086C000003213605A600023C0E90033704708B5D8
:1086D000FFF7F5FF437B23F002034373002383601E
:1086E00008BD38B504460D46FCF7FAFB637B43F042
:1086F00002036373E5B1A5602B689D4209D16B68E5
:10870000C4E900531C606C6012E06A689A42F6D0BB
:108710001B68002BF3D094F90E2093F90E108A42B7
:10872000F3D09142F1DD5A68C4E9003214605C6014
:1087300038BD10B5EFF31184202383F31288BFF303
:108740006F8FFCF7E5FB84F31188BFF36F8F10BDCB
:1087500010B50446183000F0C5F8EFF3118120235E
:1087600083F31288BFF36F8F627B12F0100204D084
:1087700081F31188BFF36F8F10BD2046BDE8104014
:10878000FCF7FABB08B5EFF31181202282F31288BF
:10879000BFF36F8F83680BB1FFF799FF81F31188E7
:1087A000BFF36F8F08BD38B50446EFF31185202362
:1087B00083F31288BFF36F8F437B13F0280F0BD125
:1087C00083680BB1FFF783FF637B51B903F0FB03B1
:1087D00020466373FCF79CFB85F31188BFF36F8F12
:1087E00038BD03F0EB03F3E701211838FFF7DBBFD7
:1087F00038B5EFF31185202383F31288BFF36F8F11
:108800000468A0420DD034B12046FFF760FF04F1A8
:10881000180000F067F885F31188BFF36F8F2046CA
:1088200038BD0024F7E710B5FFF7ACFFBDE81040F6
:10883000183000F057B838B5054604680020AC423F
:1088400000D138BD002CFCD02046FFF7ECFF2046BD
:10885000FFF76FFF2C680120A542F1E7EFF31181CC
:10886000202282F31288BFF36F8F027BD2070CD5D0
:1088700081F31188BFF36F8F002383F31188BFF357
:108880006F8F0423184602DF7047437B1B0704D514
:1088900081F31188BFF36F8F70470122FCF76CBB27
:1088A00038B5EFF31185202383F31288BFF36F8F60
:1088B0000468A04212D09CB1E16762612046FFF7D4
:1088C00006FF04F1180000F00DF82046FCF720FB2D
:1088D000012085F31188BFF36F8F38BD0020F8E7C2
:1088E0002046F6E710B5EFF31184202282F31288B8
:1088F000BFF36F8F03683BB1FCF73AFE002084F3AF
:108900001188BFF36F8F10BD6FF01500F7E708B542
:10891000FCF74CFF08BDB3F1FF3F08BFB2F1FF3FCA
:1089200070B504461D46164613D01A4315D06FF095
:1089300001024FF0FF33921B63EB0501002904DABB
:10894000FCF734FF821941EB0501C4E90021204600
:1089500070BD4FF0FF321146F7E70022FBE7B3F19D
:10896000FF3F08BFB2F1FF3FF8B5074616461C4669
:1089700010D054EA020311D0FCF718FFB0420A46A7
:10898000A14103460AD2F31A64EB0204C7E900349A
:108990003846F8BD4FF0FF331C46F7E70023FBE7EE
:1089A0002DE9F041846805460E46ECB16378012B51
:1089B00025D114F8533C9A0714D5A4F16007384622
:1089C000FFF731FF082E0CBF6FF003030023E361B4
:1089D00014F8533CDB0605D154F8483C13B938462B
:1089E000FFF7A7FE002323700020EB68A860C3F305
:1089F0008632164366F39433EB60BDE8F081022BB8
:108A0000F0D12378002BEDD054F8048CB8F1000F8E
:108A1000E8D004F11400FFF765FF0023A4F1140768
:108A200039464046E362FFF7FBFDDBE7034610B53E
:108A3000EFF31184202282F31288BFF36F8F006856
:108A4000834208D0D0E9003213605A600023C0E9A5
:108A50000033FFF7A5FF84F31188BFF36F8F10BDBC
:108A60000432D3B5044608D20026002741F00401A1
:108A7000CDE90067FFF75EFC10B9002002B0D0BD61
:108A800040F8044BFAE720B1011F50F8040CFFF73F
:108A900092BC704701460420FCF7C8BE10B56AB10D
:108AA0000139841810F8012B11F8013F9A4203D1C3
:108AB000A04201D0002AF5D1D01A10BD1046FCE723
:108AC00010B50139044632B111F8013F013A00F8FE
:108AD000013B002BF7D1002100F071F8204610BDBA
:108AE0000246014410B58A42134603D01C78013275
:108AF000002CF8D1181A10BDF0B5C3F137070446A1
:108B000003F01F031046FFB2082BE6B232D0102B41
:108B10003DD06508A40845EAC17544EA81748A0815
:108B20002D1942EB5102290941EA02716D1842EBFD
:108B30001212290A41EA02616D1842EB1222290C35
:108B400041EA02416D1842EB1242AD1842F10002B7
:108B5000EC0844EA4274D10804EB8402A6EB420517
:108B6000EDB2092D0CD90134A5F10A0541F100013E
:108B7000EDB212E0E40806F0070544EA4174C908C2
:108B8000303554EA010200F8015BBDD1F0BD240983
:108B900006F00F0544EA01740909092D84BFED1997
:108BA000EDB2EDE70A44431E914200D1704710B583
:108BB00011F8014B914203F8014FF9D110BD024465
:108BC0000346934200D1704703F8011BF9E7000008
:108BD0000148006870470000180F00207875FF7F7B
:108BE00001000000A51B000000000000E91C0000BF
:108BF0000000000005070000000000000521000043
:108C00007C8C000021470000000000004547000068
:108C10000000000091240000A48C000091240000BA
:108C2000908C0000E7730000000000009129000014
:108C3000B88C0000D92C000000000000011C0000CE
:108C4000000000006D19000000000000AD260000CB
:108C5000CC8C0000EB73000000000000254A0000EF
:108C600000000000216A0000E08C0000000000000D
:108C7000F48C0000C10100000000000072930000AD
:108C800080900000A0900000E5010020880F0020E7
:108C90007D930000BC900000EC900000E7010020F4
:108CA0002C10002089930000D4900000EC9000006C
:108CB000E901002038100020A99300002491000051
:108CC0006C910000ED0100209C00002095930000B5
:108CD0009400002010910000EB01002044100020BF
:108CE0006293000004000020588F0000E101002082
:108CF000D00300205B93000000000000689000009B
:108D0000E30100205400002000000000B96C0000C6
:108D100000000000B96C000000000000B96C000009
:108D200000000000B96C000000000000B96C0000F9
:108D300035320000FD73000000000000B96C000037
:108D400000000000B96C0000B88C0000BB7200008D
:108D500000000000B96C000000000000B96C0000C9
:108D600000000000B96C000000000000B96C0000B9
:108D70001D390000FD73000000000000B96C000008
:108D800000000000B96C000000000000B96C000099
:108D900000000000B96C000000000000B96C000089
:108DA00000000000B96C000000000000B96C000079
:108DB00000000000692D000000000000B96C0000F8
:108DC00000000000B96C000000000000B96C000059
:108DD00000000000B96C000000000000B96C000049
:108DE00000000000B96C000000000000B96C000039
:108DF00000000000B96C000000000000B96C000029
:108E000000000000B96C000000000000B96C000018
:108E100000000000B96C000000000000B96C000008
:108E200000000000B96C000000000000B96C0000F8
:108E300000000000B96C000000000000B96C0000E8
:108E400000000000B96C000000000000B96C0000D8
:108E500000000000B96C0000653B0000FD730000DD
:108E600000000000B96C000000000000B96C0000B8
:108E700000000000B96C000000000000B96C0000A8
:108E800000000000B96C000000000000B96C000098
:108E900000000000B96C000000000000B96C000088
:108EA00000000000B96C000000000000B96C000078
:108EB00000000000B96C000000000000B96C000068
:108EC00000000000B96C000000000000B96C000058
:108ED00000000000B96C000000000000B96C000048
:108EE00000000000B96C000000000000B96C000038
:108EF00000000000B96C000000000000B96C000028
:108F000000000000B96C000000000000B96C000017
:108F100000000000B96C000000000000B96C000007
:108F200000000000B96C000000000000B96C0000F7
:108F3000813D000006000000000200000002000069
:108F400000000000D89400000001000000000000B4
:108F50000338FDD87047000085070000D36A000081
:108F60006D090000B9090000990A0000B768000007
:108F70002B690000BF680000F1680000DB6800009A
:108F8000C56800000000000000000000056C000043
:108F9000F56B0000016C0000F36B000000000000A6
:108FA000000000000000000000000000E36B000073
:108FB00000000000956C00004800002040000020E8
:108FC000380000200000000030000020610E00008A
:108FD000310D0000850D0000F90D0000000000209B
:108FE000000000000600010002000000F08F0000F9
:108FF000000000004893000006000000E0FF0F00A2
:10900000000000205093000021000000E0FF062037
:10901000E919000000000000856D0000F91C000047
:10902000DB6D000000000000109000003490000094
:1090300004010000903A00201090000044900000CD
:1090400000010000B03B0020109000005490000090
:1090500003010000744300201090000064900000A1
:1090600008010000AC4E00202D6E00006B6E000069
:10907000F96D00008D2000005D2000000000000060
:10908000F1210000D12000008F6F0000A16F0000CF
:10909000896F00009B6F0000836F0000956F0000D8
:1090A00069210000016F0000636F000000000000F4
:1090B0009D6E00000000000000000000FFFF0000A7
:1090C00000288450000000000100000000D0005083
:1090D00000000000FFFFFFFF00258450000000009B
:1090E0000000000000D00050000000002525000016
:1090F000AD6F0000B96F0000CD6F0000D76F0000AA
:10910000E16F000091230000F56F000000000000F7
:109110008D7000006970000085700000897000008B
:10912000B570000000800050010000000000000049
:109130004891000000000010010000000000000045
:109140002A130020291300200080005054910000B1
:10915000010000005C910000040000001400000009
:1091600013000002160600011506000361710000DD
:10917000DD280000537100003D730000877100007E
:10918000AF710000E3710000F37100002172000074
:109190002D720000F371000011720000397200009E
:1091A00047720000557200008B7200008F72000041
:1091B000E9930000FC9300000F940000229400004B
:1091C00035940000489400005B9400006E94000009
:1091D000E48B0000E48B0000348C00003C8C000029
:1091E000748C00007C8C0000FF8FFFFFFF8FFFFF5F
:1091F000FE8FFFFFFE8FFFFFFD8FFFFFFC8FFFFF46
:10920000FC8FFFFFFB8FFFFF6D757465785F6672E3
:1092100065652063616C6C65642077697468204EB5
:10922000554C4C20706172616D6574657200000070
:1092300043616E277420696E697469616C697A652F
:10924000206D757465782C20776173204E554C4CD9
:109250000D0A0000436F756C64206E6F74206C6F94
:10926000636B20706F7765722073617665206D7512
:109270007465780048434920756172742054580021
:109280007372616D302E73686D0067656E6572690B
:1092900063002A2A2A20426F6F74696E67206E521B
:1092A0004620436F6E6E6563742053444B207632C4
:1092B0002E382E302D6132333836626663383430C2
:1092C00031202A2A2A0A002A2A2A205573696E6721
:1092D000205A6570687972204F532076332E372ECE
:1092E00039392D306263333339336662313132209C
:1092F0002A2A2A0A006D757465785F696E69742080
:1093000063616C6C65642077697468204E554C4CC1
:1093100020706172616D6574657200436F756C6475
:10932000206E6F7420616C6C6F63617465206D7565
:10933000746578206265666F726520696E6974690C
:10934000616C697A696E6700464C4153485F300032
:109350005352414D5F30000000000162745F68634A
:10936000695F69706330006E72665F62745F686324
:109370006900636C6F636B40353030300067706933
:109380006F40383432383030006770696F4038349D
:1093900032353030006D626F7840326130303000ED
:1093A00000010203040506070B7561727440383032
:1093B0003030000000000101010000010000000049
:1093C00020303030303030303030303030303000DD
:1093D00001756E72656769737465726564202573C3
:1093E000206275730A002573006D6574616C3A2004
:1093F000656D657267656E63793A20006D657461AD
:109400006C3A20616C6572743A2020202020006D37
:109410006574616C3A20637269746963616C3A20A7
:1094200020006D6574616C3A206572726F723A202B
:1094300020202020006D6574616C3A207761726E87
:10944000696E673A202020006D6574616C3A206E69
:109450006F746963653A20202020006D6574616C2B
:109460003A20696E666F3A202020202020006D652A
:1094700074616C3A2064656275673A202020202070
:109480000025733A2066726565696E67206E6F6E9F
:109490002D656D7074792076697274717565756566
:1094A0000D0A00756E657870656374656420627579
:1094B000666665722068656C6420636F756E74659E
:1094C000720D0A0072785F76710074785F767100B1
:1094D0004E53006D61696E00737973776F726B71B3
:1094E00000286E756C6C29002A666C6F61742A0006
:1094F000C36500000000000000000720000001001C
:10950000CC8C000000000000CC8C000001000000AA
:109510000200000000000000000000000002000047
:10952000180200203A0000002C0200203A0000003F
:10953000040200203A000000400200203A0000002F
:10954000F48C00000000000000000000000000009B
:109550006793000000000000F16D0000F51E0000A0
:1095600000000000F48C000078000020780000204B
:10957000000000000100000088000020880000209A
:10958000E08C0000FFFF0000FFFF0000AC000020A7
:1095900000000000000000000000000000000000CB
:1095A000000000002B13002020000000000000003D
:1095B0000090D003FFFFFFFF00000000000000004C
:1095C000000000000000000000000000000000009B
:1095D000000000000000000000000000000000008B
:1095E000000000000000000000000000000000007B
:1095F000000000000000000000000000000000006B
:10960000000000000000000000000000000000005A
:10961000000000000000000000000000000000004A
:10962000000000000000000008000000FF00000033
:109630000000000003000000000000008A9200000B
:1096400000000000A53B000000000000000000003A
:10965000000000000000000000000000000000000A
:1096600000000000000000007801002078010020C8
:1096700000000000B1580000C4010020BC0100201F
:10968000B401002000000000AC010020DD59000002
:10969000295900005D590000A55900004C11002017
:1096A0003A00003A501100203A00003A54110020CC
:1096B0003A00003A581100203A00003AD401002044
:1096C00098010020900100208C01002088010020DA
:1096D000010000000000000000000000000000FF8A
:1096E00000000000902A0020001000000000000090
:1096F000000000000402002004020020000000001E
:10970000000000000E0000001802002018020020D7
:1097100000000000000000000E0000002C020020ED
:109720002C02002000000000000000000E000000DD
:109730004002002040020020000000000000000065
:109740000E00000000000000000000005C0200208D
:109750005C0200206402002064020020000000007F
:109760000000000074020020740200207C0200202F
:109770007C02002000000000000000008C0200209D
:109780008C020020940200209402002000000000BF
:1097900000000000A4020020A4020020AC0200206F
:1097A000AC020020070007000100000000000000DC
:1097B00038900000B04200200000000000000000CF
:1097C000D0020020D0020020D8020020D8020020C1
:1097D0000A000A000100000000000000489000009C
:1097E000944D00200000000000000000FC0200205A
:1097F000FC020020040300200403002001000100FB
:10980000010000000000000028900000943B0020B0
:1098100000000000000000002803002028030020B2
:109820003003002030030020100010000100000071
:1098300000000000589000002C5F002015E015E0AB
:020000040100F9
:10000000F0B900211DC302019D30030109C30201A3
:1000100009C3020109C3020109C302010000000073
:10002000000000000000000000000000C9C4020140
:1000300009C302010000000089C4020109C30201D2
:100040004DC602014DC602014DC602014DC6020158
:100050004DC602014DC602014DC602014DC6020148
:10006000BD3603014DC602014DC602014DC6020157
:100070006F3603014DC602014DC602014DC6020195
:100080004DC60201A33603014DC602014DC6020151
:100090004DC602014DC602014DC602014DC6020108
:1000A0004DC602014DC602014DC602014DC60201F8
:1000B0004DC602014DC602012DE9F00791E8F8078F
:1000C000B2E802105B1854EB0C04B2E802104D4188
:1000D00056EB0C06B2E802104F4158EB0C08B2E8A0
:1000E000021059EB01095AEB0C0A80E8F80780412D
:1000F0000130BDE8F00770472DE9F00791E8F807F7
:10010000B2E802105B1A74EB0C04B2E802108D41E5
:1001100076EB0C06B2E802108F4178EB0C08B2E8DF
:10012000021079EB01097AEB0C0A80E8F8078041AC
:100130004042BDE8F00770472DE9F007524290E8D1
:100140007800B1E880071740DB1918EA020854EB81
:10015000080419EA020955EB09051AEA020A56EBE6
:100160000A0678C090E87800B1E8800717407B4124
:1001700018EA020854EB080419EA020955EB0905CC
:100180001AEA020A56EB0A0678C080410130BDE83F
:10019000F00770472DE9F007524290E87800B1E887
:1001A00080071740DB1B18EA020874EB080419EA01
:1001B000020975EB09051AEA020A76EB0A0678C00D
:1001C00090E87800B1E880071740BB4118EA0208C0
:1001D00074EB080419EA020975EB09051AEA020A28
:1001E00076EB0A0678C080414042BDE8F0077047D0
:1001F0002DE9F00152424FF0040890E8300091E8F8
:10020000C000A31B1340E41AF618EB1B1340ED1AB1
:10021000FF1830C0C0C1B8F10108EED1BDE8F0014F
:10022000704700BF00B592E8DC072DE9DC07B1E8B4
:10023000805702B4A7FB02510A95A8FB020B0918CC
:100240000020E7FB03105BEB000B00204041E9FBC3
:1002500002B00B91A8FB0351401800214941EAFB71
:1002600002011BEB050B0025E7FB04B568410025E7
:10027000E7FB0605694100256D41E8FB0615CDF851
:1002800030B0A9FB03B689190026EAFB03167541B5
:1002900000267641ECFB035610EB0B005FF0000BE1
:1002A000E8FB040B51EB0B015FF0000BE9FB041BB7
:1002B00055EB0B055FF0000BEAFB045B56EB0B06FE
:1002C0005FF0000B5BEB0B0BECFB046B0D90ACFBDE
:1002D0000230059C2D180020EEFB02504641002004
:1002E000E9FB04605BEB000B00204041EAFB04B03B
:1002F0005B180021E7FB04314D410021E8FB04516C
:10030000069C4E410021E8FB04615BEB010B0021E0
:10031000E9FB04B1484100214941EAFB04010E9385
:10032000A7FB0432079CB6180022E7FB04625BEBD4
:10033000020B0022E8FB04B250410022E9FB040258
:10034000514100225241EAFB0412049CED180023A3
:10035000E9FB04535E410023EAFB0463089C5BEB6A
:10036000030B0023E7FB04B358410023E8FB04031D
:1003700059410023E9FB04135A4100235B41EAFB86
:1003800004230F955DF8049B99E80006DDF80080D2
:10039000A9FB08541BEB040B0024EAFB08B4DDF8AE
:1003A000108060410024ECFB080461410024EEFB56
:1003B000081462410024E9FB0824634100246441DD
:1003C000EAFB0834DDF8048076190025EEFB0865A9
:1003D0005BEB050B0025E9FB08B568410025EAFB4E
:1003E0000805DDF8148069410025ECFB08156A4119
:1003F0000025EEFB08256B410025E9FB08356C4123
:1004000000256D41EAFB08450F96DDF80880AEFB3C
:10041000087680190026E9FB080671410026EAFBF0
:100420000816DDF8188072410026ECFB082673419F
:100430000026EEFB083674410026E9FB08467541AC
:1004400000267641EAFB0856DDF80C801BEB070B13
:100450000027ECFB08B778410027EEFB080779413D
:100460000027E9FB08177A410027EAFB0827DDF897
:100470001C807B410027ECFB08377C410027EEFB0A
:1004800008477D410027E9FB08577E4100277F414F
:10049000EAFB086708B000BD2DE9F14F87B0FFF710
:1004A000C1FEDDF81C8008F1200888E8FF00FFBCD1
:1004B00087E87F08BDE8F08F00B591E84C57A2FBB4
:1004C00002410194A2FB034524190020E2FB0650DF
:1004D0006D417F41641802940021E2FB0801A3FBF7
:1004E000034B654103950024E3FB060440417F4133
:1004F000091900246441E2FB0914FF0750EB0B00CB
:1005000004900025E2FB0A455FF0000BE3FB081BAB
:1005100049415FEA370714EB0B045FF0000BE3FB84
:10052000094B55EB0B055FF0000B5BEB0B0BE2FB94
:100530000C5BFF0F0020E2FB0EB000225141E6FBF6
:10054000061205910021E6FB084164417F416D18C8
:100550000021E3FB0A515BEB010B0021E3FB0CB133
:10056000484100214941E3FB0E010023E6FB09530A
:100570001BEB030B0023E6FB0AB358410023E6FB09
:100580000C03594100235B41E6FB0E13FF07544166
:1005900006946D417F41A8FB08265541079500222E
:1005A000E8FB09B25BEB0B0B7F4180180022E8FBF4
:1005B0000A0251410022E8FB0C125A4100235B4120
:1005C000E8FB0E230024E9FB0E340025E9FB0A15A5
:1005D00052190025E9FB0C256B410025EAFB0C357F
:1005E0006C4100256D41EAFB0E45FF075BEB060BF6
:1005F0000026ECFB0E564041494152415B416441AB
:100600006D417641AEFB0EE848F100087F00A9FB82
:100610000979784151EB0901AAFB0A7A7A4153EB37
:100620000A03ACFB0C7C7C4155EB0C0556EB0E062B
:1006300048F1000700BD00BF2DE9F14F87B0FFF77B
:100640003BFFDDF81C8008F1200888E8FF00FFBCB4
:1006500087E87F08BDE8F08F30B44FF0000310F852
:10066000014B11F8015B013A84EA050443EA0403F3
:10067000F5D1A3F101034FEAD37030BC704700BF3E
:100680004FF0000310F8012B013943EA0203F9D1BE
:10069000A3F101034FEAD370704700BF30B411F8E3
:1006A000014B12F8015B6C4000F8014B013BF6D1A5
:1006B00030BC70472DE9F00791E8F807B2E8021066
:1006C0005B1854EB0C04B2E802104D4156EB0C06DB
:1006D000B2E802104F4158EB0C08B2E8021059EB97
:1006E00001095AEB0C0A8941B3F1FF3374F1FF346D
:1006F00075F1FF3576F1000677F1000778F1000813
:1007000079F101097AF1FF3A51F100015B184C418E
:100710004D4156F1000657F1000758F1000859EB1A
:10072000D1795AEB010A80E8F807BDE8F007704775
:100730002DE9F00791E8F807B2E802105B1A74EBB4
:100740000C04B2E802108D4176EB0C06B2E8021000
:100750008F4178EB0C08B2E8021079EB01097AEBD3
:100760000C0A89415B184C414D4156F1000657F186
:10077000000758F1000859EBD1795AEB010A80E8DB
:10078000F807BDE8F007704718EB040859EB0509B6
:100790005AEB060A5BEB070B5FF0000C4CF1000C08
:1007A00018EB050859EB06095AEB070A5BEB070B38
:1007B00050EB0C005FF0000C51EB0C0152EB0C0203
:1007C00063414CF1000CB8EB070879F100097AF1AC
:1007D000000A7BEB040BA841B141A241B3416CF18B
:1007E000000CBBEB050BB041B941AA41BB416CF118
:1007F000000C4CF001068CF0020718EB060859EBD0
:100800006C095AEB6C0A7BEB6C0B70EB6C0471EBB4
:100810006C0572EB670653EB6C076CEB6C0C18EB1A
:100820000C0059EB0C015AEB0C025BF1000354F184
:10083000000455F1000556EBDC7657EB0C077047CA
:100840002DE9F14F87B0FFF7EDFCDDF81080DDF802
:100850001490DDF818A0FFF797FFBDE8000FFFF731
:1008600093FF03B05DF8048B88E8FF00BDE8F08FCC
:100870002DE9F14F87B0FFF71FFEDDF81080DDF89E
:100880001490DDF818A0FFF77FFFBDE8000FFFF719
:100890007BFF03B05DF8048B88E8FF00BDE8F08FB4
:1008A0001FB50B4B01A901934FF4B873ADF8083095
:1008B00008238DF80A30837803208DF80B30FF234E
:1008C0008DF80C3001F074F805B05DF804FB00BF42
:1008D000AD8A02011FB50B4B01A901934FF442737E
:1008E000ADF8083008238DF80A30437802208DF8DF
:1008F0000B3000238DF80C3001F05AF805B05DF88C
:1009000004FB00BF658F02011FB5002301A9012070
:1009100003930193084B0293084B1B78002B14BFE1
:10092000022301238DF80B30FF238DF80C3001F0EA
:100930003FF805B05DF804FB40010800880900217C
:100940001FB50A4B01A901934FF42673ADF8083087
:1009500008238DF80A30037800208DF80B308DF8CD
:100960000C0001F025F805B05DF804FB0D920201C2
:100970001FB50A4B01A901939023ADF80830082355
:100980008DF80A30C37804208DF80B30FF238DF8E2
:100990000C3001F00DF805B05DF804FB179302016F
:1009A0001FB50A4B01A90193A823ADF8083008230D
:1009B0008DF80A30037905208DF80B3001238DF86E
:1009C0000C3000F0F5FF05B05DF804FB65A00101F7
:1009D0001FB50B4B01A901934FF40873ADF8083014
:1009E00008238DF80A30837D09208DF80B30002311
:1009F0008DF80C3000F0DCFF05B05DF804FB00BFA3
:100A000061B400011FB50A4B01A9427D019378230F
:100A10008DF80B200222ADF8083008238DF80C2049
:100A200018468DF80A3000F0C3FF05B05DF804FBEE
:100A3000B1BA00011FB5002301A901930393054B2F
:100A40000293037E0B208DF80B3000F0B1FF05B050
:100A50005DF804FB080108001FB50B4B01A90193C9
:100A60004FF48C73ADF8083008238DF80A30C37D3D
:100A70000A208DF80B30FF238DF80C3000F098FF22
:100A800005B05DF804FB00BFA19E02011FB5002365
:100A900001A901930393054B0293437E0C208DF82B
:100AA0000B3000F085FF05B05DF804FB080108007D
:100AB0001FB50023427801A903930193074B0293CA
:100AC00003780F2013448DF80B30FF238DF80C3082
:100AD00000F06EFF05B05DF804FB00BF8800080061
:100AE0001FB572B6194B5D68E5B9BFF34F8F184952
:100AF000184BCA6802F4E0621343CB60BFF34F8F18
:100B000000BFFDE7B4FBF6F4D3B20132002CF9D1FB
:100B100003F110026A4402F80C4C0A2233B901A80E
:100B2000A847E2E7044600220A26EDE7013BDBB2D4
:100B300003F110040DEB0406B0FBF2F402FB140009
:100B4000303006F80C0C2046E8E700BF8809002189
:100B500000ED00E00400FA0513B5114C6846237C53
:100B60008DF80130E37B8DF80030A37BADF80430C5
:100B7000637BADF8023010F065F918B1DE21032077
:100B8000FFF7AEFFA07E10F0C9F908B1E121F6E74A
:100B9000607E10F0BDF908B1E221F0E702B010BDAF
:100BA000880900212DE9F34104460D4671B91C4B1B
:100BB00093F82E3053B9012101A80193FFF7F2FFFA
:100BC00020B94FF403710320FFF78AFF2368002D3B
:100BD000144F4FF0000603F10703DFF84C800CBF01
:100BE0002046002023F00703236000F0B9FE57F8E9
:100BF000043B0BB1404698470136102EF7D100F068
:100C000027FF031E09DB206818440DB1002804DB10
:100C10002060012002B0BDE8F0810020FAE700BFAB
:100C20008809002158000021900900212DE9FF4189
:100C3000B0FA80F60546039003A876093146FFF71F
:100C4000B1FF20B96FF00B0004B0BDE8F0818F4C0C
:100C5000A17B607B0331237CE27B033022F005FE25
:100C6000011EEFDB0398002D237A627A00F1030066
:100C7000134420F0030003FB01F1039008BF0020A0
:100C800001F044F8039B0DB9C342DBD41844A37AA6
:100C90000390C3B1E17D1944E37A1944FF29D1DC03
:100CA0000330002D628AC9B220F00300039008BF10
:100CB000002001F09BF8031EC4DB039818440DB913
:100CC0000028BFDB0390724F7B68F3B1617CE1B118
:100CD00094F82F300398002B00F1070014BF402335
:100CE000252320F0070014BF4FF481722822002D25
:100CF000039008BF002006F0BBFE031EA2DB039892
:100D000018440DB900289DDB0390217DC1B1A37A61
:100D10001BB97B68A3B1637C93B10398002D00F1EC
:100D2000070020F00700039008BF002013F0FCFB31
:100D3000031E87DB039818440DB9002882DB03905B
:100D4000544B1B68B3B1217BA1B10398002D627D88
:100D500000F1030020F00300039008BF0020984733
:100D6000031EFFF66FAF0398184415B90028FFF66D
:100D700069AF0390484B1B68ABB1A17D99B1039853
:100D8000002D00F1030020F00300039008BF0020B5
:100D90009847031EFFF656AF0398184415B900286C
:100DA000FFF650AF03903D4BD3F80080B8F1000F31
:100DB00019D0E17DB9B10398002DA37E00F10300A5
:100DC000227E009320F00300637E039008BF002082
:100DD000C047031EFFF636AF0398184415B9002824
:100DE000FFF630AF0390FB69BBB1217BA9B103983B
:100DF000002D227F00F1030020F00300039008BFC4
:100E0000002001F065F9031EFFF61CAF039818449B
:100E100015B90028FFF616AF039094F82700C0B16B
:100E2000039A94F821300332A17F22F0070219447B
:100E3000334642F00402C9B2039201F08BF9031E5B
:100E4000FFF600AF0398184415B90028FFF6FAAE74
:100E5000039094F82810002975D0039F002D628D0F
:100E600007F1070708BF002027F0070718BF38461B
:100E7000039722F060FD031EFFF6E4AE03981844CA
:100E800075B90028FFF6DEAE0AE000BF8809002130
:100E90005800002198000021A00000219C000021A2
:100EA00003901DB1618D38461DF0A6FA94F822100A
:100EB00000294AD094F82630002B46D00398002D04
:100EC000A28C00F1070002F1240220F0070092B288
:100ED000039008BF002022F02EFD021EFFF6B2AEE6
:100EE000039F3A4415B9002AFFF6ACAE033294F8DA
:100EF0002030A17F22F0070294F8260019443346DF
:100F000042F00402C9B2039201F016F9031EFFF683
:100F100099AE0398184415B90028FFF693AE0390D4
:100F20003DB1A28C384694F82210083292B21DF0DE
:100F3000E5FC236BA3B1039B05B123632833039323
:100F40004DB1002080E60F46ABE7002DF1D0002226
:100F500011461046EBE7002BFFF674AE039873E6DC
:100F6000002DEED1FAE700BF38B50546002844D081
:100F700021F092F810B94FF0FF3038BD2AF0D7FABF
:100F8000B0F5FA7FF7D81F4C1F486560002500F0C8
:100F9000C7FB402229461D4884F82E5021F0A0FCB2
:100FA0002622294604F10800257084F82F50256375
:100FB00021F096FC1B2240F20113627340F21B32B7
:100FC00023810123E28140F20232A37222821F2296
:100FD0002377F72362824FF40272A384FB23A28259
:100FE00044F6011263852283EFF3108472B601F098
:100FF000EBF82CB962B62046BFE76FF01500BCE7EE
:101000002846BAE788090021590B00015800002141
:1010100010B5002840F0AB80564C94F82E30032BCE
:1010200000F0A280A1B1002A70D00139142900F289
:101030009E80DFE801F00B1C1F2F575F783562653B
:10104000733B414E537D808E9195850013782372BA
:101050000020FFF7EBFD0028B7BF012302236FF04C
:101060000B0084F82E30A8BF84F82E3010BD137802
:101070006372EDE79378002B48D0D378002B45D0EE
:1010800013781A2B42D953781A2B3FD91368C4F816
:101090000D30DDE71378E27A934237D3A372D7E7B6
:1010A0001378A27A934231D8E372D1E71378A27A07
:1010B00093422BD8E375CBE713783BB35378013BCE
:1010C000DBB2F82B22D81388927823832A4B9A70AC
:1010D000BEE71078E07618F01BFEB9E71378ABB1E5
:1010E0002377B5E71378254A52680AB1012B0DD949
:1010F0006374ADE713886382AAE713782373A7E7C5
:101100001E491378C96921B9012B04D86FF0150065
:10111000ACE7002BFAD01378637599E71378082BA6
:10112000F4D8A37594E71388FF2BEFD823758FE7C6
:10113000137863778CE713780E2BE7D8A37787E7CC
:1011400013680F49C4F8223053684B6013890B8130
:101150007EE71378E3777BE7137884F8213077E72D
:10116000137884F8203073E74FF0FF307EE76FF09C
:101170002C007BE788090021A009002158000021EC
:10118000AA090021F8B50D46074660B359B311F01E
:10119000070428D1154E96F82E30012B02D16FF09E
:1011A0000B00F8BD032B02D14FF0FF30F9E700F040
:1011B000EBF90028F8D02846FFF738FD0028EEDBD1
:1011C000384621F0DDF886F834001BF073FA96F803
:1011D0003400316B11F00CF9FFF7BEFC03232046FD
:1011E00086F82E30DDE76FF01500DAE78809002178
:1011F00010B5084C94F82E30032B05D111F014F9DA
:1012000094F8340021F0D8F822F034FD002084F85E
:101210002E0010BD8809002150B1074B03F11402C4
:1012200053F8041B934240F8041BF9D10020704787
:101230006FF01500704700BF78580301074B10B5D9
:1012400093F82E4034B910F0D7FF054B054A2046DD
:10125000DA6010BD4FF0FF30FBE700BF88090021C6
:1012600058000021A1080001074B10B593F82E404B
:1012700034B910F0D5FF054B054A20469A6010BDE1
:101280004FF0FF30FBE700BF880900215800002124
:10129000D508000138B5094D95F82E405CB910F01D
:1012A000E1FF074B074A20465A60074A1A600123AC
:1012B00085F82F3038BD4FF0FF30FBE7880900215B
:1012C000580000210909000141090001054B10B532
:1012D00093F82E401CB924F05CFF204610BD4FF05F
:1012E000FF30FBE788090021054B10B593F82E402D
:1012F0001CB924F051FF204610BD4FF0FF30FBE732
:1013000088090021054B10B593F82E401CB924F034
:1013100046FF204610BD4FF0FF30FBE78809002153
:10132000054B10B593F82E401CB924F03AFF204627
:1013300010BD4FF0FF30FBE788090021074B10B5C7
:1013400093F82E4034B910F0A9FF054B054A20460A
:101350001A6110BD4FF0FF30FBE700BF8809002184
:1013600058000021710900010A4B10B593F82E4076
:1013700064B910F0ADFF084B084A20465A61084B8B
:10138000084A1A60084B094A1A6010BD4FF0FF3036
:10139000FBE700BF8809002158000021A1090001D6
:1013A00098000021FDA70101A000002141200001BB
:1013B000054B10B593F82E401CB923F0D0FF204602
:1013C00010BD4FF0FF30FBE788090021054B10B539
:1013D00093F82E401CB923F0CAFF204610BD4FF0F1
:1013E000FF30FBE788090021084B10B593F82E4029
:1013F00044B910F085FF064B064A20461A62064A99
:101400005A6210BD4FF0FF30FBE700BF8809002192
:1014100058000021050A0001D1090001094B10B54F
:1014200093F82E4054B910F089FF24F0AAFE064B21
:10143000064A20461A62064A5A6210BD4FF0FF3033
:10144000FBE700BF8809002158000021050A0001C0
:10145000D1090001084B10B593F82E4044B910F0A3
:101460008BFF064B064A20469A62064ADA6210BD96
:101470004FF0FF30FBE700BF880900215800002132
:10148000590A0001350A0001084B10B593F82E40A7
:1014900044B910F08FFF064B064A20469A62064A6E
:1014A0001A6310BD4FF0FF30FBE700BF8809002131
:1014B00058000021590A00018D0A0001074B10B5A0
:1014C00093F82E4034B910F0ADFD054B054A204687
:1014D000DA6310BD4FF0FF30FBE700BF8809002141
:1014E00058000021B10A0001074B10B593F82E40B7
:1014F00034B910F0AFFD054B054A2046DA6310BD44
:101500004FF0FF30FBE700BF8809002158000021A1
:10151000B10A0001074B10B593F82E4034B910F012
:10152000C7FD054B054A2046DA6310BD4FF0FF307A
:10153000FBE700BF8809002158000021B10A000123
:10154000074B10B593F82E4034B910F09BFD054BB6
:10155000054A2046DA6310BD4FF0FF30FBE700BFBD
:101560008809002158000021B10A0001026800200A
:10157000014B1A60704700BFC0090021014B1B6876
:10158000184700BFC0090021024B1868003818BF77
:1015900001207047C0090021F7B504462D4E071DF4
:1015A0002C48376011F0E0FF0228054606D1294992
:1015B000204621F070FA284603B0F0BD042842D13D
:1015C0003378092B0AD0252B1ED03146204621F036
:1015D000DEFAB0F5817F2DD3722112E005213E2085
:1015E00021F02CFA0028F0D1F37801A9327968466D
:1015F00043EA0223ADF8003021F069FE0028CFD085
:1016000053210820FFF76CFA1A213E2021F016FA28
:101610000028DAD17368694601A8C3F30F23ADF837
:10162000043011238DF8063021F0B3FE0028B7D026
:101630006521E6E70028B3D0A178207821F0FEF9F3
:101640000028B8D1ACE70828B5D10249204621F0DE
:101650005AFAB0E7C4090021074B4FF0FF3141F6B9
:10166000FF72C3E9001205490022C1E900221F21CF
:10167000C3E90212704700BF00000021C80A002120
:101680003F280CD801380B4BC0F3421200F01F006A
:1016900053F8223023FA00F000F001007047FF28D1
:1016A00006D04038044BC0F3421200F01F00EFE7B1
:1016B0000120704700000021C80A0021074B0146A5
:1016C000006849681A4603C240F48C221A6041F04F
:1016D000107242F4FF625A60704700BF00000021A0
:1016E0000246024B0068516803C37047C80A0021D4
:1016F0000246024B0068516803C37047080000218E
:101700000138064BC0F3421200F01F0003EB8203C6
:101710009B6823FA00F000F00100704700000021F0
:10172000014B1860704700BFD00A002110B5FFF7C9
:1017300093FF22F061FF034B04461B6803B19847F7
:10174000204610BDD00A002138B5274B0446D3F8F7
:10175000A022D3F8A412013106D1D3F8A8324FF653
:10176000FF719BB28B423DD0D3073BD51E4DD5F8C0
:10177000A422D5F8A832C4F80120A4F80530C3F398
:10178000072363F03F03A371D5F89032013323D0D0
:10179000D5F8943201331FD0D5F8983201331BD0DD
:1017A000D5F89C32013317D0002010F0B5FF98B95E
:1017B000D5F89002D5F89412D5F89822D5F89C3235
:1017C000C4F80700C4F80B10C4F80F20C4F8133095
:1017D00001230020237038BD10220021E01D21F0DC
:1017E0007FF8F5E70023F4E70000FF0170B5274D0F
:1017F000102200210446D5F8A06221F071F81022D1
:101800000021A01821F06CF8D5F8803201330BD1FB
:10181000D5F88432013307D1D5F88832013303D1AA
:10182000D5F88C3201330BD0D5F88002D5F884126C
:10183000D5F88822D5F88C3220616161A261E3611C
:10184000002010F069FF08B9F3071CD40F4BD3F840
:10185000902201320BD1D3F89422013207D1D3F870
:101860009822013203D1D3F89C2201320BD0D3F855
:101870009002D3F89412D3F89822D3F89C322060C7
:101880006160A260E360002070BD00BF0000FF0146
:1018900070B50C88C27CA6B2C4F30E04931C0588F4
:1018A00004F114021D44825AADB21A4443882A44FA
:1018B000013AB2FBF5F202FB054292B29342044BAD
:1018C0008BBF3340B34313439BB20B8070BD00BF4B
:1018D0000080FFFF4A1E062A08B50346084604D8C2
:1018E0004FF4D1711520FFF7FBF8094A914202D954
:1018F00040F2A311F6E711B903B1196008BD2BB18D
:101900001B680022C3E901211A1D1A600430F5E7A3
:10191000FAFFFF7F10B5114B00EB41041A78638981
:10192000B3FBF2F303FB0223013A1A44B2F5706FE2
:10193000027928BF00231A448378B2FBF3F01944DC
:1019400003FB1020091AB1FBF3F003FB101313443F
:101950006FEA43436FEA5343638110BDD40A002109
:10196000124B10B5E0B15A78022A04D040F22B1184
:101970001720FFF7B5F803225A70026812F007012A
:1019800002D04FF49871F3E75C685A602244BDE8D6
:101990001040026003F10C009A60402220F0A0BFCA
:1019A0000122C3E901005A7010BD00BFD40A002112
:1019B0002DE9F041254E96F801E00EF0FD0CBCF14A
:1019C000010F04D040F245111720FFF789F891F874
:1019D0000680B8F1080F02D940F24711F4E7CF7939
:1019E00097B345467B1D7268022D4FEA430402EB14
:1019F000430338BF02256A1E6D421344C8F100023A
:101A00002B408D884544013D2A40B2F5803F02D3EA
:101A10004FF4A971D8E7BEF1030F12D106EB800095
:101A20001C1BC56815B140F25711CDE7C460A77003
:101A3000228084F803C0087A09682071080C21818B
:101A4000E08007FB02337360BDE8F081D40A002117
:101A50002DE9F047364C6378012B65D0032B04D079
:101A600040F267111720FFF73BF8D4E901329A42A0
:101A700002D04FF4B571F5E7002325460F221E462C
:101A8000994605F80C3B55F82200013A58B190F8F8
:101A900004808178B8F1FF0F2FD180F804908E4236
:101AA0003CBFCEB20123511CEDD103B126700F26ED
:101AB00040F6FF6955F826709FBB013EFAD2042319
:101AC00000206370BDE8F08755F82CE0BEF1000FF0
:101AD00006D09EF804A0C24504BF9EF802E07744F9
:101AE0000CF1FF3CBCF1000FEEDA3944FF2907D9B5
:101AF00003B126704FF48371B4E794460027F1E7F1
:101B00000771CCE707EB410308F101083846A3F859
:101B10000A90FFF7FFFE5FFA88F1BB788B42F1D89D
:101B2000CBE74FF00008F6E7022360686370C9E76F
:101B3000D40A0021034B03EB8003D86800B18078FE
:101B4000704700BFD40A0021F8B54FF6FF73054671
:101B50000380184B03EB8103D868B8B1867803790A
:101B6000B3FBF6F206FB1233DBB219460A1D00EB9B
:101B70004202B2F902705488002F09DB0131B1FB37
:101B8000F6F206FB1211C9B28B42EFD10020F8BD6C
:101B9000FF29FBD0C4F30E03C4782B8024B94FF483
:101BA000D9711720FEF79CFF5380BDE8F84021F063
:101BB00017BE00BFD40A00211D4B03EB810370B593
:101BC000DC68054644B3030404D54FF4E0711720E4
:101BD000FEF786FF0146204621F0E5FDFF2801467D
:101BE00004D02046BDE8704021F0FABDA078B5FBD6
:101BF000F0F300FB1353DBB219460A1D04EB420657
:101C0000B6F90260002E09DB0131B1FBF0F200FBF6
:101C10001211C9B28B42F0D1002070BDFF29FBD058
:101C20008B4204EB42021CBF0023E3705580D8E7CF
:101C3000D40A0021094B03EB8103014610B5DC688F
:101C4000204621F0B0FDFF28014604D02046BDE823
:101C5000104021F0C5BD002010BD00BFD40A0021F6
:101C6000F8B5104B074603EB81030146DC682046BC
:101C700021F099FDFF28054611D0E688238953EA13
:101C8000064606D00146204621F0AAFD0146384608
:101C9000B04720462946FFF73DFE0020F8BD05204D
:101CA000FCE700BFD40A002138B50E4B0446827908
:101CB00003EB8203D86808B9052038BD8278E17942
:101CC0009142F9D24B1CE37100EB41035D89B3F9FA
:101CD0000A30002BF3DBA58021F082FD206000207C
:101CE000EBE700BFD40A002108B5074B03EB8103E3
:101CF0000146D86821F057FDFF2804D140F2262183
:101D00001720FEF7EDFE08BDD40A002170B5044689
:101D100010F003000E4603D04F211820FEF7E0FE1E
:101D2000FFF7D8FD054624B1034831460460FFF7AC
:101D3000D1FD284670BD00BF200B00212DE9F14FD9
:101D4000DFF870B01E4607460D46DBF800309046BF
:101D50009DF828A09DF82C901BB961211820FEF752
:101D6000BFFE52460921404621F08DFB4A4684B20F
:101D70000921304621F087FB81B2DBF800002144C5
:101D800021F0E6FC386018B9286001B0BDE8F08F9A
:101D900004445346414609222C60386821F01FFB59
:101DA0004B4609223146286801B0BDE8F04F21F0CA
:101DB00016BB00BF200B002170B50E46044621F073
:101DC00075FB0546304621F071FB044B2A1821466D
:101DD0001868BDE8704021F0DFBC00BF200B002177
:101DE000014B186821F0A8BC200B00211F2AF8B570
:101DF000044613460ED89200033222F00303B3F5D3
:101E0000803F2DD2184DACB1A00710D05F21092022
:101E1000FEF766FEFF2B4FEA420204D9FF339A42D7
:101E2000A8BF1A46E8E77C2AB8BF7C22E4E72970FD
:101E30006C602B8122F0030228230127120403FB8C
:101E400001F06B680025120CEEB28E4200D3F8BD93
:101E500014B126181F705E60104401352833F3E773
:101E60004FF0FF30F3E700BF240B0021144A00219C
:101E700038B553681478C8B2844203D8AB2109201E
:101E8000FEF72EFE1846013128330578002DF2D0DA
:101E900000218170012412898161051D447092081E
:101EA000C16100F12001446821F8022B994245F8F4
:101EB000044B1444F8D100234361037038BD00BFC4
:101EC000240B00210A4B1B89B3F5FF7F4FEA9300D7
:101ED00006D25A089B1A9BB2984238BF18467047E0
:101EE000B3F5EE6F01D8FF22F4E740F27263F3E737
:101EF000240B00212DE9F8434B7880460C4602F074
:101F0000040602F0FB07D3B1DFB12E4BD4F80490E6
:101F10001D89B7BB0123AD084A46211D637004F13A
:101F2000280004F12003A761E76123F8025B9842CF
:101F300041F8042B2A44F8D10023636101E0002F0B
:101F4000E3D0FF23A370002E18BF0226A3191B7D28
:101F5000032B03D1022F1CBF0136F6B2A3190122B5
:101F60001A7506F10C02002304EB860624F81230E1
:101F70007268A3704046C8F80020A8F80430BDE895
:101F8000F883002114226170A01820F0A9FCB5F597
:101F9000FF7F0FD26B08ED1AADB209EB0502C4F852
:101FA00004902584A2606384C4F80C90A584226107
:101FB000E384C6E7B5F5EE6F4FF0FF03EBD940F2CF
:101FC0007265EAE7240B0021F7B5D2000B684000E8
:101FD000002502F07802CDF8013000F006008B8871
:101FE0000243ADF805300D4B42F001021E785F68E8
:101FF0008DF80020EBB29E4201D800240AE0C5EB28
:10200000C5040722694601353C44204620F08CFB7C
:102010000028EFD1204603B0F0BD00BF300B0021F7
:10202000014B1878704700BF300B0021034B002193
:102030001A785868C2EBC20220F052BC300B002163
:1020400010B50C4650B1830703D020214120FEF784
:1020500047FD044B58601970FFF7E8FFC4EBC4005C
:1020600010BD00BF300B0021F8B504460D461646E2
:10207000FFF7AAFF034630BB144A92F800C0576826
:10208000DAB2944501D807201CE0C3EBC302013348
:10209000B85CB918024610F00100F1D1630022F0DB
:1020A0007F02F60003F0060306F0780643F0010312
:1020B000334313430A4602F8013B2B68C1F8013051
:1020C000AB889380F8BD1220FCE700BF300B0021E5
:1020D0002DE9F84305460C46F7200521914621F0ED
:1020E000D2F9061E22DB1DB906FB04F0BDE8F88319
:1020F00015F0030703D098211920FEF7F1FCDFF853
:102100003480C8F81050A5B2A8F81460BBB29D4244
:10211000EAD9B8F814C04B46D8F810000522F721C8
:1021200007FB0C00013721F05AF9EFE74FF0FF30C1
:10213000DCE700BF380B002107B5CDE900230B46D3
:1021400003490246081D21F043FD03B05DF804FB7E
:10215000500B002113B5064CCDE900230B46024677
:1021600004F1080104F10C0021F032FD02B010BDB1
:10217000500B0021024B0146186821F01BBD00BF27
:10218000500B0021024BD3E9002121F047BD00BFD5
:10219000500B0021034B1B28D3E9022138BF1B2021
:1021A00021F03CBD500B0021024B0146D3E9002039
:1021B00021F0F2BA500B0021024B0146D3E9022074
:1021C00021F0EABA500B0021144B012200214FF0FC
:1021D000FF309A60C3F80012C3F80803C3F8001573
:1021E000C3F804259A60C3F808034FF48040C3F88D
:1021F0000015C3F8042503F5805341F6F872084929
:10220000C3F80825C1F88000BFF34F8FBFF36F8F6D
:10221000C1F88001C3F80825704700BF00E0004105
:1022200000E100E08C463022064B00B50CF8032B91
:102230008E4607CBCEF80300CCF80410CCF808206B
:102240005DF804FB6C0B002110B5154C1BF0A2FAD5
:102250001AF0DAFB0021636A608C9847237E9BB9F1
:10226000104B628C93E8030012F0E8F9E36A1888D7
:1022700012F00EF9636B94F8301094F8310098471F
:10228000002384F8383010BD94E8070004F10C03F3
:1022900083E80700044904F1190025F016FCDFE784
:1022A000600B0021880B002125220001034B93F8CD
:1022B000383003B97047FFF7C7BF00BF600B00217C
:1022C00040F21F41062008B5FEF70AFC08B5094B8D
:1022D00093F83820022A07D1DA7A42F00102DA7242
:1022E000BDE80840FFF7B0BF40F253212720FEF7BA
:1022F000F7FB00BF600B002138B5364D044695F85A
:1023000028300BB1C2071FD4012924D82B6C2046DA
:10231000984700B395F83000E8B995F82820E2B165
:102320008CB995F84430D806C3F300142ED4EB6C66
:1023300023B30123AAB16A8F910713D5EB6BD87829
:10234000023818BF012038BD6B8F1B07DCD5EB6B43
:10235000DB78022BD8D1012038BD002CE1D12046FA
:1023600038BD6A8F002AF6D16A6D107803EA101022
:102370002043C0F1010000F0010038BDB5F8503035
:10238000B3FA83F35B09002AEBD0D4E7E96B0B784F
:1023900003F00303032B02D1CB78022B18D0A86CD7
:1023A00021F02DF948B9EB6B1B7803F00303032BE5
:1023B00006D195F828200446B9E795F82820B6E715
:1023C00010F06CF980F0010095F82820C4B2AEE757
:1023D0000024ACE7600B0021F8B5234C0646E56A03
:1023E000636D95F8A42005F1900794F85C00A3654F
:1023F0000AB1031DD8B2FF2895F87D1004D11EB98B
:1024000095F87C30994202D01AF0E6FC3A7D22B36E
:10241000206E1BF0D3FA94F82830216E003BA06D9B
:1024200018BF012384F88030D7E91E23C4E91E2396
:102430001AF088FA46B995F87D30033B012B94BF1A
:10244000282000201BF058FB95F87C1000201BF082
:1024500047FC022384F83830F8BDA06D1BF0AEFABB
:102460001AF0D2FAE6E700BF600B00212DE9F04137
:10247000394C82B006460F4694F83830E56A012B95
:102480005FFA83F805F190055ED12B796BB1638F0C
:102490000021042043F0040329716387636A98478D
:1024A00094F828300BB185F80680E16B0B7803F0C7
:1024B0000303032B31D04B7863B30223AB722B7D24
:1024C000DBB194F82830003B18BF012384F880303A
:1024D000D5E91E23C4E91E23E36A94F85C2093F82F
:1024E0007D30013BDBB2032B33D81C490020CB5C91
:1024F000009001201A491AF0BBF9012F05D126B925
:1025000031463046FFF7F8FEC8B102B0BDE8F041F1
:10251000FFF79ABE0123AB72D1E7AB7A63B9638F41
:10252000022043F002036387636A9847E16B0B78EC
:1025300003F00303032BBED10323AB72BFE702B04A
:10254000BDE8F041FFF748BF40F2A4412720FEF765
:10255000C7FAFFF7B5FE00BF600B0021F44E030180
:10256000C80B002170B5804C002382B0E56A8DF85D
:10257000053095F8A42005F1900694F85C300AB176
:102580000433DBB2FF2B11D180B995F87D3095F87B
:102590007C108B4202D0FF201AF01EFCB37A032B72
:1025A00000F2DD80DFE803F0051F817195F87C10F3
:1025B000F1E794F8C2306D48ADF80630A5F86C30FC
:1025C00010F046F8002840F095800DF105020DF15D
:1025D0000601A06C20F092FFE06320B196F8513024
:1025E000002B00F09E80624B1846E363F37ADB0019
:1025F00003F00802037803F0F3031343327B9200E5
:1026000002F00402134303F0EF0203F00303032B71
:10261000027002D1C378022B11D0A06C20F0EFFF22
:1026200048B9E06B027802F00303032B07D010F0E7
:1026300035F800286ED1E06B027842F0100202708B
:10264000F37C13B14378002B41D11BF0B7F91AF09A
:10265000DBF9E66B11F070F820B1337803F0030377
:10266000032B5AD095F87D1001201BF039FBE26B4B
:10267000012340491088927884F8C430A4F84400BB
:1026800084F838308A7002B070BD38480FF0E0FF2F
:1026900000285AD0E06BC3781B2B14D1012105F11F
:1026A00010001AF0C9FBE06B0DE0B5F86C300DF1CD
:1026B00005020DF10601A06CADF8063020F01EFFFA
:1026C000E063002846D0012384F8C3308EE7206EF3
:1026D0001BF074F994F82810206ED6E91C23B1FA87
:1026E00081F6E16B7609C4E91E2384F880601AF054
:1026F00029F9AEE7638F4FF48070E16B43F4807388
:10270000626A638790470121E06B7171C3781B2B6C
:10271000D9D1C4E7E06B027891E701201CF03EFFBD
:10272000A0E79DF8053043B1BDF8061025F091F9FA
:102730000123E06B84F8C33058E7038001218370E4
:10274000E06B24F007FFE06BEEE740F2FD2127206D
:10275000FEF7C6F940F2F3212720FEF7C1F940F257
:102760000B312720FEF7BCF9600B00219C0B0021E8
:10277000F00B0021A40B00210D4B0E4A70B50E4C3E
:102780001A6094F838301BB1E1212720FEF7A8F930
:1027900003F0FF0206460D46227611F047FF0121A5
:1027A00004F1900024F0D6FE6665256670BD00BF7A
:1027B000A4000021B4300001600B0021074A10B5CD
:1027C00092F8383013B10C24204610BD03F0FF04FA
:1027D000147611F02BFF204610BD00BF600B0021C6
:1027E000024B012283F8C520704700BF600B002117
:1027F0002DE9F04184B0BC4C02AD85E8030094F8AB
:1028000038100A98002940F0A081002B18BF002A38
:1028100000F09B81B0FA80F14909002800F0958111
:10282000236404F12803606384F8C51084F8301031
:1028300084F8C61084F8311084F8C41084F8C310EA
:1028400061876184626295E8030083E80300E56ABA
:102850001AF026FB1AF0D8F895F9800005F19006D9
:102860001AF02AFCA86B1BF08DF8286A1AF02AFCD3
:1028700096F824001AF030FC94F82870EA6941F6C2
:102880004B53002F00F0B6809A4200F228814D2071
:102890001AF0F8F901201AF089FD732195F87D20CE
:1028A00001201AF0A5FD914B18681BF071F8D5E9CD
:1028B0000523A264C4F8C83095F88B303BB9D5F82D
:1028C000843023B1F18F32898A4200F02881D6F812
:1028D0008410D6F88C30864FD6F88000D6F8882041
:1028E0000FC7D6F8903094F82810C4F88130D6F885
:1028F0009430C7F80D30002940F0BB80E36A93F8AC
:102900009E20263A012A40F2848093F89F20262AAE
:102910007FD093F87C70032F08BF042705F144088B
:102920003946404625F040F9394624F0D6F9B5F845
:102930005030024695F87D104046934228BF13461A
:1029400084F8C23025F0FDF895F87D1096F81480D3
:102950000429B5F8587008BF032124F0BEF9B8F176
:10296000000F01D1043080B2B84228BF3846C7B248
:1029700084F8CC7010F0E0FE10B12B2F38BF2B275D
:1029800094F8280084F85C70002857D1F37CDBB100
:10299000012395F87C1084F880300139D6E91C2396
:1029A000C9B2C4E91E23EA6941F64B539A4298BF63
:1029B0000420032900F2CE8000224E4B0092FB221D
:1029C0005B5C4B4919F054FF0120FFF7CBFD00235E
:1029D00096F82400C4E90033A360D5F88C302A8827
:1029E00031892071618022800BB101221A6004B00C
:1029F000BDE8F0819A427FD84D201AF043F938465D
:102A00001AF0D4FC7D2195F87C2000201AF0F0FC0F
:102A100049E793F87C7093F84232002B3FF47EAF85
:102A2000FA1E012A40F28880DA1E012A40F28480D0
:102A3000012F72D0012B70D002276FE7337DA3B135
:102A400095F87D100120013984F88000C9B2D6E9DB
:102A50001E230329C4E91E237CD8264B3A465B5C1F
:102A600000210091224919F003FF0120FFF7B4FC77
:102A7000ADE7E26A92F89E30A3F12600012827D93B
:102A800092F89F70262F23D0A3F12100134601282E
:102A900001D8242F4AD100293FF43BAF242F7FF4E3
:102AA00038AF92F84E3192F87C7092F8752013404E
:102AB0005A0741D413F0010240D19B077FF52EAF96
:102AC000FB1EDBB2012B37D9012F18BF022725E7E8
:102AD00092F8D63292F87C70002BA1D11EE7962096
:102AE0001AF0D0F89C21D9E6600B0021A400002147
:102AF000C80B0021F44E030196201AF0C3F8164BC0
:102B000095F87C2003EB42039988144B01F5FA7188
:102B1000A3FB013189097D3177E70127FEE6B5F88E
:102B200088100A44F28701221A60D0E692F84E31EA
:102B300092F87C705907BDD50427EFE6FB1EDBB287
:102B4000012B8CBF17460427E8E640F26F112720BF
:102B5000FDF7C6FFFFF7B4FBF44E0301D34D62103F
:102B600008B5124B93F8382092B193F8282022B977
:102B700093F83830012B14D108BD93F83820022A7D
:102B80000AD1DB6AD3F81802BDE808401AF04EBF3C
:102B9000BDE80840FFF758BB40F235212720FDF77C
:102BA0009FFF40F231212720FDF79AFF600B0021A3
:102BB000FFF74ABB014B1876704700BF600B00213E
:102BC000014B93F8C4007047600B0021034B93F84E
:102BD000C30010B9588CC0F300307047600B00215F
:102BE000024B588CC0F3C020704700BF600B00211F
:102BF000014B93F8C6007047600B00212DE9F041AE
:102C00001E4F820782B00546FC6A0E4604F190040E
:102C100011D4EB070CD5217BD4E91E32013342F1EC
:102C200000020129C4E91E320CBF002301232373D3
:102C300002B0BDE8F081FB6CDBB1B7F8502018465C
:102C4000B96D033291F801801FF0D4FD0DF102023D
:102C500001A9B865D7F8C80020F064FD019820F0FC
:102C60004BFD012230604146D7F8C80020F011FD2D
:102C7000CFE740F295412720FDF732FF600B00219E
:102C80002DE9F04F0023B74C87B00646E56A884629
:102C9000CDE9043394F8383005F19007022B40F069
:102CA000F781638C13F0400106D1636A4020984796
:102CB000638C43F040036384002E5BD03B7D002B8C
:102CC00040F02B81D4F858B09BF8013099B2A4F8A9
:102CD0005010002940F039810023E3649BF80090F4
:102CE000638CF97AC9F3800243F4007391426384E0
:102CF00000F0D380E26A94F8280002F1900A9AF872
:102D00000A20EAB1022A00F0988100218AF80A100C
:102D100020B19AF80630002B40F085819AF80530F2
:102D2000002B40F031819AF80B30D4F858B0012BC9
:102D30000CBF002301238AF80B30638C9BF80090B2
:102D4000397BC9F3C00243F400634FF0000A91429B
:102D5000638400F0A9804FF0000910F0EDFCF0B1A1
:102D60009BF8003003F00303032B18D101201CF063
:102D700015FC14E03A7D002A40F0EF8043F48063B4
:102D80004FF00009638494F8C630013384F8C630EC
:102D900095F87D30033B012B40F2B180CA46FB7CA5
:102DA00003B394F8283095F87C10B3FA83F3E869FC
:102DB00001395B09C9B284F8803041F64B5398421F
:102DC00094BF042000200329D7E91C23C4E91E2353
:102DD00000F263810022644B0092FB225B5C63493A
:102DE00019F046FDB8F1000F08D194F8C610012083
:102DF000FFF782FA0546002800F0BC8001251AF092
:102E0000A9FFB9F1000F38D1BAF1000F08D094F83A
:102E10002830002B78D1B4F809300133A4F80930F8
:102E200086B3B4F805300022013384F8C620A4F834
:102E300005304F4811F01AFB049830B120F05CFCCB
:102E4000E16A0022027210F0CDFB059B33B1E16A0A
:102E500000221A720C22059810F0A4FBC5B9638CED
:102E60001B0607D4636A294680209847638C43F089
:102E70008003638407B0BDE8F08F05A90220FFF747
:102E8000BDFEC1E7B4F807300133A4F80730D0E73E
:102E9000FFF7DAF907B0BDE8F08F397BC9F3C0025C
:102EA000B24691427FF457AF09F00301E26A032969
:102EB00002F1900265D143F48053012059460392F8
:102EC00063844FF00009638F107143F0010363873F
:102ED000636A9847D4F858B0039A137B013B18BF34
:102EE000012313739BF80130002B3FF436AF936F2F
:102EF00001339367D36F43F10003D3672DE70120BC
:102F0000CA461CF04BFB4AE7B4F80530B4F807108A
:102F10003A890B43134383D07DE719F0B9FD19F0CB
:102F20009BFDD4F858B000287FF4CEAE9BF801107A
:102F3000002946D09BF800303A7BC3F3C0039A4285
:102F400000F08E8089B2A4F85010D4F8C80020F0A8
:102F500077FBD4F858B0E064C0E619F0D3FD638C79
:102F60000CE700BF600B0021F44E0301C80B0021E9
:102F7000880B0021FFF7F6FAB9F1000F3FF444AFD8
:102F80007BE709BB8946A8E74FF000098AF805905E
:102F90000FF06EFB002800F08280638F4946082006
:102FA00043F008036387636A9847DAF870300133A7
:102FB000CAF87030DAF8743043F10003CAF874309C
:102FC000B1E6A4F8501087E69BF801100029D9D08B
:102FD00043F4805392F814900392638419F06CFECA
:102FE000042894F8CC30039A07D1B9F1000F14BF2C
:102FF0001B211F218B4228BF0B46D4F858B09BF8E9
:103000000110994232D8E36C002B3FD094F8C530C0
:10301000002B39D0636A002120204FF00009984727
:10302000D4F858B099E6638F10208AF8061043F060
:1030300010036387636A984770E604A9A06C20F0C8
:103040007FFA88B3DAF8703094F828000133CAF8B0
:103050007030DAF8743043F10003CAF8743054E683
:10306000012384F83130FFF7EFF803E794F83030AC
:1030700001204FF0000943F0100384F830301CF0B9
:103080008DFAD4F858B068E6B14626E7994664E66A
:103090004FF4A3612720FDF723FDFFF711F940F25C
:1030A00025412720FDF71CFD40F20E412720FDF7AA
:1030B00017FD00BFCD220001812C00016D2400010D
:1030C000AD2200012DE9F843002800F0E38004461A
:1030D000072900F2D380DFE801F0AB2525A7D12036
:1030E0009ECD0146204625F0EBFCD4F84C3100F192
:1030F000EC059D4240F2C680E81A0321402838BF03
:1031000040201EF039FC0346C4F84C5120461D46B1
:1031100025F09AFD002D00F09C802046BDE8F84384
:1031200025F093BD25F01BFD0023D4F81C21054696
:103130000E4684F8483184F85131BAB150EA01039F
:1031400014D0CA00C30042EA50721B1A62EB01029B
:10315000D4F838115B18D4F83C1142EB0102D4E9E1
:103160005601834272EB0103C0F09280022304F502
:10317000A47784F8503138461DF04AFE002800F04C
:103180008D8094F8683103F0FF01002B6AD16FF055
:103190000043D4E958029A4208BFB0F1FF3F12D071
:1031A0002046D4E9569825F08BFCD4F86031EC30F9
:1031B000D4F86421B3EB090362EB08021B1A62F135
:1031C0000002002A4BDB394694F818011DF00CFF71
:1031D00000286DD0D4E95601D4E94C32834272EB19
:1031E00001071FD255EA06071CD0C01A334661EB0F
:1031F00002012A461FF0BAF905FB01F1A5FB0053B5
:1032000000FB0616D4E94C213344551943EB010366
:10321000C4E94C5306E090F818011DF0D1FD0023DD
:1032200084F84031BDE8F883BDE8F8431AF0A6BD44
:1032300013F096F8D4F84C01DC381EF0FBFA90B38A
:10324000204625F0CEFC00283FF44BAF204625F069
:10325000FBFCD4E95623C4E94E23BDE8F88320469D
:1032600013F086F894F818011DF0AAFD002384F8E5
:103270004031AFE7F4213020FDF732FCF821302057
:10328000FDF72EFC2046C4F84C5125F0DDFCE0E7AC
:1032900001236CE7D7213020FDF722FC40F2926138
:1032A0003020FDF71DFC40F251213020FDF718FCC5
:1032B00040F296613020FDF713FC00BF2DE9F04F7E
:1032C000044689B000201F460E46914694F87DA022
:1032D000049023F0A7F894F800320B2B00F2188327
:1032E000704A94F89F8032F8135089F00103284403
:1032F000029385B2B9F1000F1AD0B4F8901204F518
:103300001879B4F898B0711AA6EB0B0B09B20FFA42
:103310008BFB0029C0F24982384694F84432032BD3
:1033200000F21083DFE813F0BD018301C4003A000E
:1033300094F84432032BE0D1B8F10E0FDDD1B4F88C
:10334000D432B342D9D1B4F81C222046B4F8923218
:103350001344C4F84032D4F84C32C4F83832E3692C
:10336000C4F83C3214F0F2F9D4F8DC32E2699A4243
:1033700005D004F1280027F0EEF8D4F8DC32E36140
:10338000D4F8D832E363B4F8D632A4F84030D4F895
:10339000E0326362022384F84432AEE7E36903FB60
:1033A00001F20492002F00F00A82B4F81C52002DA2
:1033B00040F0058284F85B52D4F84CC294F89E30F9
:1033C0000CFB1121262B049100F0088294F89F3009
:1033D000262B00F0038200283CD0002D3AD1D4E9FE
:1033E000A0E0D4E99E237245834180F0A68294F840
:1033F0007D00C31E012B40F2808203911AF0FCFE77
:103400004AF2A13CD4F88032274D8444A3F18301D1
:1034100094F87D00A5FB0C3CA0F1030ED4E99E239B
:10342000BEF1010FA1EB020303991944A1EB9C111A
:1034300040F27D8203911AF0DFFE00F2E730D4F80B
:103440004CC20399A5FB0030B4F81C52800901441A
:1034500010390491AB44AAF103030CFB0BFBDBB264
:103460000BF1300B012B4FEA4B0B40F2FF81504622
:103470000D4D1AF0C1FE4AF2A1330344A5FB03230C
:103480009D0950461AF0B0FE0BF1730341F64B5202
:103490001D44E36928449342044D286040F2218290
:1034A000049A6FE0044F0301D34D6210300C0021E9
:1034B000E36B2946D4F83C02184428F032F8294638
:1034C000C4F84802E06928F02CF841F64B53E26951
:1034D00094F87DA09A42C74D98BF0230C4F84C02C0
:1034E00050461AF089FEAAF1030A4DF64171BAF16D
:1034F000010F01442046A5FB013194BF282300237E
:1035000003EB9111803124F0B7FBB4F81C3213B9EE
:10351000002F40F0AD81D4F83C32E26B94F87DB0DE
:103520001344D4F84802ABF103011B1AC9B2049347
:10353000D4F838320129D4F84022B4F840A002FB74
:1035400003050AF1730A05F130054FEA450540F21B
:103550003D8158461AF050FE4AF2A1330344A54873
:10356000A0FB03239B095846039355441AF03CFEE5
:10357000039B049A1D44A04B28441860012384F83F
:103580004432E369D4F84C52D4F888125D1B6FF4CE
:10359000B3731D44D4F88C32854228BF0546891880
:1035A00004F1440043F10003C4F81852C4F8701247
:1035B000C4F87432002384F8603224F0C0FA28443E
:1035C000A4F89062C4F86402D4E99C23C4E9A2235D
:1035D00013F004FB20B1D4F864321E33C4F8643213
:1035E000B4F8081200238E1B84F8683236B29E426B
:1035F00002DD022384F86832B8F10E0F00F0FE807D
:10360000002F40F0FE8094F84432002B40F01981E6
:10361000494694F85C021DF0E7FC002800F07D812B
:10362000029B84F85832002009B0BDE8F08FD4F82E
:103630004C02E269D4F84052B4F81C32121AB4F8C1
:1036400040A09B4402FB01F1D4F84832EA430AF15E
:10365000730A049130339344D4F8382202FB0535C1
:1036600094F87D20D31E00FB0B55012B4FEA450536
:1036700040F2AE80104603921AF0BEFD4AF2A1332A
:1036800003445C48A0FB0323039A4FEA931B554471
:1036900010461AF0A9FD584B5D44049A284418605E
:1036A00081E094F87D1094F8160223F03DFB8246E9
:1036B000E06B2946DFF83CB1504427F032FF294641
:1036C000C4F84802E06927F02CFFE26941F64B5349
:1036D00005A99A4298BF0230C4F84C0206A81AF015
:1036E00041FB059B0093DDE90623D4E9A2011EF00E
:1036F0009DFB94F87D300546184603931AF07CFD37
:10370000039B4DF64171033B01442046012BABFB6B
:10371000013194BF2823002303EB9111803124F061
:10372000ABFAD4F89432E26B94F87D0004930392E0
:103730001AF062FD4AF2A133039AC318D4F8480282
:10374000ABFB0331049B933B13441B1A5344B4F863
:1037500040A05B1B00F130050AF1950AA3EB911321
:103760006D00049394F87D30DA1E012A33D918468F
:1037700003931AF041FD00F52340A130ABFB003B61
:10378000039B4FEA9B1B184655441AF02DFD049AE3
:10379000D4F894325D441849D31A2844B3F5A07F75
:1037A0000860C0F0BF80E369ECE6002359460120C1
:1037B00084F85B32D4E99E23C4E9A223ADE594F8F2
:1037C0005B52002D4FD00C490868DBE66523CAE642
:1037D0004FF0650B5BE74FF0650BD4E7B4F8D432DC
:1037E000F31A1A043FF5F7AD94F8D732002B18BF3F
:1037F0009A46F0E5D34D6210300C0021002F3FF4C3
:1038000007AFB4F83022CAB1B4F8320294F83412D7
:1038100000FB011101308A427FF7FAAE002B3FF422
:10382000F7AE0023A4F8320284F868320FF08AFF62
:1038300000F00700013084F83402E9E6A4F83222EF
:10384000E6E6D4F84C324846E169C91A23F014FA86
:1038500083B2002B3FF4DCAE129A0120002A3FF421
:10386000E3AE1380E0E6B4F81C52A5E5652508E652
:10387000E26BD4F83C3294F87D0003EB020A1AF0B4
:10388000BBFC4AF2A13394F87DB0AAF1930A034439
:10389000ABF10301D4F84802A5FB0323C9B2D4F865
:1038A0008022AAEB000A9B09012992440393D4E9E0
:1038B0009E23AAEB020A29D958461AF09DFC94F8D7
:1038C0007DB000F2E732D4F84802ABF10301A5FB6A
:1038D0000235C9B2AD09039BAAEB03022A44049244
:1038E00026E618462A4604AB594623F03AFA049ACB
:1038F00084F85B02E369286844E6AEF1E80E3C20F8
:10390000D4E99E23AEEB020E7144A0E53C25E2E72C
:1039100040F2B5310620FDF7E3F840F27B5130204C
:10392000FDF7DEF840F2C6413020FDF7D9F8B4F8D3
:103930001C523C20D4F84CC289E540F21A51302088
:10394000FDF7CEF840F232513020FDF7C9F800BF44
:10395000F0B585B0002800F015810446072900F273
:103960000081DFE811F09200080008007B00FE00F3
:1039700080008800FA001BF00FFED4E99E23801A15
:1039800061EB0301012871F10003C0F20D816FF0BA
:103990000102002382428B41C0F20181E3690BB135
:1039A000B0FBF3F394F89F200E2A00F0CF80B4F818
:1039B0009810B4F856220B449BB2D11A0D0454BF90
:1039C000531C01339BB2A4F8563294F85932B4F820
:1039D000561223B9B4F80C328B4200F0C680B4F80A
:1039E000D40002ADB4F89830B4F892220344B4F88D
:1039F000D20001326F4E013BA4F892221B1A9FB2F3
:103A0000336853B101390022204689B29847B4F88F
:103A10005612014489B2A4F856127B1A18046ED4C7
:103A20000023204600951A46FFF748FC00284AD19B
:103A3000D4F884303BB3B4F8CE20B4F856329B1A95
:103A40001BB2002B1FDDB4F888100B44013BB3FB05
:103A5000F1F303FB0123A4F8CE3014E005B0BDE878
:103A6000F0401AF08BB901201BF098FD05B0BDE8BD
:103A7000F040FFF79DB890F84432042B40F08B8063
:103A8000002380F8443205B0F0BD90F8583253B3AB
:103A9000B0F85632B0F8982093426BD09A1AA0F83A
:103AA0009830A0F80E222046D4E99C23C4E99E2336
:103AB00013F03AFD94F81332002BE4D005B0BDE8C2
:103AC000F04025F074BA012860D1B4F85612B4F869
:103AD0000832CA1A12042FD4BDF80830194489B22A
:103AE000A4F856128CE7B0F85432B0F89810B0F839
:103AF00054225B1AA0F89820A0F80E32D3E794F86D
:103B0000A220012328460394002A8DF808300CBF18
:103B10003E23082384F8C13010F02AFA204625F00D
:103B200048FA002394F85C0284F844321DF048F906
:103B3000202384F85C32A6E7BDF80820114489B23E
:103B40007A1A12F4004F18BF1946C9E7B4F8561292
:103B5000013189B2A4F8561241E7CB213020FCF79D
:103B6000BFFFCF213020FCF7BBFF013189B2A4F8A1
:103B7000561234E7B0F80C22D31AA0F89820A0F817
:103B80000E3290E7A6213020FCF7AAFF40F25461E4
:103B90003020FCF7A5FFC5213020FCF7A1FF40F243
:103BA00007613020FCF79CFF40F206613020FCF7F3
:103BB00097FF00BFA80000212DE9F043D0F81C3189
:103BC000002683B0054680F820610F46D0E956896B
:103BD00083F8162280F840610121D0F81C010FF013
:103BE000A7F9D5F81C41324631462046C4E99E89E2
:103BF00095F81831C4F8947284F85C32334684F82E
:103C00004462A4F89062C4E9A2890096FFF756FBCB
:103C1000D0B90123C4F84002C4F8380284F8443211
:103C2000A4F85602A4F8540284F85902B4F8983063
:103C3000A4F89202013BA4F8983019F035FE03B0C5
:103C4000BDE8F0431CF046BF40F2F3113020FCF712
:103C500047FF00BFD0F81C01704700BF2DE9F043BB
:103C6000002385B00322FF26CDE900338DF806201E
:103C70006846FEF719F8044620BB009D95F84031D0
:103C8000002BF5D085F868610121284624F0DFFF7C
:103C900095F84031002BEBD095F818011DF000FC91
:103CA00095F818011DF08CFF95F818011DF088F8A3
:103CB00000283CD085F840416846FDF7F5FF0446F2
:103CC0000028DAD0DFF87C800123002502264FF699
:103CD000FF7788F804301AE0029BE3B193F85C2286
:103CE000202A18D01888B8421BD00221FDF7A2FF65
:103CF000814608B390F85C021DF062FF99F85C02FF
:103D000089F844421DF05CF8202389F85C32CDE943
:103D100002558DF80E6002A8FDF7C6FF0446002884
:103D2000DAD0002388F8043005B0BDE8F08340F213
:103D3000DF113020FCF7D4FE40F22B113020FCF7CD
:103D4000CFFE00BF300C0021044B002242F2107164
:103D50005A71D9801A71FFF781BF00BF300C002162
:103D60002DE9F84390F84031002B76D1044688467F
:103D700001465648154603F0FF071CF0F5FF2028C2
:103D800006466AD05822394604F58C701EF0A8FD0C
:103D900084F81861C4F81C81FF2384F84031B8F11D
:103DA000000F06D00FF0E6FC00F00700013088F8A5
:103DB000340202234FF00008A4F8503184F84881FF
:103DC00027F0B7FB00F1BC062046B6B224F009FF8D
:103DD000002846D022F026FB00F5CD6128464FF0A2
:103DE000010989B227F09DFB2844C4F84C011BF05F
:103DF000D3FB3018A4F8268041F10001C4F8580123
:103E000084F820912046C4F85C1124F000FF0028BB
:103E100045D0A5F59D654946204624F051FE2D1A52
:103E2000C4F824514FF0FF326FF00043C4E9582327
:103E300004F5A47194F818011DF0D6F800283FD0BD
:103E400020460021D4E95623C4E94C23C4E94E237B
:103E500024F0FDFE3846BDE8F8830C273846BDE85F
:103E6000F8830146204624F02BFEDFF86480EC3016
:103E7000C4F84C01B8F8060008B1E08CB8B90644A3
:103E80001BF08AFB361841F10001C4E95661002D90
:103E9000C8D0AE1941F10001C4E95861C8E7EC3D52
:103EA000484624F0A4FF2D1AC4F82451BAE70FF0B5
:103EB00061FCB8F80630B0FBF3F202FB1300DEE75A
:103EC00040F2C1113020FCF70BFE00BFC5300001ED
:103ED000300C002190F840310BB90020704710B52C
:103EE0000446FF2380F86831012124F0B0FE94F8E5
:103EF00040310BB9002010BD94F818011DF0D0FA24
:103F000094F818011DF05CFE94F818011CF058FF9D
:103F100020B1002384F84031002010BD40F2DF11B1
:103F20003020FCF7DDFD00BF014B5871704700BF2A
:103F3000300C002190F8682182B910B502F0FF041E
:103F400090F8202112B90122104610BDD0E9493164
:103F50009942F9D912F00CFA2246F5E700221046F0
:103F6000704700BF10B5044618F0CAFE074B9A68A8
:103F7000824208D3E16941F64B52914203D9187944
:103F800080F0010010BD002010BD00BF300C0021EA
:103F900040F20B2108B523F077FEB0F5296F28BF5A
:103FA0004FF4296080B208BD90F81332002B73D112
:103FB000F0B503F0FF0590F8443285B00446032BBA
:103FC00001D005B0F0BD1BF0E7FAD4E99E23801ABA
:103FD00061EB0301012871F10003F2DB6FF00103D3
:103FE000834275EB01035ADBE369B4F89820002B98
:103FF00053D0B0FBF3F080B20132B4F80C3210446D
:1040000080B2A4F85402B4F854229B1A1BB2002BBD
:10401000D7DD94F85C021DF043FA0028D1D0FF23CD
:1040200084F85932B4F898500DF10E06B4F8D42043
:10403000B4F8D23015441F4F013DED1A3B68ADB2C4
:1040400063B1B4F8541200222046013989B298476E
:10405000B4F85432184480B2A4F85402B4F854327C
:10406000EB1A1B04ADD4B4F85412002301222046ED
:1040700089B20096FFF722F90028A2D0012813D1B7
:10408000B4F85432BDF80E2013449BB2A4F8543255
:104090003B68002BD5D1E1E770471846ACE740F20A
:1040A000AF513020FCF71CFD40F2F6513020FCF7F8
:1040B00017FD00BFA80000212DE9B043044682B0DF
:1040C000062900F29780DFE801F0041D0A1A232A6E
:1040D0006D004B4B1B7903F0FF02002B7CD00423B7
:1040E00084F8443219F0E0FB1CF0F4FC0023B4F82F
:1040F0009820A4F89232A4F8562284F8593202B0DB
:10410000BDE8B083032380F8443202B0BDE8B08339
:1041100018F01AFEC4E9A00102B0BDE8B08390F81F
:104120007D30C569033BD0F84C12DFF8D480012BF9
:1041300098F8053094BF4FF4BD794FF4A9798D42BA
:104140008CBF6D1A00251BB9436C9D4228BF1D46CC
:10415000D4F8187204F1440023F0F1FC0744022063
:104160001DF0B6FB0221ED1B25EAE575854228BF4F
:10417000054628461DF000FC00B92F444A46394642
:10418000204623F066FDE269D4F81832C8F808002A
:10419000D0181DF04FFB0028B1D140F2793130200A
:1041A000FCF79EFC90F87D502846033D1AF024F859
:1041B0004DF641710246134B012D20461144A3FBDD
:1041C000013194BF2823002303EB9111803102B009
:1041D000BDE8B04323F050BDB0F80C1201230092AB
:1041E000FFF76CF800283FF47DAF40F2CA61302041
:1041F000FCF776FC40F265713020FCF771FC00BFE3
:10420000300C0021D34D6210012A70B5064609D04A
:10421000022A14460D461ED04AB140F28F7130205A
:10422000FCF75EFC18F06CFDC6F8940270BD18F047
:1042300067FD224601462846FFF7BEFC32460F497D
:1042400095F818011BF094F90028EFD14FF4EF61B5
:104250003020FCF745FCD0F8941201222846FFF7E5
:10426000ABFC3246054995F818011BF081F900288E
:10427000DCD140F289713020FCF732FC5139000169
:10428000F8B5044651B1012960D1002380F82031EE
:1042900019F00AFBBDE8F8401CF01CBCC58C002DD1
:1042A0004CD12046D4E94C7624F059FC40194FF00B
:1042B000000341F10001C01984F848314FF00203B6
:1042C00046EB0101C4F85801C4F83001C4F85C1190
:1042D000A4F85031C4F8341194F8683103F0FF01A8
:1042E000002BD5D16FF00043D4E958029A4208BFA1
:1042F000B0F1FF3F0CD104F5A47194F818011CF043
:1043000073FE0028C4D140F2E9613020FCF7E8FBDD
:104310002046D4E9565624F0D3FBD4F86031EC3073
:10432000D4F864215B1B62EB06021B1A62F10002E7
:10433000002AE0DA204612F01BF8A9E70FF002FA93
:10434000E58CB0FBF5F303FB1505AAE740F29F717E
:104350003020FCF7C5FB00BF90F84001003818BFC3
:1043600001207047014BD880704700BF300C0021FE
:1043700006220B4603F8032BB0F809C0C27AA1F855
:1043800003C09A70704700BF18230B70704700BFBE
:1043900040F2A921322008B5FCF7A2FB70B5002835
:1043A00044D0437A04460E467BB300214089FDF792
:1043B00041FC054600283ED000880EF009F9002196
:1043C0002888FDF74DFC00283AD11321334604F12B
:1043D0000902293403F8031BD2F800C0103252F846
:1043E0000C5C103352F8080C52F8041CA24243F83B
:1043F00010CC43F80C5C43F8080C43F8041CEBD1D8
:10440000107800221870B27170BD036DD0F80E20C4
:10441000C3F80320428AA3F80720427B036D12F001
:10442000FD0F14BF012200229A70CEE740F2F22164
:104430003220FCF755FB40F2FE213220FCF750FB06
:1044400040F202313220FCF74BFB00BF044B00224C
:104450001B68A3F8BA2083F8BC2083F8702070474B
:104460003C0C002108B50EF01FFE034B187019F02C
:1044700091F9032008BD00BF1000002108B50EF01F
:1044800013FE024B024601201A7008BD10000021E5
:1044900038B50D4D2C6894F8893063B9002301219B
:1044A000204684F87010A4F8BA3084F8BC30BDE817
:1044B000384005F0DBB919F069FB18F045F9002325
:1044C00084F889302C68E9E73C0C002138B5114CA0
:1044D000002003F061FB256803F0F2FA2368E86727
:1044E000D86F60B103F028FB70B119F067FA0020B3
:1044F00019F002FB2368042283F8702038BD40F2D3
:10450000B6413220FCF7ECFA4FF497613220FCF709
:10451000E7FA00BF3C0C002108B50EF0C5FD044BC6
:10452000024600201A7003F08DFC012008BD00BF78
:104530001000002170B53D4C0646236893F87020AA
:10454000032A34D093F87020042A30D093F85430E2
:104550009B0731D16568002D4FD0236893F8542014
:10456000002A40D06EB3284622F0BDFF18B9284675
:1045700022F0D4FF20B3236893F87020022A4BD98D
:1045800093F87020082A4CD893F870102846A26837
:10459000274B12690B4452F8233098470C2827D830
:1045A000A368DB68BDE8704053F820301847D86F27
:1045B00003F0C2FA0546CEE703F0D6FA0546CAE78D
:1045C000236893F87020022A1CD993F87020082AD7
:1045D0001DD893F87010A268154B52690B4452F81D
:1045E00023309847DAE741F291313220FCF778FA2C
:1045F00041F2A4313220FCF773FA41F28B313220C0
:10460000FCF76EFA41F271313220FCF769FA41F29F
:1046100072313220FCF764FA41F211313220FCF79A
:104620005FFA41F212313220FCF75AFA3C0C0021B9
:10463000FDFFFF3F38B5144C236893F854309B07B7
:1046400019D16568DDB12368FF2093F8B91018F01F
:10465000C3FB284619F0B2F9236893F8B930033B3D
:10466000012B94BF2820002019F046FA2368072266
:1046700083F8702038BD03F077FA0546E2E740F290
:10468000DD413220FCF72CFA3C0C0021F0B5514CF6
:1046900000220E460546236841F2707083B0196D02
:1046A0005A72CA69B1F800C0A3F80AC0A2F57A7CB0
:1046B000844540F281804848A0FB0202C2F38F2269
:1046C0001A848A8C5A84CA8C9A844FF47F42DA8482
:1046D0004FF6FF721A85002D64D00121304622F07A
:1046E00024FE3278D209236893F8481009B1002AD1
:1046F00036D193F8860000210828596119833CD0EF
:1047000003F10E0203F10D010EF054FA00285BD004
:1047100023685A7B03F11A0742F002025A73002DF4
:104720003AD103F1980002683A608288BA8093F91E
:104730005810186D0EF09CFC2068284923F0BCF935
:10474000236827491A6D03F12A001488A3F833401F
:1047500092F8A62083F8352023F0B7F903B0F0BD16
:10476000427902F0C002402AC3D102685A618288AD
:1047700093F886001A830828C2D193F89E10D3F8C4
:104780009820B3F89C0059730021C3F80E2058827A
:10479000C3F81A10D983CAE70021304622F0C5FDBC
:1047A0002368C0E76068694622F072FC6368684667
:1047B0001A78C2F3801296E70A48A0FB0202920917
:1047C00002F5506292B27BE741F2DA313220FCF717
:1047D00087F900BF3C0C00215917B7D19D43000158
:1047E00071430001D34D621008B5002003F000FBB7
:1047F0000EF05AFC024B024601201A7008BD00BFA1
:1048000010000021034A0223106880F8703004F081
:10481000B1BE00BF3C0C002140F25A31322008B535
:10482000FCF75EF930B504788DB004F00F0402A9EE
:10483000224603F09DFC18F0ADFF0EF035FC204B36
:10484000042C187002D003200DB030BD1D49054660
:10485000039A0868147890F898108C42F3D1547831
:1048600090F899108C42EED1947890F89A108C427E
:10487000E9D1D47890F89B108C42E4D1147990F867
:104880009C108C42DFD1517990F89D209142DAD171
:104890009DF8191090F89E209142D4D17F2D0CD014
:1048A0007F2202A97C301A7090F82C30827A009511
:1048B00003F0B8FB03200DB030BDFFF7ADFF00BF24
:1048C000100000213C0C00212DE9F04F044687B078
:1048D00006290CD8DFE801F0AC34110B0B0B0400F7
:1048E000BA4D286890F88C30002B40F0CD8018F03D
:1048F00051FF032007B0BDE8F08F18F04BFFB34B1A
:10490000186890F854309D07F3D090F88C30002B45
:10491000EFD0AF4B93F900207F2A00F0098202927A
:10492000FF2590F886107F22CDE900511A702146AC
:1049300000F1420302227C3003F0C8FA0320D9E7D9
:10494000A24D867C2968012E91F88C3091F88D90CB
:10495000059391F8483083F0010B00F0B4800026F5
:1049600091F85420374612F0040000F0B48091F81A
:104970004D30002B00F0AF8091F88880B8F1080F1F
:1049800040F0AC8091F841800027C44620B36268B3
:1049900091F85B0092F800E0864500F062814FF0EC
:1049A000000A91F88520082A05D091F888009042E5
:1049B00008BF4FF0010A002F40F0F280BBF1000F5A
:1049C00040F048813846B9F1000F40F0EB8018F014
:1049D000E1FE2B6893F8542093078AD018F0DAFE92
:1049E000059B002B85D02868A36800F14201A27CBA
:1049F00090F8410022F0B6F817B9002800F06E8157
:104A0000734A92F900307F2B00F092810293214685
:104A1000286890F8864000F14203CDF800807C3091
:104A200001947F241470012203F050FA032061E7FF
:104A3000664D286890F854305F071BD590F88D308C
:104A4000002B5DD0636890F85B201978914200F0EC
:104A5000DC8090F85630012B00F0B38090F888305D
:104A6000082B04D090F885209A4200F0AA8018F014
:104A700091FE286890F88C30002B46D190F88D304C
:104A8000002B7FF436AF32E790F85430990769D5A0
:104A90004F4A92F900307F2B00F04A810293214661
:104AA00090F886307F240193FF23009300F14203A6
:104AB00014707C30062203F009FA2B6800220920CA
:104AC00083F8A82016E78268527902F0C002402AD3
:104AD0007FF445AF44E791F885804FE740460DF0FD
:104AE00077FF002818BF8346002F40F0E780296831
:104AF00091F8418091F85420C44602F0040045E743
:104B000090F88C30002B3FF4F2AE90F854309E07B2
:104B100060D4D8077FF5EDAE590700F102812C4B28
:104B200093F900207F2A00F003817F200292FF2664
:104B3000002218702146286890F88630CDE900637D
:104B400000F142037C3003F0C1F92B68032093F895
:104B50008D20002A7FF4CEAE93F88C30002B7FF4AA
:104B6000C9AEC4E6DA077FF5C2AE5B0700F1D680B6
:104B7000174B93F900207F2A00F0DA802868FF2580
:104B800002927F2290F88610CDE900511A702146DA
:104B900000F1420306227C3003F098F90320A9E6D5
:104BA000012010E72B6893F85630012B06D0002B1C
:104BB0007FF40DAFBAF1000F3FF409AF00283FF4C6
:104BC00006AF0A2007B0BDE8F08F00BF3C0C002103
:104BD00010000021574A92F900307F2B00F0A88086
:104BE0000293214690F886307F240193FF2300939F
:104BF00000F1420314707C30002203F067F92B6847
:104C00000122092083F8A820A1E7597890F85C20B8
:104C100091427FF41EAF997890F85D2091427FF425
:104C200018AFD97890F85E2091427FF412AF1979CD
:104C300090F85F2091427FF40CAF5A7990F8603081
:104C40009A427FF406AF627C90F85A309A427FF421
:104C500000AFB6E742316046A368A27C21F082FF34
:104C6000B1E692F801E091F85C0086457FF497AEDA
:104C700092F802E091F85D0086457FF490AE92F8DC
:104C800003E091F85E0086457FF489AE92F804E077
:104C900091F85F0086457FF482AE507991F86020EC
:104CA00090427FF47CAE94F811A091F85A20AAEBC0
:104CB0000202D2F1000A4AEB020A72E6A1684046FB
:104CC0000EF090F82968074691F841C091F85420F9
:104CD00050B34CF0020802F0040057E6286890F840
:104CE0005530023B012B3FF604AE002E3FF401AEDF
:104CF000104B93F900207F2A1AD00292FE2590F8DB
:104D000086107F22CDE900511A70214600F142033E
:104D100001227C3003F0DAF80320EBE518F03AFDCD
:104D200026E718F037FDFAE6E04602F004002DE62B
:104D3000FFF772FD1000002130B5184C85B094F9D2
:104D400000307F2B27D00A467F21217014490C6840
:104D500094F87010032916D094F8701006290CBF2F
:104D600003210121CDE9023194F88650014604F176
:104D70004203019594F8B9000090002002F032FF40
:104D800018B905B030BD0021ECE7002005B0BDE842
:104D9000304003F02DB8FFF73FFD00BF10000021A9
:104DA0003C0C00210F4A136810B593F870100229CB
:104DB0000ED993F8701008290FD893F870109268E4
:104DC000094B92680B44BDE8104052F82330184755
:104DD00041F291413220FBF783FE41F292413220B1
:104DE000FBF77EFE3C0C0021FDFFFF3F38B51C4D5C
:104DF0002B6893F87020022A2DD8027C044683F891
:104E000084201A44C168596792F8BD2083F8B920FC
:104E10004268C3F88020037A022B0ED018F040F8C5
:104E200018F0B4FE17F090FC0E4818F0B1FD0E48D3
:104E300018F0A8FD0D4818F045F9637C03B938BD9A
:104E40002868643021F084FE2B68DB6E002BF6D0DE
:104E500001221A6038BD40F6AC013220FBF740FE5B
:104E60003C0C00215C01002155555500D6BE898EB1
:104E700038B505460C460DF01DFB420704D4A37857
:104E800003F0E003402B0DD00DF014FB830704D496
:104E9000A37803F0E003202B04D0237803F03F0332
:104EA000242B01D9002038BD17F00CFF94F90030F5
:104EB00094F802C0002B62780CF01F03ACBF1E21D7
:104EC0004FF4967142EA032301FB03F31A1AB2F579
:104ED000877FE7D39842E5D8054A2946238810689A
:104EE000A0F8BA3080F8BCC0BDE8384004F0DABAA7
:104EF0003C0C002170B5334E84B0336893F88C506D
:104F00007DB30A4693F8A810044631B90178002908
:104F10000CBF0121022183F8A81093F87010062914
:104F2000C8B241D0072814BF01250225264991F9AE
:104F300000007F2843D04233CDE9020593F84400B6
:104F4000019093F8770000907F20087021460020A0
:104F500002F048FE40B9022D28D00020054602F09C
:104F600071FF284604B070BD6378DB061ED5A169C9
:104F70000220FFF77DFF05460028EED033680022AF
:104F800083F894206169C1B14A780978100902F068
:104F90000F0241EA0222A3F8962083F8950018F048
:104FA000F9FB284604B070BD0325BFE70020054685
:104FB00002F01EFF284604B070BDFF20EDE7FFF7AA
:104FC0002BFC00BF3C0C00211000002110B5044652
:104FD0008AB00EF069F8194A2378107003F00F03B5
:104FE000072B02D001200AB010BD2046694603F00D
:104FF0005DF9684603F048FA9DF80030002BF1D1C6
:105000009DF80130DB07EDD50D4C019922689DF824
:10501000110002F1980392F89E2021F0A3FD0028D0
:10502000E0D020680121903021F0CBF9FF216846C3
:10503000FFF760FF0028D5D00220D4E71000002140
:105040003C0C00212DE9F04104468AB00EF02CF80A
:105050004E4A2378107003F00F03082B04D001246C
:1050600020460AB0BDE8F0816946204603F0B4F856
:105070009DF80030002BF2D19DF8013003F00303BE
:10508000032BECD1424E356895F84D30002B46D0BD
:1050900095F8888095F88930002B43D1002705F1D9
:1050A000980395F89E2001999DF8110021F05AFD72
:1050B00008B9002FD3D0336895F8482093F8417091
:1050C00003F14205002A49D19DF8120002990128F6
:1050D00034D02B463A4621F045FD0028BFD0306839
:1050E0000121903021F06DF9356895F88930002B59
:1050F00043D121460120FFF7C9FA306890F85430B7
:1051000013F0030432D023F00403032180F8543059
:105110000C4604F0D5FB002002F03EFDA0E795F818
:105120008580B7E721F062FD0828B7D0A0EB08071B
:1051300085F88600B7FA87F77F09B0E74B7903F067
:10514000C003402BC5D12B463A4621F00BFD002869
:10515000C5D1029940460DF045FEBEE740460DF030
:105160007BFE0028B0D005460127ADE7022104F000
:10517000A7FB204602F010FD72E718F007FD17F0BC
:10518000E3FA002385F88930B3E700BF100000215F
:105190003C0C0021F0B5544F85B03B6893F8AF301C
:1051A000D3B1437804461B0716D50378A3B93B68EF
:1051B0000E46D3F8B000503024F0F5FA054658B941
:1051C0003A68D2F8B000837D53B9616991F801C0A3
:1051D000817AB1EB1C1F03D00025284605B0F0BD35
:1051E0006168002951D092F88520082A2ED01046F7
:1051F0000DF1070102AA0DF0DDFC064600286DD076
:105200003B68D3F8B000837D002B4AD0636902A9C4
:105210009DF807005A7812091EF0C5FC0028DCD062
:105220003B68BDF80C10D3F8B02002981182D06012
:105230009DF80710D3F8B020D1726369012135467B
:105240005B789174C3F303139372C6E7002B36D0D7
:105250006369607C5A7812091EF0A5FC0028BBD057
:10526000636939685A78D1F8B030C2F303129A7280
:1052700062681068D86092881A82D1F8B030627C77
:10528000DA72002201259A74A7E72EB3012EA3D16A
:10529000084602F043FF00289ED03B6893F88E50EA
:1052A0009BE700F10C0102AB9DF80720C07A21F0CA
:1052B00059FC002891D03B68D3F8B020BDE70B46DD
:1052C000627C00F10C01C07A21F04CFC002883D0F4
:1052D0003B68D3F8B030D4E701257EE740F69F71F4
:1052E0003220FBF7FDFB00BF3C0C00214378F0B5FA
:1052F0000446580687B071D4227803F01F0352EA9F
:1053000003236BD008466188052967D9227A636830
:10531000C2F3040253EA020560D0344D2D68002D1B
:105320005ED000285CD0A847002857D0304E01211D
:10533000227A3068C2F304026368D0F8B05069760C
:105340008DF814201A0A8DF8103005F11E008DF822
:1053500011201A0C1B0E04A98DF812208DF81330A1
:1053600021F04EFD628840F2E24303FB02F2637BD0
:10537000AA67D4F809202A60A27B43EA0223E27BD1
:1053800043EA0243227A6B60C2F34212238A85F811
:105390009220013B3268A5F8623092F8B930EB7583
:1053A000637825789A0603F01F0354BF1E224FF43A
:1053B000967245EA0323174602FB03F517F0C4FC77
:1053C0000B46218A024630680631D0F8B00089B217
:1053D000019750300095029114F08AFB07B0F0BDA0
:1053E000034E3168D1F8B050AAE700BF3C0100215C
:1053F0003C0C00212DE9F04FDFF8F8A09346847CA7
:1054000083B0DAF800200646012C894692F84870ED
:10541000984687F001073ED0002492F88950234631
:1054200005B392F85410490725D47068002839D084
:1054300092F88550082D26D0284601930DF0C8FA21
:10544000019B002818BF07461BB3DAF8003093F819
:105450008B3083B321F0D4FBDAF80030002205460C
:1054600083F88B208BF8005089F8004088F8007092
:1054700003B0BDE8F08F92F84D100029D5D092F816
:105480008850082DD8D123B1DAF8005095F88A1049
:10549000B9B10025E6E783685B7903F0C003402BD0
:1054A000BAD1BAE7019302F039FE019B0028EAD095
:1054B000DAF80020BCE72846B1680DF093FC0546F9
:1054C000D0E7B06801910DF08DFBDAF8003085F877
:1054D000890093F88950002DC4D021F087FB08285B
:1054E000019904D0DAF8003083F88500BAE70D4658
:1054F000B8E700BF3C0C00212DE9F0416A4C0022C6
:1055000005460F466368D4F8008018461A8018F0E4
:1055100055FA032D37D0052D4AD0606808F198015F
:1055200021F0BDFD98F89E10606821F0CCFD236845
:1055300093F8482003F1420693F8417052B193F872
:105540005420520718D493F885000DF085FC08B15B
:10555000064601273146606821F093FD39466068B0
:1055600021F0A4FD514BD3F80431002B40F096807C
:10557000052D12D0BDE8F08193F84D20002AE2D02D
:1055800093F88800E1E76068037823F00F0343F0A5
:10559000030303700C234370C0E7236831681A6D5E
:1055A000C2F80A10B188D1811B6D5F72BDE8F0812D
:1055B000D4E9000622233178737021F02F0141EAEB
:1055C000471141F00501317041F64B51036D1B6AE3
:1055D000C6F80F30026D936BF3741F0A1B0C3775FE
:1055E0007375D369B2F840708B42D16B3BD9DFF849
:1055F000C0C0ACFB01E1ACFB07C7890ABF0AF1756B
:10560000C1F30721B77531762949A1FB0313C3F311
:105610008F2373761B0AB376938CF3761B0A33774A
:10562000D38C73771B0AB377D2F8A730C6F81F3034
:1056300092F8AB3096F8242086F82330036D22F0E0
:105640001F0293F8B23003F01F03134386F824308F
:105650000CF056FF96F8243003F01F0343EA401382
:1056600086F8243059E7DFF84CC0ACFB01E1ACFB15
:1056700007C749097F09F175C1F30721B775A3F57C
:105680007A77317641F270718F42BDD80A49A1FB19
:1056900003139B0903F550639BB2BAE740F2F9513B
:1056A0003220FBF71DFA00BF3C0C002100800041B6
:1056B0005917B7D11F85EB51D34D621010B50DF0BE
:1056C000F3FC0B4A0B4B1468187094F889301BB923
:1056D00018F060F8032010BD18F058FA17F034F8ED
:1056E000002384F8893018F055F8032010BD00BF5E
:1056F0003C0C00211000002170B51F4C0E202368C7
:1057000093F8B91017F068FB236893F854309B079F
:1057100029D165685DB3284618F050F9236893F8DD
:10572000B930033B012B94BF2820002018F0E4F986
:105730002668681D96F8B9500DF082FA236886F83D
:10574000890093F8892052B1033D012D94BF55255E
:10575000502516F0DDFF284618F00CFA23680822C1
:1057600083F8702070BD02F0FFF90546D2E740F2E1
:10577000CA413220FBF7B4F93C0C0021F8B52E4C9D
:105780000546236893F8BC205F2A2CD851092B4A80
:10579000565C93F8BA0000F03F0017F09DFC2368B8
:1057A00093F9580017F088FCFDB1236832460120B8
:1057B000596F17F01DFE2368314693F89430022B81
:1057C0000CBF4020FF2017F007FB256895F85430E8
:1057D0009B0710D195F8A8306768A3B13846BDE89B
:1057E000F84018F0EBB80026D3E7324673210120C9
:1057F00017F0FEFDDFE702F0B7F92568074695F8D8
:10580000A830002BEAD1781D0DF01AFA236885F82C
:10581000890093F88930002BE0D0033E012E94BF1D
:105820005524502416F074FF204618F0A3F938468A
:10583000BDE8F84018F0C2B83C0C00211C4F030131
:10584000F0B52F4C83B00546236893F8BC205F2A3F
:1058500030D851092B4A575C5A6F7ABBD3F8800075
:1058600018F0E4F8266896F854309A0703D596F8AD
:105870009420022A34D05B072ED425BB284602F0A0
:105880004DFC014628460D4602F052FC024606F148
:10589000A9002946256895F8943095F8B9500095E7
:1058A00002F09AFD2368002283F8B97083F88A20F9
:1058B00003B0F0BD5A6F0027002ACFD00120FFF7B8
:1058C0005DFF2368CAE7002002F042FC014606F1B2
:1058D000A90002F077FDE5E796F89430012BCCD1D2
:1058E000FB1E012B05D93946002018F0F9F926686E
:1058F000C3E796F85930012B14BF39460321F3E76B
:105900003C0C00211C4F030107292DE9F04F0D46E7
:1059100087B004469046476803D12FB9002A00F0AB
:10592000C880002F00F09080637CDFF8C092012BCC
:105930005DD0072D40D0D9F8003093F885000828B5
:1059400040D00DF10F0104AA0DF034F9002800F049
:10595000488104A99DF80F0022F0ADFD0746D9F853
:10596000006096F8543013F0030076D1824613F0AD
:10597000040386F88CA040F0C88000219C4B86F878
:105980008D101B6833B141462046984786F88E003B
:10599000D9F80060636843B1627C86F89E201A687B
:1059A000C6F898209B88A6F89C30A06808B1072DFF
:1059B00039D007B0BDE8F08FD9F8006096F88500BF
:1059C0000828BED16168607C22F075FDD9F80020FE
:1059D000074661688532607C0DF022F80028BED150
:1059E000D9F80060A6F88C0086F88E00DDE77B7998
:1059F00003F0C003402B9CD1D9F80060072D96F826
:105A0000893000F0A480002BD8D021F0EFF8D9F82D
:105A1000003086F88500012293F8850083F88A20FB
:105A200083F886008BE7D6F88C3096F8851033F033
:105A30007F43BED00829BCD00DF0F2F8D9F8003071
:105A4000012283F88B20B4E7DFF8A091D9F8006039
:105A500096F8543013F0030088D0062D96F84CA029
:105A600070D9082D00F28C8096F88CB08BF0010173
:105A7000B8F1000F0CBF002101F0010100297FD116
:105A80006268002A5ED1B8F1000F40F0938062781E
:105A9000D00640F18F80012086F88C0058077FF5F2
:105AA0006DAF96F84D1096F88DA0D30674D50121F0
:105AB00064E7DFF83891D9F8002092F8543013F0F9
:105AC000030118BF012113F0040382F88C1005D0E4
:105AD0000378A3F10103B3FA83F35B0982F88D30F5
:105AE00092F8AF30002B3FF464AFD9F80030D3F810
:105AF000B000503023F057FE00287FF45AAFD9F899
:105B00000030012283F88E2053E7062D96F84D10C1
:105B100004D800297FF432AF39462FE796F88DA0DC
:105B2000082D3FF62AAFBAF1010F03D0B8F1000FEC
:105B30007FF423AF6368002BEBD1B8F1000F2BD1BA
:105B40006278B2E7BAF1000F08BFBA460FE7002B40
:105B50003FF434AFB8F1000F7FF455AF96F8B910A9
:105B600001297FF452AF38460DF03CF886F88900E1
:105B7000D9F8006096F88930002B3FF41FAF44E756
:105B8000002213F0040386F88C203FF4F6AE96F85A
:105B90004D1096F88DA0C3E70020019102F0BEFAE7
:105BA0001AEA000702D10199A9B10F46D9F800609D
:105BB0003946E3E6002002F0B1FA1BEA000B0ED1F1
:105BC000BAF1000F02D10CF025FF8246D9F800602F
:105BD00096F85430CBE60CF01DFF0746E6E7DA46B0
:105BE000F4E740F664313220FAF77AFF3C0C0021EA
:105BF000AC00002138B50F4D002002F023F92C68CD
:105C000094F8893063B900230121204684F870108C
:105C1000A4F8BA3084F8BC30BDE8384003F026BEA2
:105C200017F0B4FF16F090FD002384F889302C683B
:105C3000E9E700BF3C0C002138B50F4D0DF034FAF8
:105C40000E4B2C68187094F8893063B90023012139
:105C5000204684F87010A4F8BA3084F8BC30BDE84F
:105C6000384003F003BE17F091FF16F06DFD0023DE
:105C700084F889302C68E9E73C0C002110000021F1
:105C800038B5114D002002F0DDF80DF00DFA2C684A
:105C90000E4A94F88930107063B900230121204620
:105CA00084F87010A4F8BA3084F8BC30BDE83840ED
:105CB00003F0DCBD17F06AFF16F046FD002384F800
:105CC00089302C68E9E700BF3C0C0021100000215E
:105CD00038B5124D0DF0E8F9114A00212B6810700B
:105CE00003F1900020F06DFB2C6894F8893063B9C3
:105CF00000230121204684F87010A4F8BA3084F8FB
:105D0000BC30BDE8384003F0B1BD17F03FFF16F0DE
:105D10001BFD002384F889302C68E9E73C0C002146
:105D20001000002138B5144D002002F061F80DF08C
:105D3000BBF9024628680021104B90301A7020F001
:105D400040FB2C6894F8893063B900230121204678
:105D500084F87010A4F8BA3084F8BC30BDE838403C
:105D600003F084BD17F012FF16F0EEFC002384F858
:105D700089302C68E9E700BF3C0C002110000021AD
:105D800070B5154D0521286803F08CFB50B12B68C8
:105D9000012093F8B91017F0A3FF2B680B2283F8AA
:105DA000702070BD2E6896F8893063B900230121F8
:105DB000304686F87010A6F8BA3086F8BC30BDE8D8
:105DC000704003F053BD044617F0E0FE16F0BCFC33
:105DD00086F889402E68E9E73C0C002170B5164D25
:105DE00000210320FFF788FB0321286803F05AFBFA
:105DF00040B10121084617F073FF2B68092283F890
:105E0000702070BD2E6896F8893063B90023012197
:105E1000304686F87010A6F8BA3086F8BC30BDE877
:105E2000704003F023BD044617F0B0FE16F08CFC62
:105E300086F889402E68E9E73C0C002170B5244CB7
:105E4000236893F8BC205F2A29D85109214A565C5F
:105E50005A6F42BBD3F8800017F0E8FD256895F82B
:105E600054309A0703D595F89420022A20D05B0776
:105E700003D595F89430012B1AD0002002F068F970
:105E8000014605F1A90002F09DFA236800210622CF
:105E900083F8B96083F88A1083F8702070BD5A6F58
:105EA0000026002AD6D00120FFF768FC2368D1E73E
:105EB000F31E012B05D93146002017F011FF25688C
:105EC000DBE795F85930012B14BF31460321F3E786
:105ED0003C0C00211C4F0301F0B52B4C83B0236810
:105EE00093F8BC205F2A35D85109284A575C5A6F6D
:105EF000A2BBD3F8800017F099FD256895F85430BF
:105F00009A0703D595F89420022A2CD05B0703D575
:105F100095F89430012B26D0002002F0FFF80646B9
:105F2000002002F005F9024605F1A9002568314676
:105F300095F8943095F8B950009502F04DFA236821
:105F40000021052283F8B97083F88A1083F8702045
:105F500003B0F0BD5A6F0027002ACAD00120FFF716
:105F60000DFC2368C5E7FB1E012B05D9394600202F
:105F700017F0B6FE2568CFE795F85930012B14BF0E
:105F800039460321F3E700BF3C0C00211C4F0301FD
:105F900070B5234C236893F854309B072FD1606869
:105FA000C0B30C232068012180F8703003F088FC16
:105FB00000210520FFF7A0FA0621206803F072FAFD
:105FC000054658B12368012093F8B91017F088FEF0
:105FD000236801221B6D83F8A62070BD266896F801
:105FE00089307BB900230121304686F87010A6F86D
:105FF000BA3086F8BC30BDE8704003F037BC01F021
:10600000B3FDCDE717F0C2FD16F09EFB86F8895070
:106010002668E7E740F247513220FAF761FD00BFFA
:106020003C0C0021012970B515D1A0B91E4A136896
:1060300093F8701008292DD993F870100C292ED8D8
:1060400093F870109268194B52680B44BDE8704089
:1060500052F823301847144D002001F0F3FE2C684D
:1060600094F889306BB9002304F1BA02012120466B
:10607000A4F8BA3084F870109370BDE8704003F053
:10608000F5BB17F083FD16F05FFB002384F8893021
:106090002C68E8E741F261413220FAF721FD41F234
:1060A00062413220FAF71CFD3C0C0021F7FFFF3F54
:1060B00030B5244D83B02B68D86F01F03DFD00282A
:1060C0003BD004460A232868002180F8703003F092
:1060D000F7FB2A6823780520126D92F8A64004EA9F
:1060E000531404F001042146FFF706FA042128683E
:1060F00003F0D8F928B12B681B6D83F8A64003B0D4
:1061000030BD2C6894F889306BB9002301212046FA
:1061100084F87010A4F8BA3084F8BC3003B0BDE83D
:10612000304003F0A3BB019017F030FD16F00CFBDC
:10613000019884F889002C68E7E740F22251322068
:10614000FAF7CEFC3C0C0021F0B5684C83B000207F
:1061500001F022FD256801F0B3FC2368E867D86FE1
:10616000002800F0BD8001F0E7FC0546002800F0A3
:10617000B280236893F8B430002B67D1206890F880
:10618000843090F87020034493F8BD7080F8B970A3
:106190001AB190F87030012B76D190F88720544BCB
:1061A0001344187916F098FF236893F88420134459
:1061B00093F8BD60022E65D041D9F31E012B40D863
:1061C00001F078FC314616F007FE284617F0F6FB82
:1061D0003146012016F08EFF012F46D0681D25683C
:1061E0000CF02EFD236885F8890093F8892052B1C0
:1061F000033F012F94BF5525502516F089FA2846F4
:1062000017F0B8FC236893F8542012F0060F06D05C
:1062100093F884201A4492F8BD1001293AD0002244
:1062200040F608000321A3F88500C3F88A2083F80C
:106230008E2083F8A82083F8701003B0F0BD012EE3
:10624000BED040F2B5713220FAF74AFC236893F8C9
:10625000542093F8B500196D0243C3F8341183F844
:106260005420002283F8B42088E7E81C25680CF04D
:10627000E7FC236885F8890093F88920002AC2D0BA
:106280004025BAE70D209DE7002103F00BF930B15E
:10629000206882E7002017F023FD2368BFE7256808
:1062A00095F889306BB900230121284685F87010D4
:1062B000A5F8BA3085F8BC3003B0BDE8F04003F073
:1062C000D5BA019017F062FC16F03EFA019885F8F5
:1062D00089002568E7E740F206413220FAF700FC22
:1062E00040F204413220FAF7FBFB00BF3C0C0021D6
:1062F0001C4F030108B50CF0D7FE044B187017F0C3
:1063000049FABDE80840FFF71FBF00BF1000002199
:1063100010B50CF0C9FE0D4A0D4B1468187094F8B6
:1063200089302BB917F036FABDE81040FFF70CBFE3
:1063300017F02CFC16F008FA002384F8893017F0C7
:1063400029FABDE81040FFF7FFBE00BF3C0C00215A
:106350001000002138B5194C256895F889302BBB01
:1063600000206168FEF792F9206890F8543013F02D
:1063700003050DD023F00403032180F8543003F00B
:106380009FFA002001F008FCBDE83840FFF7DCBEB2
:10639000022103F095FA284601F0FEFB2368A3F8DA
:1063A000BA5083F8BC5083F8705038BD17F0EEFB3C
:1063B00016F0CAF9002385F88930D1E73C0C00219A
:1063C00038B50446FEF712FD237A032B63D0012B68
:1063D0006AD051D84E4C4F49226892F8873092F8D3
:1063E0004B000133A1FB035C0CF4FF7505EB5C056E
:1063F0005B1B40FA03FCDDB21CF0010F16D1013328
:10640000A1FB035C2CF0010505EB5C055B1B40FA6E
:1064100003FCDDB21CF0010F08D10133A1FB0351D5
:1064200021F0010505EB51015B1ADDB282F88750BE
:1064300092F9580016F040FE2368002283F8A82045
:10644000FFF782FE256895F84830A3B16FF000434E
:10645000D5E928129A4208BFB1F1FF3F0BD019F0DD
:106460009BF8D5E92823904271EB030303D3012065
:106470000CF084FC18BB38BD023B012BFBD8244C2C
:10648000236893F8A80090B9FFF7DAF9236805228A
:1064900083F8702038BD1E4B1B68586F90BBFFF708
:1064A0006DF9237A012B94D1194C2268C0E70120A1
:1064B000FFF7C6F92368062283F8702038BD2568E7
:1064C0000CF072FB044619F067F86301E20E1B1B27
:1064D00062F10002520242EAD3525B021B1942F1FE
:1064E000000C9A014FEA8C1ED21A4EEA936E6EEBA4
:1064F0000C0C13194CF100021B1842EB0101C5E909
:10650000283138BD40F6F3013220FAF7E9FA00BF2E
:106510003C0C0021ABAAAAAA2DE9F041A54E86B0F9
:10652000336893F8572052B193F88C2005466AB12E
:106530002C78012C15D0022C6CD0002C59D00324BF
:1065400017F028F9204606B0BDE8F08193F88D20B9
:10655000002AEDD193F88E30002BF0D02C78012C4E
:10656000E9D117F017F9346894F8B930022B6B7839
:1065700000F0838003F01803182B46D194F85430B0
:10658000580700F1F780990717D08B4A92F900302D
:106590007F2B00F07081002002937F21039094F8FC
:1065A0008630019394F8B930009304F142031170DE
:1065B000FF22294601F016FB38B3A9690120FEF736
:1065C00057FC10B30123326882F894306B69002BBA
:1065D00000F0E38059780224C1F3031182F895108A
:1065E00059781B7801F00F0143EA0123A2F8963095
:1065F000A8E717F0CFF8336893F85420970704D032
:10660000D3F88C3013F0FF1F3DD10324204606B091
:10661000BDE8F08117F0BEF8336893F85420920774
:10662000F3D06A7802F01802182AEED1624A92F981
:1066300000107F2900F01F81002002914233039057
:1066400093F84410019193F8771000917F21117015
:10665000FF22294601F0C6FA0028D6D0A9690120F8
:10666000FEF706FC0028D0D0326882F894406B69AF
:10667000002B00F0F7805978AEE703F01903192BCF
:106680003FF47CAFC1E76B7813F0100FC3F3001732
:1066900014BF0822012232EA0303B6D1AB688DF899
:1066A00015408DF816408DF81740002B00F0A4809F
:1066B0000DF117030DF116010DF115022846FEF735
:1066C00099FE31689DF8153091F84180002B40F01B
:1066D000BF804231AB68AA7C404620F043FA78B9CB
:1066E000336893F85530023B012B8ED89DF8163055
:1066F000002B8AD09DF81530002B86D14FF0FE0874
:10670000002F7CD02C4991F900307F2B00F0B38012
:106710000293002433684246039493F88600423380
:10672000019093F8770000907F200870294620465A
:1067300001F058FA00283FF468AFA9690120FEF77C
:1067400097FB00283FF461AF336883F894406A698F
:10675000002A00F08B8051780224C1F3031183F8E2
:1067600095105178127801F00F0142EA0122A3F846
:106770009620E7E66B680BBBAB68002B7FF445AF58
:10678000AB699B7813F0E0030CD194F84930002BEF
:106790003FF43BAF94F85430F5E6FF23022482F82F
:1067A0009530CFE6402BF5D194F84A30002BF1D14B
:1067B0002BE700BF3C0C00211000002104F15B031B
:1067C00094F85A2004F1980194F89E0020F0CAF938
:1067D000346894F88530082B03D094F888209A42C6
:1067E00039D094F85630012BC6D0002B7FF40DAF72
:1067F00000283FF40AAFBFE74FF0FF0880E71F4AC9
:1068000092F900307F2B36D030687F21117090F8DC
:106810007020032A05D090F87020062A0CBF0324AC
:10682000012442462946CDE9023490F8864000F121
:106830004203019490F8B9000090002001F0D2F9D1
:1068400000283FF4E2AE0020032401F0D1FA79E6FB
:1068500048F0020854E794F85630012B8CD0002BF6
:106860008AD0D2E6FF2382F895306BE6FF2202241D
:1068700083F8952066E6FDF7CFFF00BF10000021EA
:1068800030B505468BB00CF00FFC354B2C7802462A
:106890006946284604F00F041A7001F007FD072C22
:1068A00037D0304D002221466846FFF72DF82B687F
:1068B00093F8B930012B0CD0023B022B4AD80324A9
:1068C00016F068FF2D6895F889308BB920460BB01B
:1068D00030BD062C02D015D8022CF0D821466846CF
:1068E000FDF7F2FF2D68044695F88930002BEDD0B6
:1068F00017F04CF915F028FF0023204685F8893061
:106900000BB030BD072CDAD16846FFF705FE044610
:10691000D8E7144D68462B6893F8B91001F002FDD2
:10692000002221466846FEF7EFFF2B6893F8B93046
:10693000022B07D00BD8012B0CD16846FFF7ECFDDA
:106940000446BFE79DF80030012BB8D1DCE7033BDC
:10695000012BD9D941F2F8113220FAF7C1F800BF62
:10696000100000213C0C00212DE9F04790B0A64C0E
:106970000D4606A901F09AFC206806A9A93001F08D
:1069800055FD23689DF8181093F89420914205D185
:10699000032D1AD09DF8192011076BD40020012671
:1069A00001F050FA256895F889301BB9304610B0CF
:1069B000BDE8F08717F0EAF815F0C6FE0023304670
:1069C00085F8893010B0BDE8F08793F89520FF2A4C
:1069D000E0D12A4606A80721FEF796FF2568D5F8DC
:1069E0008C0030F07F40DAD00023089F8DF81530FE
:1069F0008DF816308DF81730002F52D00DF1170397
:106A00000DF115020DF1160106A8FEF7F3FC25683D
:106A10009DF8159095F84180B9F1000F01D048F02C
:106A200002089DF816A09DF817709DF81860012EB9
:106A30003CD0022E2FD0002EB0D195F854309807BC
:106A40002DD09DF81930990700F19F804FF0FF0875
:106A500095F88E3033B16D4B1B681BB10D9808B1A2
:106A60000F999847414606A8FEF744FA2568B0B149
:106A7000022698E70B9993F895004A78B0EB121F1D
:106A80008CD1097802F00F02B3F8963041EA022265
:106A90009A4283D19DE795F854309A074CD101264C
:106AA00081E7BA46B9464FF0FF08BEE79DF81930B6
:106AB00095F8A91003F00902092A05D000293FF42E
:106AC00072AF1A077FF56FAF95F854305B0703D5A7
:106AD00095F88D30002B76D195F88C30002B3FF453
:106AE00062AF95F854309F073FF45DAF9DF81930C1
:106AF00013F0020300F0F080B9F1000F40F088803D
:106B0000089B05F142019DF82A2095F8410020F0EC
:106B100029F800287CD1256895F85530023B012BD7
:106B20003FF641AFBAF1000F3FF43DAFFE2106A89A
:106B3000FEF702F9256836E795F88C20002AAED0DA
:106B40009DF8192002F009010929A8D113F00206C5
:106B500000F0888012F0020600F00581B9F1000F04
:106B600040F05D81002F40F04E81256895F855304A
:106B7000023B012B93D8BAF1000F90D0FE2106A85A
:106B8000FEF7DAF8012625680DE7B9F1000F7FF46A
:106B90005FAF05F1420195F84100089B9DF82A205E
:106BA0001FF0E0FF256800287FF452AF95F85530BC
:106BB000023B012B3FF673AFBAF1000F3FF46FAF0A
:106BC0004FF0FE0844E7002900F0AB80089B8BB132
:106BD000B9F1000F0ED1002F3FF47EAF05F1420155
:106BE00095F841009DF82A201FF0BCFF2568002879
:106BF0003FF472AF05F190001FF005FC25680028F6
:106C00003FF46AAF0C26CEE63C0C00214001002187
:106C10009C4991F900207F2A00F0318123687F2070
:106C2000087093F87010032900F09B8093F870109F
:106C300006290CBF032101214233CDE9022193F83B
:106C40004400424606A9019093F877000090002086
:106C500000F0C8FF00283FF4A5AE002001F0C8F8FE
:106C60002568A0E612F0020200F0A480B9F1000F3E
:106C70000BD1089B05F142019DF82A2095F84100AF
:106C80001FF070FF00283FF470AF7E4991F900209B
:106C90007F2A00F0F48023687F20087093F870103A
:106CA000032905D093F8701006290CBF032601268E
:106CB00006A94233CDE9022693F8440042460190EA
:106CC00093F877000090002000F08CFF002840F03F
:106CD00094802568012666E66A4991F900207F2A9A
:106CE00000F0CD807F20087095F87010032905D042
:106CF00095F87030062B0CBF0323012306A9002052
:106D0000CDE9022395F88630019305F1420395F809
:106D1000B9200092FF2200F065FF00283FF442AE48
:106D20009BE705F15B0395F85A2005F1980195F86A
:106D30009E001FF017FF256895F88530082B04D0BA
:106D400095F888209A4200F0918095F85630012BF2
:106D50003FF43CAF002B7FF4BFAE00283FF4BCAE45
:106D600034E7002168E7474B93F900507F2D00F08E
:106D700086807F22314603201A70FEF7BDFB236810
:106D8000304601260295424606A90396423393F8FF
:106D90004450019593F87750009500F023FF0028A8
:106DA0003FF400AE206890301FF02DFB28B325681B
:106DB0000B26F8E5334991F900307F2B5FD07F2017
:106DC000087095F87010032905D095F87020062AF0
:106DD0000CBF0322012206A90020CDE9023295F85A
:106DE000862005F14203019295F8B9200092FF2216
:106DF00000F0F8FE00283FF46CAF0020012600F000
:106E0000F7FF2568CFE5089B05F142019DF82A2090
:106E100095F841001FF0A6FE00283FF4A6AE194BDE
:106E200093F900507F2D2AD07F22002103200126D4
:106E30001A70FEF761FB23684246029506A9039685
:106E4000423393F84400019093F8770000900020BB
:106E500000F0C8FE00283FF4A5AD206890301FF078
:106E6000D2FA256800283FF49EADA1E795F8563088
:106E7000012B3FF4ABAE002B3FF4A8AE2CE6FDF7A0
:106E8000CBFC00BF1000002110B504460CF00CF93B
:106E9000084A2378107003F00F03072B05D1204612
:106EA0000321BDE81040FFF75FBD002000F0CAFFDE
:106EB000012010BD1000002110B504460CF0F4F8BC
:106EC000084A2378107003F00F03072B05D12046E2
:106ED0000121BDE81040FFF747BD002000F0B2FFE0
:106EE000012010BD1000002190F83E00003818BFAE
:106EF00001207047007A003818BF0120704700BF9A
:106F0000036D10B583B10222FF21044642721A8834
:106F10004FF6FF7380F8271003850649428120F061
:106F2000CBFD0023236510BD40F229313220F9F753
:106F3000D7FD00BF9D4300012DE9F843012107461D
:106F40000020FAF777FE012104460846FAF772FEA0
:106F50000546204602F0C6F902E094F870301BB1F5
:106F600094F87030012BF8D1002D42D0284602F061
:106F7000B9F902E095F870301BB195F87030012B2B
:106F8000F8D100F089FD002140F201194FF0070807
:106F90000E463F2220461BF0A3FC04F16400A4F837
:106FA0004C9084F8546084F8876084F8587084F8B2
:106FB0004B801FF0C6FD3F2231462846E6661BF097
:106FC0008FFC05F16400A5F84C9085F8546085F8B5
:106FD000876085F8587085F84B801FF0B2FDEE662B
:106FE000002384F8AF30C4F8B03084F8B430BDE882
:106FF000F88300F051FD3F22294620461BF070FC2B
:1070000040F20112072304F1640084F85450A4F8FC
:107010004C2084F8875084F8587084F84B301FF067
:1070200090FDE566DCE700BFF8B503461C4E0F4651
:10703000002001217360FAF7BFFD38B34FF4A0724E
:10704000002104461BF04CFC01210846FAF7B4FD70
:10705000054688B14FF4A07200211BF041FCB368D3
:10706000CBB13846FFF768FF204602F01DF92846ED
:10707000BDE8F84002F018B9B36863B13846FFF7CD
:107080005BFF2046BDE8F84002F00EB940F649012A
:107090003220F9F725FD40F653013220F9F720FDA3
:1070A0003C0C0021014B024A9A6070473C0C0021C5
:1070B0004401002103490448044B054A08601A6052
:1070C000704700BF40010021ED520001AC000021DB
:1070D00095510001036823B1054A916813600B685C
:1070E000184740F61D11322010B5F9F7F9FC00BF22
:1070F0003C0C002138B50F4D002000F0A3FE2C6899
:1071000094F8893063B900230121204684F8701077
:10711000A4F8BA3084F8BC30BDE8384002F0A6BB11
:1071200016F034FD15F010FB002384F889302C682C
:10713000E9E700BF3C0C002180F84B10704700BF0E
:1071400011F001031FD04FF0010C0222634680F8BA
:10715000BDC011F0020F0ED000EB030C490700B5C3
:107160004FF0020E8CF8BDE003D51044042380F8E4
:10717000BD305DF804FB4A0704D51844042380F8A9
:10718000BD30704770470122E3E700BF80F8571019
:10719000704700BF38B5054690F84000A0F1020CDA
:1071A000BCF1010F98BF00290CBF0124002408D0B6
:1071B00010F0FD0FBDE8384014BF012000200BF097
:1071C000ABBA12F0FD0F194614BF012000201FF0CA
:1071D00003FD082801D0204638BD95F84000E7E7B8
:1071E00090F8403013F0FD0F14BF012000200BF089
:1071F00093BA00BF90F8B420F2B908B5034602F084
:10720000FF0093F85420022A07D0012A08BF04295E
:107210000CBF0120002002D008BD0429FCD1D3F806
:1072200034215AB91A6D72B1042283F8B520FF22B5
:1072300083F8B420012008BD0020704740F69B1160
:107240003220F9F74DFC40F69C113220F9F748FC4A
:1072500080F84010704700BF38B590F840300446C1
:1072600000F1420113F0FD0F14BF0120002084F84B
:1072700041000BF039FA94F84030023BDBB2012BAD
:1072800094BF0123002384F8483000D938BD0BF0A7
:107290008BFC054618F080F96B01EA0E5B1B62F16E
:1072A0000002520242EAD3525B025B1942F1000C27
:1072B0009A014FEA8C1ED21A4EEA936E6EEB0C0CBA
:1072C00053194CF100021B184FF0000042EB010172
:1072D000C4E928310BF052FD0028D7D140F6B61191
:1072E0003220F9F7FDFB00BFB1F1000C4FF00801AF
:1072F00010B504460CBF0120002084F856C084F865
:107300004D0084F8881009D112F0FD0F194614BF02
:10731000012000201FF060FC84F8880010BD00BF31
:1073200008B5A2B180F85A10D2F800C0036DC0F8B9
:107330005BC090F841109288A0F85F205972D0F895
:107340004220C3F80A20B0F84620DA8108BD40F692
:10735000D4113220F9F7C4FB80F84910704700BF00
:1073600080F84A10704700BF2DE9F041D0F8E05096
:107370009DF81840954203D190F840208A4202D0EF
:107380000020BDE8F08114F0020190F83A5126D0B7
:107390000026B4463146324612E04EEA010100EBC7
:1073A000820253F82C700CF1010E0136D2F8E42061
:1073B0005FFA8EFC7632BA42E2D1F2B295422CD319
:1073C00000EB020E0CF101089EF8BDE0AEF10307E0
:1073D000012FE2D841F004015FFA88FCDFE78E4616
:1073E0000A4601E0954218D386180EF1010E96F870
:1073F000BD60F71E012F53F8227088BF314300EBA8
:10740000820698BF41F004015FFA8EF2D6F8E4607C
:1074100006F1760C6745E5D0B2E704F00500401AA6
:10742000B0FA80F04009BDE8F08100BF90F8543018
:10743000024659070DD413F0030000D1704792F8AB
:10744000550000F0FD00A0F10100B0FA80F0400905
:10745000704790F85600A0F10100B0FA80F04009A2
:10746000704700BF012910B504460BD094F8543082
:107470009B0716D10023A4F8BA3084F8BC3084F8F6
:10748000703010BD90F88930002BEFD016F07EFBE5
:1074900015F05AF9002384F8893094F854309B078A
:1074A000E8D0002000F0CEFCE4E700BF90301EF0F2
:1074B000B3BF00BF0149363020F0FEBA8943000156
:1074C00010B5012104460020FAF7B4FB78B36378C5
:1074D00080F85430227812F0010323D1012112F0F8
:1074E000020F05D000EB030C0B4602218CF8BD10F7
:1074F000520703D50344042283F8BD20A37880F803
:107500004030E37813F0FD0F80F855300CBF0123B5
:10751000002380F84C30237980F84B30637980F871
:10752000573010BD0123022180F8BD30D7E740F667
:107530006B213220F9F7D4FA10B590F87030022B95
:107540000BD10446002000F07DFC0023A4F8BA30E3
:1075500084F8BC3084F8703010BD40F69921322098
:10756000F9F7BEFA08B5002364301A4619460AF046
:10757000FFFF00280CBF0C20002008BD10B5012122
:1075800004460020FAF756FB68B1034690F8AF2096
:1075900002F0FF002AB9C3F8B040FF2283F8AF2001
:1075A00010BD0C2010BD40F6CE213220F9F798FA1C
:1075B00008B501210020FAF73DFB18B1002380F83F
:1075C000AF3008BD40F6DF213220F9F789FA00BF5D
:1075D00038B501210020FAF72DFBF0B1044690F8F0
:1075E000AF30BBB1002380F8AF30D0F8B00001213C
:1075F000503022F093F9D4F8B03093F8443003F0CF
:10760000FF053BB9D4F8B00012F038FF2846C4F8A3
:10761000B05038BD0C25284638BD40F6E621322052
:10762000F9F75EFA08B501210020FAF703FB28B14B
:1076300090F8AF00003818BF012008BD40F60931AE
:107640003220F9F74DFA00BF2DE9F04304468DB022
:107650000D4600200121FAF7EDFA002800F0F8812C
:107660000646C03001F05AFE002847D096F8543044
:10767000042B43D0666A002E00F03781B34F07F128
:107680000C039E4262D007F108039E425ED006F1D1
:1076900037090AF0E7FE074602A9484600F006FE51
:1076A000002F40F02E81E37A05F11C00DB0600F18B
:1076B0002E81002E00F0B5809DF80830022B00F0DE
:1076C000B080014694F82E30E52248461FF091FE26
:1076D00094F82E3080464846434484F82E301FF0FC
:1076E00080FE94F82E30181AB0FA80F04009002F6E
:1076F00032D108F11803954FDBB29AE03046FFF71C
:10770000F3FB0028B6D1914F07F1080507F10C06ED
:107710000023626A002A00F00681616A0A68A942B1
:1077200062620B704B708B70CB70F2D0B142F0D0B4
:1077300038681CF038F9EFF3108272B63B790133E8
:10774000DBB23B71002AE3D162B6E1E70AF08AFEC0
:1077500000286AD04FF00008E37AD90640F1818111
:107760005A0703D5E37EFE2B00F04A81032108F17E
:107770000A032970A27A02FB03F3EA7002336B70EA
:10778000637B6B71D4F80E30C5F80630638A85F8D8
:107790000C80A8446B81237E88F80D30E37A13F0C7
:1077A000080700F00C81DFF8A8810423674F4645E5
:1077B0002B715FD12B79022262F34613626A2B711F
:1077C0006AB1EFF3108272B6636A19686162002AC7
:1077D00000F0A78000221A705A709A70DA70A4F133
:1077E000080138681CF0DFF8EFF3108272B63B79BD
:1077F0000133DBB23B71002A00F0918002264FF08A
:1078000004088DF804808DF805609DF804200020A0
:107810009DF8053062F3070063F30F200DB0BDE85B
:10782000F083002F40F01D81484F18234FF00008CF
:10783000012004222A70A27A02FB03F3EA700233C9
:107840006B70D4F80B20D4F80F30D4F813C0D4F8F0
:1078500017106A60AB60C5F80CC02961D4F81B2012
:10786000D4F81F306A61AB6185F81B80DFF8E080D7
:1078700046459FD008F104094E456BD0002E00F01C
:10788000908050B3636A63B1EFF3108272B6636A9B
:107890001968616202B962B600221A705A709A7051
:1078A000DA70314638681CF07EF8EFF3108272B659
:1078B0003B790133DBB23B7102B962B6636A0022E5
:1078C000434584F82E203FF475AF4B4500F0B4805B
:1078D0009DF80830022B00F088802B7901264FF0AC
:1078E000040866F346132B718BE704F12F090AF0A5
:1078F000B9FD074602A9484600F0D8FC002F3FF426
:10790000D2AEE37A05F10D00DB067FF5D2AE9DF82D
:107910001880059942461AF06DFF0120E7E662B62D
:107920006CE762B656E7A4F1080138681CF03BF832
:10793000EFF3108272B63B790133DBB23B7102B9CF
:1079400062B64FF40073ADF804305EE7480C0021D6
:10795000500C0021636A63B1EFF3108272B6636A60
:107960001968616202B962B600221A705A709A7080
:10797000DA70637D93BB2A794FF0040863F34612F3
:107980002A71A4F1080138681CF00DF8EFF3108299
:1079900072B63B790133DBB23B71EAB962B60226BB
:1079A0002FE794F80B8018F010083FF42AAF2B79DA
:1079B000A4F10801386866F346132B7112E703F04F
:1079C0000302032A19D05B070BD4022A3DD0002AF8
:1079D00043D1264F297149E7022612E74FF00008EC
:1079E000CFE70123214F2B7140E72B7901264FF080
:1079F000040823F068032B7103E72F711B4F35E751
:107A000011221A4F2A70A27AEA70120102326A70A9
:107A100001222A71627B6A71D4F80E20C5F8062013
:107A2000628A2B736A81E369C5F80D30238CA5F84F
:107A30001130237EEB7419E72B7962F34613626AE7
:107A40002B71002A7FF4BDAEC9E6084F2A710DE7FD
:107A50004FF4E1713320F9F743F89D213320F9F712
:107A60003FF856213320F9F73BF800BF480C0021BE
:107A7000303270B5054692B20C461E461BF05BFFD5
:107A800035B1044A0023156014745674147153619F
:107A900070BD00BF480C002138B5054C002520689A
:107AA000A5611BF06AFF237C6561237138BD00BFAF
:107AB000480C0021014B587C704700BF480C002146
:107AC00038B51C4D6C6954BB28681BF05CFF03463D
:107AD000686148B32A7908301C63013A9C86A86122
:107AE000D2B2C3F81140C3F815402A71C3F8194047
:107AF000C3F81D40C3F82140C3F82540DC62A3F859
:107B000029401C740125DA7CFF2147F6FF7465F3D8
:107B10004612DC83597583F82310DA7438BD4FF4AC
:107B2000A4713320F8F7DCFF40F24B113320F8F753
:107B3000D7FF00BF480C002108B50A4B5B6933B181
:107B400003F10802904207D103F1370008BD40F26B
:107B50005B113320F8F7C4FF40F25D113320F8F7D2
:107B6000BFFF00BF480C002110B50A4C606908B186
:107B7000373010BD20681BF006FF606128B1237903
:107B80003730013BDBB2237110BD4FF4B4713320A9
:107B9000F8F7A6FF480C002110B5114C6169D1B16E
:107BA00020681BF000FF2379D4E905210133083256
:107BB000DBB2914223714FF000030ED0636149B1F3
:107BC000083920681BF0EFFE237900220133A261FF
:107BD000DBB2237110BDA169F1E7C4E9053310BD23
:107BE000480C00212DE9F0477D4E17460D469DF8C3
:107BF00020C032799DF824009DF928109DF82C9022
:107C0000002A00F0AB8098467369002B00F0D0800A
:107C1000B469002C00F0D080EA684AB195F810E011
:107C2000A28D724440F2726E724500F3BA80A28552
:107C300001220CF1FF3C21765FFA8CFCA272B9F1B3
:107C4000000F00F08380BCF1030F00F2BA80654A98
:107C500012F80C20627583F811906A691AB1527893
:107C6000C2F30312A275EA6912B15288A4F819206E
:107C700095F800A0E17AAAF10102D5F808C0B2FA9D
:107C800082F2520962F30001BAFA8AF2C1F3400E9D
:107C90005209BAF1020F08BF4EF0010E6EF3410116
:107CA00002EA510262F3C301E172BCF1000F03D09A
:107CB000CAB242F00402E2722A6A12B192F90020BA
:107CC000E2756A6882B1082804F10E025BD004F103
:107CD0000D010AF06FFF00287DD0637B43F00203A3
:107CE00063737369D5F808C0BCF1000F0BD0BA1EDE
:107CF00004F11C01012A3ED9DCF80020E261BCF845
:107D000004208A80E776B9F1000F0FD000221A70A4
:107D10005A709A70DA70626A002A3FD0A26A1360C1
:107D2000A362314920461FF0D3FE7369AA6932B1BC
:107D30005178927802F01F0251EA022213D0002BF0
:107D400044D0002301207361BDE8F087BCF1030F2C
:107D500037D8244A12F80C2022757CE702F0FF0382
:107D60001846BDE8F087616AB260E9B1A16A1F4AAE
:107D70000A60A262E3E7D8F80020E261B8F80420C4
:107D80008A80E776BFE7697C617369680868C4F830
:107D90000E0089889180D5F808C0A5E76362A362C8
:107DA000BFE70020BDE8F087104A6262A262C6E722
:107DB00050213320F8F794FE4FF444713320F8F744
:107DC0008FFE40F20B310620F8F78AFE4FF4D17196
:107DD0003320F8F785FEBC213320F8F781FE00BF81
:107DE000480C0021244F030149760001500C00216A
:107DF00038B5124DAC69DCB1114920461FF068FE60
:107E00000023EB60EFF3108272B6636A4BB1A16A94
:107E100005F10C030B60A36202B962B60023AB61EB
:107E200038BD05F10C036362A362002AF6D1F4E7C2
:107E300040F273313320F8F753FE00BF480C0021A5
:107E40004976000138B51E4CA3691BB35A7D0AB3AD
:107E50000022A260EFF3108172B65A6AEAB1986A02
:107E600004F1080202609A62A9B1A56915B3154927
:107E700028461FF02DFE0023E360EFF3108272B658
:107E80006B6A8BB1A96A104B0B60AB6202B962B628
:107E90000023A36138BD62B6E7E704F108025A6225
:107EA0009A620029E1D1F6E7074B6B62AB62002AC8
:107EB000EED1ECE740F273313320F8F711FE00BF4A
:107EC000480C002149760001540C00212DE9F843AB
:107ED000524D0F46002604682979984606609DF8A1
:107EE00020909DF824009DF9283081B9A4F1080163
:107EF00028681BF058FD2B790133DBB22B7100236E
:107F00006A69AB61002A7FD06B61BDE8F88301210B
:107F1000C4F80960C4F80D60C4F81160C4F81560B5
:107F2000C4F81960C4F81D60A4F82160A172062A83
:107F300065D8DFE802F02A3138643D640400E27A53
:107F400022F0120242F01202E27223760123082884
:107F500004F10E02237547F6FF73E3822FD004F17C
:107F60000D010AF027FE002853D0637B43F0020383
:107F70006373E37A5B072DD4FF23E3760023237238
:107F8000274920461FF09BFDB9E7E27A22F0130251
:107F900042F01302E272D8E7E27A22F0150242F0D0
:107FA0001502E272D1E7E27A42F01002E272CCE707
:107FB000E27A22F01A0242F01A02E272C5E77B7CF2
:107FC00063737B681968C4F80E109B889380E37A0A
:107FD0005B07D1D5A9F1020304F11C02012B07D9DB
:107FE000BB681968E1619B88938084F81B90C5E7A2
:107FF000D8F80030E361B8F804309380F5E74FF427
:1080000075713320F8F76CFD4FF4D1713320F8F718
:1080100067FDBC213320F8F763FD00BF480C002149
:1080200049760001F8B53B4D8446002610462A7972
:108030000F46DCF800409DF91810CCF800607AB9C2
:10804000A4F1080128681BF0AEFC2B790133DBB2E8
:108050002B7100236A69AB61002A52D06B61F8BDB5
:10806000C4F8096008286289C4F81560217641F6D1
:10807000012122F4DF52C4F8116041EA032141F6E4
:10808000FF3322F01F02C4F80D6003EA0103C4F8B5
:108090001960C4F81D6043EA0203A4F8216004F1EA
:1080A0000E0263814FF00103237547F6FF73E382ED
:1080B00014D004F10D010AF07DFD38B3637B43F069
:1080C00002036373E37A5B0713D4FF23E376002391
:1080D0002372114920461FF0F2FCBAE77B7C6373E0
:1080E0007B681968C4F80E109B889380E37A5B075D
:1080F000EBD5BB68FF221968E1619B88E276238497
:10810000E5E74FF4D1713320F8F7EAFCBC213320C6
:10811000F8F7E6FC480C002149760001034B98690A
:1081200018B1407BFF3818BF01207047480C002170
:1081300008B5064B9B6923B1D87EFF3818BF0120D4
:1081400008BD40F234413320F8F7CAFC480C002146
:1081500008B5064B9B6923B1987DFF3818BF0120F5
:1081600008BD40F23F413320F8F7BAFC480C00212B
:1081700070B50C46164605461EF0A1FF034628467C
:1081800063741EF0A7FFA074062E13D8DFE806F074
:10819000041904120412040000230121EA1C617076
:1081A000C4E901236B78063BDBB223743BB109358C
:1081B000E56070BD002363702374C4E90133E3609C
:1081C00070BD032100236A18093561702374E360D0
:1081D000C4E9012570BD00BF70B50C46C17811F02F
:1081E0003F015CD005461EF06AFF034628466374D3
:1081F0001EF070FFA0742B796370E87883092370F8
:108200002B7913F0010641D14FF0050C4FF00B0E06
:10821000624613F00201666002D005EB0C01724663
:10822000A160590701D50132D2B213F0080102D082
:10823000961CA918F2B2616113F0100102D0D61C8D
:10824000A918F2B2A16113F0200103D002F11206C5
:10825000A918F2B213F04003E16102D0AB18013269
:10826000D2B200F03F002362011D891A11F0FF0114
:1082700014BFAB180B4663626B78013B1B1ADBB271
:10828000237453B10A441544E56070BD4FF00B0CE4
:108290006E1D4FF0110E6246BBE7E36070BD2046D5
:1082A0002822BDE870401AF01BBB00BF70B50678ED
:1082B00006F00F06072E26D00C4605461EF0FFFEE0
:1082C0000346284663741EF005FFA074062E13D8DB
:1082D000DFE806F0041D041204120400002301214B
:1082E000EA1C6170C4E901236B78063BDBB223749E
:1082F0003BB10935E56070BD002363702374C4E9A8
:108300000133E36070BDBDE87040FFF765BF032136
:1083100000236A18093561702374E360C4E90125FC
:1083200070BD00BF0378012B2FD0022B23D003395F
:10833000C9B2A3B1012908D9427800236FF34512CD
:10834000C3610374C360427070474378DA06F3D5A3
:10835000437800226FF3861302624370ECE7012931
:1083600023D94378DB06E7D4437800226FF3C303B5
:1083700042614370DEE743780022033923F00303B0
:108380004260C9B282604370D4E742780023022978
:108390006FF3410283604270CED0D2B203394360A2
:1083A00063F30002C9B24270C4E7427812F0100FC2
:1083B000DAD022F00302C0E90133D3064270C7D4F9
